:020000040800F2
:1000000000000110B11F03084D860208D1770108D6
:10001000B5200308B5200308B52003080000000040
:10002000000000000000000000000000998C0208A1
:10003000958C020800000000918C0208396B0108C1
:10004000B5200308B5200308B5200308B520030830
:10005000B5200308B5200308A972010899730108A7
:10006000B52003085D73010821730108856101084B
:100070007561010865610108556101084561010864
:10008000316101081D610108B5200308B52003088E
:10009000B5200308B5200308B5200308E572010860
:1000A000B5200308B5200308B5200308B5200308D0
:1000B000E5810108B5200308D5810108B5200308B2
:1000C000B5200308B5200308B5200308B5200308B0
:1000D000B5200308B5200308096C01086D6B010801
:1000E0006D720108B5200308B58C0208B52003081D
:1000F000A5810108B5200308B5810108096101083F
:10010000B5200308B5200308C5810108B520030800
:10011000B5200308B5200308B5200308B52003085F
:10012000F5600108E1600108CD600108B9600108CF
:10013000A5600108B5200308B5200308B520030811
:10014000B5200308B5200308B5200308558602082A
:10015000916001087D60010869600108B52003080D
:10016000B5200308B5200308B5200308B52003080F
:10017000B5200308B5200308B5200308B5200308FF
:08018000B5200308B5200308B7
:100188001400020028220020802200200000000025
:100198005C0500080B100C00641E0020842200205F
:1001A800000000005E05000827000400A4230020CA
:1001B80098240020000000006A05000802020300DD
:1001C8009C25002098250020000000000000000069
:1001D800F7010600A8250020A02500200000000047
:1001E8006E05000816000800B0250020B82500207C
:1001F8000000000074050008010104000826002022
:10020800FC2F002000000000000000000802090088
:10021800D42F00200030002000000000BD6301083A
:1002280002000C00E02F00200C300020000000002D
:1002380000000000031232005B380020293800203B
:10024800000000000000000025005A00753700205B
:10025800CF370020000000000000000001000A0065
:1002680094380020A0380020000000007C05000819
:100278001A000800684000207C40002000000000B0
:100288008605000815007000A4390020844000206D
:10029800000000000000000003000100A039002059
:1002A800F440002000000000000000002A00600068
:1002B800B0380020F84000200000000045EC01089C
:1002C800290050007C440020184500200000000050
:1002D800000000001E000400EC460020D448002066
:1002E800000000008E05000822000C00684600206F
:1002F800D84800200000000092050008FC01090011
:100308008454002070550020000000008D740108FE
:100318000A001200E84800207C5500200000000078
:100328009E05000818002C000C5D0020385D002098
:100338000000000041DE0208FD012400E85C002006
:10034800645D0020000000003563010806001A0003
:1003580018580020885D00200000000001EC01080A
:100368003400100044570020A45D00200000000065
:10037800BDEB0108FB01010020560020B45D002000
:1003880000000000C17401080400C000AC70002027
:10039800EC7100200000000000000000F9010400DA
:1003A8003C6E0020AC72002000000000A56301082C
:1003B80003010600FC7200204473002000000000C6
:1003C800B00500080D002C00107C00203C7C0020AB
:1003D80000000000F1AD0108FE010800FC750020D6
:1003E800687C002000000000C974010813000400A4
:1003F800687E0020707E002000000000B80500081C
:1004080010000300647E0020747E002000000000BD
:10041800BC05000828000C00587E0020787E0020CB
:1004280000000000C005000826000800507E0020DB
:10043800847E002000000000CC05000823000E0088
:10044800407E00208C7E0020000000001D0802086D
:1004580019000500387E00209C7E00200000000066
:10046800D4050008F8010100347E0020A47E002095
:1004780000000000DA05000800010400307E0020BA
:10048800A87E002000000000DC0500082C001000F9
:1004980088810020788100200000000091DA02089D
:1004A8002B002400BC81002098810020000000005F
:1004B80061DA02081F000E008882002004830020F1
:1004C80000000000E005000805020100D0820020BD
:1004D8001483002000000000EE0500080500050058
:1004E8007E840020AC84002000000000F005000895
:1004F800120016005A840020B48400200000000076
:10050800F60500080C0024002C840020CC84002070
:1005180000000000C58701080E00DE0030830020BF
:10052800F0840020000000006DEC010802010300C7
:1005380021830020D085002000000000F1860108FA
:100548000002050018830020D48500200000000068
:04055800000000009F
:10055C0003002B21231E0002000001000A012003CE
:10056C000000000001000000C40900001901282847
:10057C000A0AE8030000640001007E05EA05B405E0
:10058C00320000000100C800141E010064002C01A0
:10059C00280000300100005A0000000090012C01DE
:1005AC00C800640004010100000000000801000004
:1005BC000001050000000001000000000000000028
:1005CC0001155802D903C5030000280100000400DE
:1005DC009001000000000000000001000000000578
:1005EC0000000000010103000100000000010000F8
:1005FC0000000000000000000000000000000000EF
:10060C000101000078700308DC9E03080000000064
:10061C0000000000887003089070030800000000C0
:10062C0001200000947003089C7003080000000077
:10063C0001400000A0700308408E03080000000079
:10064C0001200000AC700308B87003080000000023
:10065C0004000000BC700308C87003080000000010
:10066C0004000000CC7003085C8503080000000047
:10067C0001000000020000000000803F0000803FED
:10068C00FF0000000000803F0000803F0000803F22
:10069C0050010000070000000200000000000000F4
:1006AC00000000000102030406070809CC4E0308F1
:1006BC000508040000000000D86B0308746B0308E5
:1006CC00B84E030800000000F84E030805080A00A5
:1006DC0000000000D86B0308746B0308F06B030870
:1006EC0000000000E9840208A1840208F1830208DA
:1006FC0000000000E180020865820208E582020821
:10070C00CD8102080000000000000000D580020826
:10071C00B980020851860208B5800208A980020837
:10072C00A5800208B1800208AD800208C9800208C9
:10073C00BD800208A5810208B981020891810208D6
:10074C007D81020869810208FFFFFFFF0000803FE6
:10075C00910E0208000000000000000001000000E3
:10076C00847E0308000000000000000001870108DF
:10077C00A086010004000000000000000000000042
:10078C00000000000000000000000000000000005D
:10079C0000000000449C03081477030800000000CC
:1007AC0031CD00087D0000000600000000000000B4
:1007BC00000000000000000000000000000000002D
:1007CC0000000000000000009C92030800000000E4
:1007DC0000000000190B0308E803000003000000F0
:1007EC0000000000000000000000000000000000FD
:1007FC00000000000000000000000000A4920308AC
:10080C00000000000000000095D601081027000031
:10081C0003000000000000000000000000000000C9
:10082C0000000000000000000000000000000000BC
:10083C00B0920308000000001DD9020851200108E5
:10084C00204E000005000000000000000000000029
:10085C00000000000000000000000000000000008C
:10086C0000000000D47F030800000000000000001E
:10087C00D50503081027000001000000000000004F
:10088C00000000000000000000000000000000005C
:10089C000000000000000000B492030800000000FB
:1008AC000000000059740108E80300000500000076
:1008BC00000000000000000000000000000000002C
:1008CC00000000000000000000000000C0920308BF
:1008DC000000000000000000E5890108204E000027
:1008EC0003000000000000000000000000000000F9
:1008FC0000000000000000000000000000000000EC
:10090C00D09203080000000000000000ED870108F1
:10091C00204E00000300000000000000000000005A
:10092C0000000000000000000000000000000000BB
:10093C0000000000E092030800000000000000002E
:10094C004D040308400D03000300000000000000EC
:10095C00000000000000000000000000000000008B
:10096C0000000000000000002077030800000000D9
:10097C00000000006DFB02081027000003000000BF
:10098C00000000000000000000000000000000005B
:10099C00000000000000000000000000F0920308BE
:1009AC000000000000000000ADAE0108A0860100B0
:1009BC00010000000000000000000000000000002A
:1009CC00000000000000000000000000000000001B
:1009DC007C6F0308000000000000000081AE0108DD
:1009EC00A00F00000100000000000000000000004B
:1009FC0000000000000000000000000000000000EB
:100A0C0000000000687B03080000000000000000EC
:100A1C0011ED02081027000001000000000000008A
:100A2C0000000000000000000000000000000000BA
:100A3C000000000000000000087703080000000020
:100A4C000000000009AE02081A410000010000007D
:100A5C00000000000000000000000000000000008A
:100A6C00000000000000000000000000F8920308E5
:100A7C000000000000000000CDAD0108400D030097
:100A8C00000000000000000000000000000000005A
:100A9C00000000000000000000000000000000004A
:100AAC00009303080000000000000000D98B01082F
:100ABC00A086010003000000000000000000000000
:100ACC00000000000000000000000000000000001A
:100ADC00000000000000803F000101010101010045
:100AEC0000000000010203040102030406070809C8
:100AFC00010100000403090412010002020200407B
:100B0C008304405700020102030100000902430064
:100B1C00020100C032090400000102020100052498
:100B2C000010010524010001042402020524060022
:100B3C0001070582030800FF09040100020A0000F6
:100B4C00000705010240000007058102400000007B
:100B5C00FF000000D185020811830208C14E020873
:100B6C00258102087D850208358102085181020821
:100B7C001581020805810208000000000000000039
:100B8C00F09603080E000000419B020800000000D4
:100B9C000000000000070020B496030800000000CD
:100BAC00000000000000000000000000DC9E0308B4
:100BBC0000000000000000006C0700200400000092
:100BCC00389603080C00000075A00208C80B002022
:100BDC00000000005C9503080C0000004BA002080C
:100BEC00BC0B002000000000D49603080800000095
:100BFC0000000000B00B002004000000C4960308A5
:100C0C000C000000E99E0208A40B0020000000006C
:100C1C004895030803000000E1AC02088C0B00208F
:100C2C0000000000CC96030803000000E1AC0208B1
:100C3C00740B0020000000004C950308010000001C
:100C4C000000000000000000000000000000000098
:100C5C000D0000000000000000000000000000007B
:100C6C00B496030800000000000000000000000023
:100C7C0000000000DC9E03080000000000000000E3
:100C8C006C07002004000000DC9503080300000042
:100C9C00E19C02085C0B002008000000C4960308CD
:100CAC000C000000E99E0208A40B002000000000CC
:100CBC004895030803000000E1AC02088C0B0020EF
:100CCC0000000000CC96030803000000E1AC020811
:100CDC00740B0020000000004C950308010000007C
:100CEC0000000000000000000000000000000000F8
:100CFC000D000000000000000000000000000000DB
:100D0C00DC9603080000000000000000000000005A
:100D1C0000000000DC9E0308000000000000000042
:100D2C006C07002004000000E49503080300000099
:100D3C00E1AC0208D40B0020000000004C95030825
:100D4C000100000000000000000000000000000096
:100D5C00000000000D00000000000000000000007A
:100D6C000000000000FFFF00000000002D202D2DD2
:100D7C00202D2D2D2D202D2D2D00000000000000EC
:100D8C000000000000000000000000AA5505010052
:100D9C0000AA550B010000AA5507010000AA55092D
:100DAC0002000000AA5503009F0000000100000093
:100DBC00C0122D202D2D202D2D2D2D202D2D2D2D06
:100DCC000000000000000000000000000000000017
:100DDC0000000000BA72002088130C1701000000FC
:100DEC00BC72002088130C1700000000209503082B
:100DFC0000000000000000000000000000000000E7
:100E0C00309503080800000000000000E0070020F7
:100E1C00040000003C9503080800000000000000DE
:100E2C00D4070020000000004895030804000000CF
:100E3C00CDA0020800000000000000004C95030843
:100E4C000100000000000000000000000000000095
:100E5C00000000000D000000000000000000000079
:100E6C0000000000B872002088130C17010000006D
:100E7C00B672002088130C17000000008C95030834
:100E8C000E000000919B0208000000000000000012
:100E9C00EC070020C972002001000000986B0308C9
:100EAC00B572002001000000A46B0308BE72002084
:100EBC0002000000AC6B0308B271002000000000BF
:100ECC0000000000B07100200000000000000000D5
:100EDC00AE7100200000000000000000AC7100208A
:100EEC000000000000000000AA71002000000000BB
:100EFC0000000000A87100200000000000000000AD
:100F0C00B00700200000000000000000B4720020B8
:100F1C0002000000B86B0308949503080000000061
:100F2C0000000000000000000000000030950308E5
:100F3C000800000000000000700800200400000001
:100F4C003C95030808000000000000006408002025
:100F5C00000000004895030804000000719B020883
:100F6C0000000000000000004C9503080100000088
:100F7C000000000000000000000000000000000065
:100F8C000D00000000000000000000000000000048
:100F9C00A495030800000000000000000000000001
:100FAC0000000000B49503080C0000008D9F02089F
:100FBC00AC08002004000000C09503080C000000E1
:100FCC00B59B0208A008002004000000CC95030883
:100FDC000C000000599F020894080020000000003B
:100FEC00D895030803000000019D02087C0800202E
:100FFC0008000000E495030803000000E1AC0208BF
:10100C00D40B0020000000004C95030801000000E8
:10101C0000000000000000000000000000000000C4
:10102C000D000000000000000000000000000000A7
:10103C00EC95030800000000000000000000000018
:10104C0000000000F4950308040000002DA1020824
:10105C0000000000000000004C9503080100000097
:10106C000000000000000000000000000000000074
:10107C000D00000000000000000000000000000057
:10108C004096030800000000000000000000000073
:10109C0000000000509603080C0000000000000047
:1010AC000C090020040000005896030808000000FA
:1010BC0000000000000900200400000064960308F2
:1010CC000800000000000000F408002004000000EC
:1010DC006C9603080800000000000000E8080020DF
:1010EC0004000000749603080800000000000000D3
:1010FC00DC080020040000007C96030808000000B7
:10110C0000000000D00800200400000084960308B2
:10111C000800000000000000C408002004000000CB
:10112C008C9603080800000000000000B80800209E
:10113C00040000004C9503080100000000000000B2
:10114C000000000000000000000000000D00000086
:10115C00000000000000000000000000949603084E
:10116C000E000000819B020800000000000000003F
:10117C00180900209C9603080E00000000000000D7
:10118C00000000000000000090090020A496030855
:10119C000E00000000000000000000000000000035
:1011AC00300A0020CB72002004000000C46B03083E
:1011BC00B0720020E0150C1700000000B372002084
:1011CC0008000000746B0308B272002005000000D8
:1011DC00D86B0308AC9603080E000000000000005A
:1011EC000000000000000000800A0020189B03088B
:1011FC000E000000000000000000000000000000D5
:10120C0050180020FFFFFFFFFA0000000100000053
:10121C0001000000EC950308000000000000000035
:10122C0000000000000000001697030804000000F6
:10123C00EB4B020800000000000000004C95030876
:10124C000100000000000000000000000000000091
:10125C00000000000D000000000000000000000075
:10126C0000000000122200200100C4090000000050
:10127C00102200200100C409000000000E220020F2
:10128C000100C409000000000C2200200100C40968
:10129C0000000000082200200100C409000000002A
:1012AC000A2200200100C4090000000006220020D0
:1012BC000100C40900000000042200200100C40940
:1012CC0000000000389703080E000000000000002A
:1012DC000000000000000000140C002038730020F7
:1012EC009CFF2C0100000000DC0400200A00000020
:1012FC00F06B0308CC720020E0150C170000000006
:10130C00DD04002008000000746B0308DE040020DC
:10131C0005000000D86B03089F5500200200000058
:10132C00086C0308848400200120010083840020C1
:10133C0002000000146C0308168400200000F40165
:10134C0001000000148400200000F40101000000E2
:10135C00128400200000F401010000001084002021
:10136C000000F401010000000E84002000FF0100C9
:10137C002A840020E803D0070A00000028840020FB
:10138C00006401000A0000002984002000640100B0
:10139C000A00000022840020006401000A00000002
:1013AC0027840020006401000A000000268400202D
:1013BC00006401000A000000258400200064010084
:1013CC000A0000002184002000FF01000A00000038
:1013DC002084002000FF01000A0000002C83002064
:1013EC000000F401010000002A8300200000F40139
:1013FC0001000000288300200000F401010000001F
:10140C00268300200000F401010000001D84002050
:10141C0000C801001C84002000C801001B840020AF
:10142C0000C801001A840020006401000A000000BA
:10143C001984002000FF01000A00000059840020DC
:10144C0000C801005884002000C801005784002007
:10145C0000C801005684002000C8010055840020FB
:10146C0000C801005484002000C8010053840020EF
:10147C0000C801005284002000C8010051840020E3
:10148C0000C80100409703080000000000000000A5
:10149C000000000000000000509703080900000045
:1014AC0000000000B80C002004000000589703084E
:1014BC000900000000000000AC0C0020040000003B
:1014CC00D49903080900000000000000A00C0020C3
:1014DC0004000000609703080900000000000000F1
:1014EC00940C00200400000064970308090000001D
:1014FC0000000000880C0020040000006C9703081A
:10150C0009000000000000007C0C0020040000001A
:10151C00749703080900000000000000700C002004
:10152C00040000007C970308090000000000000084
:10153C00640C0020040000004C950308010000001E
:10154C00000000000000000000000000000000008F
:10155C000D00000000000000000000000000000072
:10156C008497030800000000000000000000000049
:10157C0000000000DC9E03080000000000000000DA
:10158C00B207002004000000909703080C00000034
:10159C00A54B0208180D0020000000003896030827
:1015AC000C000000994C02080C0D002000000000FB
:1015BC005C9503080C0000007D4C0208000D002017
:1015CC0000000000D4960308080000000000000092
:1015DC00F40C002004000000C49603080C0000006A
:1015EC00614B0208E80C00200000000094970308EF
:1015FC000900000000000000DC0C002004000000CA
:10160C004895030803000000E1AC0208C40C00205C
:10161C00000000004C9503080100000000000000D1
:10162C000000000000000000000000000D000000A1
:10163C000000000000000000000000009C97030860
:10164C00000000000000000000000000000000008E
:10165C00AC9703080C000000000000002C0D0020CB
:10166C0000000000B49703080A000000000000000E
:10167C008584002000000000C09703080A000000C9
:10168C00000000008D84002000000000C8970308B3
:10169C000A000000000000009584002000000000FB
:1016AC00D09703080700000000000000240D002064
:1016BC00000000004C950308010000000000000031
:1016CC000000000000000000000000000D00000001
:1016DC00000000000000000000000000DC97030880
:1016EC0000000000000000000000000000000000EE
:1016FC00F09703080700000000000000680D0020B0
:10170C0000000000FC970308080000000000000027
:10171C005C0D002000000000089803080800000081
:10172C0000000000500D0020000000001498030879
:10173C000800000000000000440D00200000000024
:10174C00209803080800000000000000380D00205D
:10175C00000000004C950308010000000000000090
:10176C000000000000000000000000000D00000060
:10177C000000000000000000000000002C9803088E
:10178C000000000000000000CB1A00200000000048
:10179C00389803080B00000000000000D00D00205A
:1017AC0000000000409803080B000000000000003F
:1017BC00C40D0020000000004C9803080B00000032
:1017CC0000000000B80D002000000000589803082D
:1017DC000B00000000000000AC0D00200000000019
:1017EC00649803080B00000000000000A00D00200E
:1017FC0000000000709803080B00000000000000BF
:10180C00940D002000000000789803080B000000E5
:10181C0000000000880D00200000000084980308E0
:10182C000B000000000000007C0D002000000000F8
:10183C00909803080800000000000000700D0020C4
:10184C00000000004C95030801000000000000009F
:10185C000000000000000000000000000D0000006F
:10186C000000000000000000000000009C9803082D
:10187C00000000000000000000000000000000005C
:10188C00B09803080800000000000000000E0020C3
:10189C0000000000BC9803080800000000000000D5
:1018AC00F40D002000000000C89803080800000098
:1018BC0000000000E80D002000000000D498030890
:1018CC000800000000000000DC0D002000000000FB
:1018DC004C9503080100000000000000000000000F
:1018EC0000000000000000000D00000000000000DF
:1018FC000000000000000000DC980308000000005D
:10190C0000000000C81A002000000000EC9803083A
:10191C000B00000000000000300E00200000000052
:10192C00F89803080B00000000000000240E0020B3
:10193C0000000000049903080700000000000000EC
:10194C001C0E002000000000109903080700000086
:10195C0000000000140E0020000000001C99030879
:10196C0007000000000000000C0E0020000000002A
:10197C004C9503080100000000000000000000006E
:10198C0000000000000000000D000000000000003E
:10199C00000000000000000028990308000000006F
:1019AC0000000000C81A0020000000003499030851
:1019BC0007000000000000007C0E0020000000006A
:1019CC003C9903080700000000000000740E002082
:1019DC00000000004499030807000000000000000C
:1019EC006C0E0020000000004C990308070000005A
:1019FC0000000000640E0020000000005499030851
:101A0C0007000000000000005C0E00200000000039
:101A1C005C9903080700000000000000540E002031
:101A2C00000000006499030807000000000000009B
:101A3C004C0E0020000000006C9903080700000009
:101A4C0000000000440E0020000000007499030800
:101A5C0007000000000000003C0E00200000000009
:101A6C004C9503080100000000000000000000007D
:101A7C0000000000000000000D000000000000004D
:101A8C0000000000000000007C9903080E0000001C
:101A9C000000000061F9020800000000840E002024
:101AAC00258300200A3201002483002001FA010062
:101ABC002083002000C801001E830020E803D0070B
:101ACC0001000000454C4C4530000000849903088F
:101ADC000E000000254C0208000000000000000071
:101AEC00600F00208C9903080E00000029000308E9
:101AFC000100030869FB02083C10002094990308BC
:101B0C000E000000EDF90208BDF90208000000000B
:101B1C00DC1000209C9903080E00000065FA0208F6
:101B2C00A9FA0208000000007C1100201E8400208D
:101B3C0001030100A89903080E00000099F902089E
:101B4C0077F90208000000006C120020B09903081D
:101B5C000E0000001DFA020833FF0208000000000E
:101B6C00F8120020BC9903080E000000D5FA0208F8
:101B7C007DFF02080000000098130020188400204C
:101B8C0001030100C49903080000000000000000DC
:101B9C000000000000000000D099030808000000BD
:101BAC0000000000B814002000000000D8990308C1
:101BBC000700000000000000B0140020000000002E
:101BCC00E89903080700000000000000A81400209A
:101BDC0000000000F499030807000000000000005A
:101BEC00A014002000000000009A0308030000006D
:101BFC00E1AC020888140020000000004C9503089A
:101C0C0001000000000000000000000000000000C7
:101C1C00000000000D0000000000000000000000AB
:101C2C0000000000089A03080000000000000000FB
:101C3C000000000000000000189A03080A000000D1
:101C4C0000000000906E030800000000209A0308BA
:101C5C000A00000000000000289A030800000000A1
:101C6C00309A03080A000000000000007084002075
:101C7C0000000000389A03080A0000000000000071
:101C8C00C4140020000000004C9503080100000063
:101C9C000000000000000000000000000000000038
:101CAC000D0000000000000000000000000000001B
:101CBC00409A030800000000000000000000000033
:101CCC0000000000B06F030803000000E1AC020844
:101CDC00E414002000000000549A030803000000E4
:101CEC00E1AC020880050020000000005C9A0308AB
:101CFC0003000000E1AC0208CC140020000000003E
:101D0C004C950308010000000000000000000000DA
:101D1C0000000000000000000D00000000000000AA
:101D2C000000000000000000649A0308000000009E
:101D3C00000000000000000000000000709A030882
:101D4C0007000000C9FF02087C15002000000000FD
:101D5C00449C030803000000E1AC02086415002059
:101D6C00000000007C9A030803000000E1AC0208AC
:101D7C004C15002000000000849A030803000000AA
:101D8C00E1AC020834150020000000008C9A030816
:101D9C0007000000ADFF02082C1500200000000019
:101DAC005C96030803000000E1AC02081415002047
:101DBC0000000000989A030803000000E1AC020840
:101DCC00FC140020000000004C95030801000000EA
:101DDC0000000000000000000000000000000000F7
:101DEC000D000000000000000000000000000000DA
:101DFC00A49A03080E00000035F9020807F902083E
:101E0C000000000084150020AC9A03080E000000AE
:101E1C003DFB02080000000000000000241600201A
:101E2C00B89A03080E00000000000000000000003B
:101E3C0000000000B0160020C89A03080E00000035
:101E4C0019FB0208E5FF020800000000281700201B
:101E5C00D09A030800000000000000000000000001
:101E6C0000000000DC9A030803000000E1AC02084B
:101E7C003818002000000000BC9A03080300000082
:101E8C00E1AC02082018002000000000E49A0308CE
:101E9C0003000000E1AC020808180020000000005C
:101EAC00F09A030803000000E1AC0208F0170020D0
:101EBC0000000000F89A030802000000EDAB0208D5
:101ECC000000000000000000009B0308020000005E
:101EDC00EDAB020801000000000000000C9B0308A1
:101EEC0002000000EDAB0208020000000000000040
:101EFC00000000000D0000000000000000000000C9
:101F0C000000000000600240106002400000000071
:101F1C00000B00000000200000000000000000008A
:101F2C00006002402860024000000000060C000027
:101F3C0000002000000000000000000000600240D3
:101F4C004060024000000000100D00000000200066
:101F5C0000000000000000000060024058600240D9
:101F6C0000000000160E0000000020000000000021
:101F7C0000000000006002407060024000000000A1
:101F8C00200F0000000020000000000000000000F6
:101F9C000060024088600240000000002610000033
:101FAC000000200000000000000000000060024063
:101FBC00A060024000000000301100000000200072
:101FCC00000000000000000000600240B860024009
:101FDC0000000000362F0000000020000000000070
:101FEC000000000000640240106402400000000089
:101FFC00003800000000400000000000000000005D
:10200C000064024028640240000000000639000011
:10201C0000004000000000000000000000640240CE
:10202C004064024000000000103A00000000400034
:10203C0000000000000000000064024058640240F0
:10204C0000000000163B00000000400000000000F3
:10205C0000000000006402407064024000000000B8
:10206C00203C0000000040000000000000000000C8
:10207C000064024088640240000000002644000016
:10208C00000040000000000000000000006402405E
:10209C00A064024000000000304500000000400039
:1020AC00000000000000000000640240B864024020
:1020BC000000000036460000000040000000000058
:1020CC00000000000101010120700020702D720041
:1020DC0043000000000000000000000000000000B1
:1020EC0000000000000000000000000000000000E4
:1020FC004300000000000000000000000000000091
:10210C0000000000000000000000000000000000C3
:10211C004300000000000000000000000000000070
:10212C0000000000000000000000000000000000A3
:10213C004300000000000000000000000000000050
:10214C000000000000000000000000000000000083
:10215C004300000000000000000000000000000030
:10216C000000000000000000000000000000000063
:10217C004300000000000000000000000000000010
:10218C000000000000000000000000000000000043
:10219C0043000000000000000000000000000000F0
:1021AC000000000000000000000000000000000023
:1021BC00BD22030815210308000000005A9F0308E4
:1021CC00119703081F9403081F9403081F94030816
:1021DC001F9403081F9403081F9403081F940308FB
:1021EC001F9403081F940308FFFFFFFFFFFFFFFF6F
:1021FC00FFFFFFFFFFFF000001004153434949006F
:10220C0000000000000000000000000000000000C2
:10221C000000000000000000000041534349490049
:10222C0000000000000000000000000000000000A2
:10223C00000000000000000000000000401C002016
:10224C000000000000000000000000000000000082
:10225C000000000000000000000000000000000072
:10226C000000000000000000000000000000000062
:10227C000000000000000000000000000000000052
:10228C000000000000000000000000000000000042
:10229C000000000000000000000000000000000032
:0422AC00010000002D
:108000002DE9F04FB0F908502DED048B0D81EDB244
:10801000382D8FB00C4600F08D8480462ED9802DEF
:1080200000F0E48078D8522D00F0948040F2748201
:10803000542D00F0C8846E2D40F02081814B0A68D9
:108040001B88814DFF2BA8BFFF23511C216013709B
:10805000A96881F3100189B220460DF091F87B4B9D
:10806000204619880DF08CF8296801F30F0189B2B8
:1080700020460DF085F801252B4646E0042D60D002
:1080800040F20182202D00F0958040F23082242DB4
:1080900000F09284282D40F0F1800B68DFF8D08149
:1080A0006B4E591C022221601A70236806275A1C45
:1080B00022601F7023680A22591C21601A702368ED
:1080C00001255A1922601D70B8F8001020460DF0E5
:1080D00057F8B8F8021020460DF052F823685A19E4
:1080E00022601F7023685022591921601A7023687A
:1080F0000022591921601A70318820460DF040F88D
:10810000718820460DF03CF82B46284663810FB05D
:10811000BDEC048BBDE8F08F822D23D0C0F06C84C1
:10812000A02D00F05D84FE2D40F0A880494D05F1A2
:10813000080635F8021B20460DF022F8B542F8D1AA
:1081400099E72A46444920460CF0D2FF00212046F8
:108150000DF016F822680021531C012523602B46E0
:108160001170D2E70B683D4A374D11783C4A581CD4
:1081700020601970D18820460DF002F8314B22683A
:108180001B88FF2B02F10101A8BFFF2321601370A0
:10819000A96881F3100189B220460CF0F1FF29682B
:1081A00001F30F0189B220460CF0EAFF2D4B226843
:1081B0001978D1E70B682A4D591C6A7821601A702A
:1081C00023682A78591C21601A702368AA78591CE0
:1081D00021601A70E98820460CF0D2FF23682A79C2
:1081E000591C21601A7022686979B5E7DFF884802C
:1081F0001D4F1E4EDFF880A008F10D090A2517E07B
:10820000322D00F05881A5F13C00C0B2132840F295
:10821000588100232268511C216015702268C845CE
:1082200002F10101216013703FF425AF18F8015BE2
:108230000A2DE5D1BAF80030FF2BA8BFFF23DBB22F
:10824000E8E700BFA0820020A48200208020002058
:1082500008260020F4810020986E0308DF820020A9
:10826000641E0020C41E002067666666202600206B
:10827000307E0020E147030850260020A5F10A03C4
:10828000E72B00F2EA80DFE813F00F09E800E800CE
:10829000E800E800E800E800E800E800E800E8009E
:1082A000E800E800E800E800E800E800E800E8008E
:1082B000E800E800E800E800E800DE08E800E80080
:1082C000E800CD08E800E800E800C808E8008708F2
:1082D000E800E800E800E800E8008208E8005C0840
:1082E000E8004908E800E800E80055048509E800CE
:1082F0007B09E800E8007209E800E800E800E8000F
:10830000E8004804E800E800E800E8005609E80052
:108310003409E80021093108E800E800E800E80035
:10832000E800E800E800ED07E8009607E8006707C6
:10833000E8001D07E8000C07E800E800E800E80096
:10834000E306B006A7067F066D0621060B06F205BA
:10835000E605E800AC051305E800E800E800E800E1
:108360000705E800E800E504E800E800E800AC04E0
:1083700093048204E800E800E800E80071045D046A
:10838000A105E800E800E800E800E800E800E800EF
:10839000E800E800E800E800E800E800E800E8009D
:1083A000E800E306E800E800E800E800E800E8008C
:1083B000E800E800E800E800E800E800E8006805F8
:1083C000E800E800E800E800E800E800E800E8006D
:1083D000E800E800E800E800E800E800E800E8005D
:1083E000E800E800E800E800E800E800E800E8004D
:1083F000E800E800E800E800E800E800E800E8003D
:10840000E800E800E800E800E800E800E800E8002C
:10841000E800E800E800E800E800E800E800E8001C
:10842000E800E800E800E800E800E800E800E8000C
:10843000E800E800E800E800E800E800E800E800FC
:10844000E800E800E800E800E800E800E800E800EC
:10845000E800E800E8005B053005742D00F0238398
:10846000772D6FD1D8F80030D8F804209A421EBF7B
:108470005A1CC8F8002019782D4A08BF0021204650
:108480000FF038F9F7E5022D00F08D8200F27982C5
:10849000012D7FF4F3AE0B680022591C21601A7085
:1084A00023685A1C22601D7022682421531C2360FB
:1084B0002B46117029E63388FF2BA8BFFF23DBB2C0
:1084C000A8E626F06FFF00283FF4A3AE03780A2B3E
:1084D00000F2FB82B0F9023087FB0312DB17C3EB1B
:1084E000A2039BB2FF2BA8BFFF23DBB292E6052DB0
:1084F0007FF4C4AE0B220F4920460CF0F9FD082290
:108500000D4920460CF0F4FD012507220B492046B9
:108510000CF0EEFD2B46F8E5442D7FF4AFAE002ABB
:108520003FF4A9AD064B136001252B46EDE500BFD6
:108530004D740108A06E0308AC6E0308B86E030802
:1085400001750108762D00F0C282292DD8F800307F
:1085500001F03086392D01F04580212D01F0038690
:10856000D8F804600B3DF61AEF2D01F2518001A2FC
:1085700052F825F0FF98000811960008119600089F
:10858000119600081196000811960008119600082F
:10859000119600081196000811960008119600081F
:1085A000119600081196000811960008119600080F
:1085B00011960008119600081196000811960008FF
:1085C00011960008119600081196000811960008EF
:1085D00011960008919800081196000877980008F5
:1085E0001196000855980008119600081196000889
:1085F00011960008779B000811960008C19A0008A0
:1086000011960008119600081196000811960008AE
:10861000119600088B9B0008119600085F9A0008CD
:1086200011960008199A0008119600081196000882
:10863000119600081196000877800008119600082E
:10864000F99900081196000811960008DD990008B4
:10865000119600081196000811960008119600085E
:10866000119600081196000811960008119600084E
:1086700011960008119600089199000811960008BB
:10868000579F00081196000811960008239F0008C4
:10869000119600081196000811960008119600081E
:1086A0001196000811960008119600084D9E0008CA
:1086B00011960008C79D000811960008679D0008E4
:1086C00011960008019D000811960008899C000879
:1086D00011960008119600081196000811960008DE
:1086E00011960008119600081196000811960008CE
:1086F00011960008119600081196000811960008BE
:1087000011960008119600081196000811960008AD
:10871000119600081196000811960008119600089D
:10872000119600081196000811960008119600088D
:10873000119600081196000811960008119600087D
:10874000119600081196000811960008119600086D
:10875000119600081196000811960008119600085D
:10876000119600081196000811960008119600084D
:10877000119600081196000811960008119600083D
:10878000119600081196000811960008119600082D
:10879000119600081196000811960008119600081D
:1087A000119600081196000811960008119600080D
:1087B00011960008119600081196000811960008FD
:1087C00011960008119600081196000811960008ED
:1087D00011960008119600081196000811960008DD
:1087E00011960008119600081196000811960008CD
:1087F00011960008119600081196000811960008BD
:1088000011960008119600081196000811960008AC
:10881000119600081196000811960008119600089C
:10882000119600081196000811960008119600088C
:10883000119600081196000811960008119600087C
:10884000119600081196000811960008119600086C
:10885000119600081196000811960008119600085C
:1088600011960008119600082F9C000841A00008EE
:10887000DB9F00081196000897A00008AD9D000836
:10888000BF9F000811960008A59F0008C59B00081F
:108890009B9B000843980008E39700081196000886
:1088A000BB970008119600081196000899970008D8
:1088B0006597000851970008239700081196000853
:1088C00001970008CD960008B5960008119600089B
:1088D00011960008119600081196000811960008DC
:1088E00011960008119600081196000811960008CC
:1088F00011960008119600081196000811960008BC
:10890000119600089B960008119600081196000821
:108910003396000811960008119600081196000879
:10892000119600081196000811960008119600088B
:108930001B9600080A68B34B0125511C2160157075
:108940002268052150192060117022680A215019EF
:108950002060117022680021501920601170226877
:1089600019785019206011702268597850192060C8
:10897000117022689978531923602B461170FFF704
:10898000C4BB0B680222591C21601A7023680125A0
:108990005A1922601D7022680021531923602B464A
:1089A0001170FFF7B2BB04229749204601250CF055
:1089B0009FFB2B46FFF7A9BB944B196820460CF090
:1089C000C7FBFFF758BB0B6800215A1C22601970C7
:1089D00022680125531923602B461170FFF795BBC0
:1089E0008B4B084619680CF0B3FB8A4B204619687C
:1089F0000CF0AEFB884BE0E7DFF85492874F09F1AB
:108A00000E064FF00A081DE0B8F1500F32D0B8F151
:108A1000320F31D0A8F13C00C0B213282FD9002565
:108A2000294623685A1C2260204683F800800CF0F7
:108A3000A7FB294620460CF0A3FB4E453FF41BAB99
:108A400019F8018BB8F10A0FDED1754B9D681968D2
:108A500005EB85054FF6FF736D009D42A8BF1D46CF
:108A60009942A8BF194625EAE57521EAE171ADB240
:108A700089B2D6E76B4BE9E797E82200E8E726F0F2
:108A800091FC0028CBD003780A2BC8D8B0F9043069
:108A9000B0F9061003EB830383F3500521EAE1717B
:108AA000ADB289B2BDE7D8F80030D8F804209A42B8
:108AB0001EBF5A1CC8F8002019785B4A08BF002165
:108AC00020460EF017FEFFF7D6BA00230DE5D8F8C2
:108AD00000305A1CC8F800201B78002B01F02884B5
:108AE000102B07BF514A92E8220000252946226830
:108AF000501C2060137020460CF02AFB29462046AB
:108B00000CF026FB4A4B204699680CF021FB002113
:108B100020460CF035FBFFF719BB236800255A1CD3
:108B20002260294620461D700CF012FB2946204683
:108B30000CF00EFB0021204601250CF009FB2B4612
:108B4000FFF7E3BA22683B4B501C19782060117084
:108B500022685978501C2060117022689978501C46
:108B6000206011702268D978FFF7F6BA324D20469E
:108B7000A98A0CF005FBE98A20460CF001FB298B41
:108B8000204601250CF0FCFA2B46FFF7BEBA2368FD
:108B90002A4A2B4910782B4A5D1C256018702368DF
:108BA0009278581C20601A7022688978FFF7D4BA2E
:108BB0002268254B25491878551C256010702268BD
:108BC0005878551C2560107022689B78501C2060D6
:108BD0001370C988204601250CF0D2FA2B46FFF706
:108BE00094BA1A4D204629880CF0CAFA69882046A2
:108BF0000CF0C6FAA988204601250CF0C1FA2B46D4
:108C0000FFF783BA21830020906E0308687E00205E
:108C1000107AFF1F147AFF1F187AFF1F18260020F2
:108C2000CC2500200C260020D974010888250020BE
:108C3000A41C0020EC46002018580020E848002022
:108C4000587E0020407E0020387E002068400020B2
:108C5000D1470308B04D05F16006A98820460CF005
:108C60008FFAE98820460CF08BFA298920460CF00F
:108C700087FA2368AA7A591C21601A702368EA7A55
:108C8000591C21601A7055F80C1B20460CF060FA34
:108C9000B542E2D1FFF7EFB9A04952232268501C38
:108CA0002060137011F8013F002BF7D1FFF7E3B9F3
:108CB0009B4D00232268286803EB4301561C405C4F
:108CC000266010702A6820680A44461C5278266084
:108CD00002702A6820680A4401339278411C0A2BEA
:108CE00021600270E6D1FFF7C6B98E4B03F1700523
:108CF00022681978501C2060117022685978501C25
:108D00002060117022689978501C206011702268D0
:108D1000D978501C2060117022681979501C20608D
:108D2000117022685979501C20601170226899795D
:108D30000733501C9D4220601170D9D1FFF79BB9B9
:108D4000794D2046A9890CF01BFA69892046012536
:108D50000CF016FA2B46FFF7D8B92368DFF800C2EB
:108D6000591C9CF8002021601A709CF80030002BE0
:108D70003FF481A96D4E6E4D6E486F490023226805
:108D800016F8017F02F1010EC4F800E017702268A6
:108D900015F8017F02F1010EC4F800E01770226897
:108DA00010F8017F02F1010EC4F800E0177022688C
:108DB00011F8017F02F1010EC4F800E017709CF871
:108DC000002001339342DADBFFF755B95B4B5C4976
:108DD000B3F9003081FB0321DB17C3EBA101FFF7DF
:108DE00046B9584D23682A68591C127821601A70B8
:108DF0002B6822689978531C2360002311702A681D
:108E000021681A4401335279481C032B20600A70F0
:108E1000F5D123682A68591C127A21601A702368D8
:108E20002A68591CD27821601A7023682A68591C54
:108E3000127921601A702B68204659890CF0A0F92C
:108E400023682A68591C527A21601A702B6822689C
:108E50005978FFF781B9002120460CF079F90125F6
:108E6000002120460CF08CF92B46FFF74EB9364D09
:108E7000204629880CF084F9698820460CF080F996
:108E8000B5F904302E49DA1781FB0313C2EBA303B3
:108E900099B2204601250CF073F92B46FFF735B93E
:108EA0002A4B204619880CF06BF9294B204619886B
:108EB0000CF066F9274B21681A7801254B1C02F04B
:108EC000010223602B460A70FFF71FB9224B22686C
:108ED0001B78224D511C03F002032160137023689C
:108EE0002A78591C21601A70696820460CF030F904
:108EF000A96820460CF02CF9A98920460CF040F90D
:108F0000698A20460CF03CF9A98A204601250CF01C
:108F100037F92B46FFF7F9B8B0380020A04703080F
:108F200048200020A4390020407E00200747002070
:108F3000174700203747002027470020587E002091
:108F4000676666664C2000205C1E0020F41E002030
:108F5000F61E0020D8450020721E0020741E00203E
:108F600005470020A94E3378002B3FF484A8A84F72
:108F7000002537F8021F20460CF002F9337801353E
:108F80009D42F6DBFFF777B8A24DA34EDFF8C8820B
:108F9000DFF8C892DFEDA18ADFEDA19A9FEDA19ADB
:108FA00005F1200708E0204604350CF0E9F8AF424F
:108FB00006F118063FF45FA8717C0029F3D095ED07
:108FC000008AB0EE480A29F01FFA98F80030002B0A
:108FD00041F0DC8181B2E6E7102293492046012569
:108FE0000CF086F82B46FFF790B8904E338AB3F515
:108FF000007F06F1340594BF01270427403655F859
:10900000041B91FBF7F1204689B20CF0B9F8AE428F
:10901000F5D1874D874F05F10C06B5EC010AD7ED68
:10902000087A80EE270A29F0EFF981B220460CF089
:10903000A7F8AE42F1D1804D05F10C0655F8041B9E
:10904000204689B20CF09CF8B542F7D1FFF713B86F
:109050000DF1140900220592DFF804A2774B039268
:109060000492C9F80420904601214FF6FF7B07E0E7
:1090700008F10108B8F10B0F01F0B4801AF9011FD3
:109080004E1CF5D04BFA08F2D007F1D51A8842FAF7
:1090900008F2D207ECD5484601930CF0F3FB019B94
:1090A000E6E72368664A6749D078674A5D1C256011
:1090B000187023681278581C20601A702268C978CA
:1090C000FFF74AB8002120460CF05AF8002120464C
:1090D0000CF056F8002120460CF052F822685B4D47
:1090E0000023511C2160137022682968501C91F8DC
:1090F0002F102060117022682968501C91F83A10D6
:109100002060117022682968501C91F83B10206083
:1091100011702268511C216013702268511C21605B
:1091200013702268511C216013702B682046D98F60
:109130000CF026F82B682046998F0CF021F8236854
:109140002A68591C92F8312021601A702B68226815
:1091500093F83210FFF700B83D4D23686A793B4E13
:10916000591C21601A7033682046198C0CF008F8DD
:1091700033682046598C0CF003F8698920460BF0BF
:10918000FFFFA98920460BF0FBFF33682046998C2E
:109190000BF0F6FF33682046D98C0BF0F1FFE9891C
:1091A00020460BF0EDFF298A204601250BF0E8FF51
:1091B0002B46FEF7AABF264EF378002B01F0AB80BA
:1091C00023680822591C21601A702368012299180B
:1091D00021601A7023681F4D591C2A7921601A706A
:1091E0002368AA78591C21601A70298820460BF040
:1091F000C7FF698A20460BF0C3FF2368F279591C28
:1092000021601A702268E978FEF7A6BFF8210020D5
:109210000222002044440020245600200000404246
:109220000040744400E0824434440020181E0020B2
:1092300024510020FC480020244400204420002029
:10924000407E0020587E0020507E002048200020D4
:10925000E84800201858002040580020386E0020B0
:10926000F047030827F0CAF8FF28064601F0B68049
:109270000EA9002501F82E5D0DF109008DF80950A9
:1092800020F096F90EA800F82D5D20F085F90EA8C3
:1092900000F82C5D20F074F90EA820F8245D27F06A
:1092A0008DF823685A1C22601E7023689DF80920DF
:1092B000591C21601A7023689DF80A20591C2160EE
:1092C0001A7023689DF80B20591C21601A702368BE
:1092D0009DF80C20591C21601A70BDF8141020460E
:1092E00001250BF04DFF2B46FEF70FBF2268AE4B5A
:1092F0000125511C21601570226899785019206051
:1093000011702268197850192060117022685978FC
:10931000531923602B461170FEF7F7BEA34DA44EE0
:1093200005F1280795F902100023F2568A4200F051
:10933000FC860C333C2BF8D10835AF42F2D1FEF756
:109340009ABE9C4B03F15A0522685979501C206043
:10935000117022681978501C2060117022685978A9
:10936000501C2060117022689978501C2060117088
:109370002268D978501C2060117022681979063350
:10938000501C9D4220601170DED1FEF774BE8A4BE6
:109390002268597DFEF7E0BE874D23682A7A591C62
:1093A00021601A70A98B20460BF0EAFE298B20461B
:1093B0000BF0E6FE698B20460BF0E2FE2368EA7CA8
:1093C000591C21601A70E98C20460BF0D9FE298DBA
:1093D00020460BF0D5FE2368AA7F591C21601A7025
:1093E000236895F82020591C21601A70A98C20460A
:1093F0000BF0C6FE2368EA7A591C21601A70E968EE
:1094000020460BF0A5FE23682A7C591C21601A70A7
:10941000226895F82110FEF79FBE684B22681978E4
:10942000FEF79ABE664D204629880BF0A9FEA98852
:1094300020460BF0A5FE2989204601250BF0A0FE51
:109440002B46FEF762BE5F4D5F4F05F150060021CF
:1094500028785E4A0B4607E00133242B02F10C0208
:1094600000F0608612F80C1C8842F5D103EB430330
:10947000226807EB8303511C93F86430216013705A
:1094800023686A78591C21601A702368AA78591CCD
:1094900021601A702368EA780435591CAE422160B5
:1094A0001A70D4D1FEF7E7BD494828F0C3F8002868
:1094B0007EF7E1AD464B1D18226813F8011B501CC6
:1094C0009D4220601170F7D1FEF7D5BD23680025BD
:1094D0005A1C22601D7023685A1C22601D7023686C
:1094E0005A1C226029461D7020460BF031FEFFF702
:1094F00021BB384E3378002B3EF4BDAD364F0025EE
:10950000B846236817F81520591C21601A7098F87E
:10951000011001EB810101EB810101F2EE2189B221
:1095200020460BF02DFE337801359D4208F10208EC
:10953000E7DBFEF7A0BD2368284D591C2A7821607F
:109540001A7023686A78591C21601A70698820464D
:109550000BF016FE23682A79591C21601A70E988DD
:1095600020460BF00DFE2268297AFEF7F5BD082291
:109570001149204601250BF0BBFD2B46FEF7C5BD6A
:109580002268174B501C9978206011702268597816
:10959000FEF7E2BD22680121531823600D460B46F9
:1095A0001170FEF7B2BD00BF7E840020107C002049
:1095B000AC5C0020753700200C5D002028220020C4
:1095C000E02F00207C440020A0470308084803083F
:1095D0005F840020F8210020BC8100209438002006
:1095E000647E00205A1CC8F800201A780A2A0FD17D
:1095F0009A1CC8F80020D04A59781170D91CC8F8B4
:10960000001099785170191DC8F80010DB7893701C
:109610004FF0FF352B46FEF778BDC84B1B78DB07B4
:10962000F6D401250EF006F90EF08EF92B46FEF762
:109630006CBD5A1CC8F800201A780F2AE8D8991C6B
:10964000C8F80010C2EBC202BD4958788854D81C33
:10965000C8F800000A4499785170191DC8F8001024
:10966000D9789170591DC8F800101979D170991DD9
:10967000C8F8001059791171D91DC8F800109979EE
:10968000517103F10801C8F80010DB7993710125CD
:1096900015F0D2FE2B46FEF738BD40460BF01CFD00
:1096A000A84EB08140460BF017FD012570812B4676
:1096B000FEF72BBD40460BF00FFDA34A00EB8000E8
:1096C0004300012513802B46FEF71FBD19465A1C87
:1096D000C8F800209D4A11F8020B1070C8F800105D
:1096E00059785170D91CC8F8001099789170191DDB
:1096F000C8F80010DB78D37001252B46FEF705BDB6
:1097000040460BF0E9FC924EB08240460BF0E4FC80
:10971000F08240460BF0E0FC012530832B46FEF73B
:10972000F4BC1A46591CC8F800108A4912F8020BFA
:109730000870C8F8002083495A788A70DA1CC8F883
:109740000020814A9B78937001252B46FEF7DDBCF3
:10975000814B824918684A2201252AF048FF2B468E
:10976000FEF7D3BC19465A1CC8F800207C4A11F8F1
:10977000020B1070C8F8001059785170D91CC8F845
:1097800000109B78937040460BF0A6FC754B0125AA
:10979000D8802B46FEF7B9BC40460BF09DFC714EBD
:1097A000308040460BF098FC708040460BF094FCF3
:1097B0000125B0802B46FEF7A8BC6B4F3B78002BF1
:1097C0003EF459AC694E002540460BF085FC16F07E
:1097D000E5FA3B78A6EC010A01359D42F4DBFEF781
:1097E0004ABC0F2E7FF414AF5A1CC8F800201D7815
:1097F000072D3FF60DAF5E4F40460C260BF06CFC7C
:1098000006FB05F6BD19A88040460BF065FCE88014
:1098100040460BF061FCD8F8003028811A46591CEC
:10982000C8F8001012F8021BA972C8F800205B7873
:10983000EB7240460BF038FC0125B8512B46FEF781
:1098400064BC40460BF048FC4A4B012518802B466F
:10985000FEF75BBC40460BF03FFC474E3060404695
:109860000BF03AFC706040460BF036FC0125B0600E
:109870002B46FEF74ABC414E0023336040460BF0B6
:1098800013FC33680125034333602B46FEF73DBCD0
:109890005A1CC8F80020187813283FF6B9AE9A1C55
:1098A000C8F800205D78364A002105E001312429FE
:1098B00002F10C023FF4ACAE167AAE42F6D1314D55
:1098C000314A0C2606FB0151DD1C91F85C1002F8B0
:1098D0002010C8F8005002EB800299785170191DD1
:1098E000C8F80010D8789070581DC8F800001A49C0
:1098F0001B790868D3701CF0CFFEFEF7BCBB234B6E
:10990000102E4FF0000228BF10261A605A609A608D
:10991000DA601A74002E3EF4AEABD8F8002016447C
:109920000132C8F8002012F8011C03F8011BB242F2
:10993000F6D1FEF7A0BB00BF21830020B455002064
:10994000A4390020407E0020587E0020EC460020F4
:1099500018580020E84800204820002068610308CB
:10996000387E0020684000206C710020703F00208D
:10997000B0380020E4460020E02F0020687E002060
:10998000FC470308A04703087C4400205F840020B4
:109990001A46591CC84DC8F8001012F8021B29704D
:1099A000C8F800205B786B7040460BF095FBD8F848
:1099B000003068805A1CC8F800201B782B71404684
:1099C0000BF08AFBD8F80030E8805A1CC8F8002059
:1099D0001B782B7201252B46FEF797BBB74A03F184
:1099E00008010133C8F8003013F8010C02F8010F28
:1099F0009942F6D1FEF73FBB591C1A46C8F8001031
:109A0000AF4912F8020B8870C8F800205B784B70E1
:109A100001252B46FEF779BB0722B6FBF2F2C2EB1B
:109A2000C201761A7FF4F4ADD2B2571EFFB2002AFB
:109A30003EF421ABDFF88CA201375A1CC8F8002095
:109A400093F900109F4B002593F902208A4200F001
:109A5000CD840135052D03F10803F5D1D8E55A1C55
:109A6000C8F800201A780E2A3FF6D2AD991CC8F823
:109A700000105D78032D3FF6CBAD9348062101FB26
:109A800002F14218DE1C5571C8F800609D784554FB
:109A9000191DC8F80010D9785170591DC8F8001068
:109AA00019799170991DC8F800105979D170D91D94
:109AB000C8F800109B79137101252B46FEF725BBD2
:109AC0005A1CC8F80020814D1B782B7240460BF0C1
:109AD00003FBA88340460BF0FFFA288340460BF0B7
:109AE000FBFAD8F8003068835A1CC8F800201B78AD
:109AF000EB74082E7EF6BFAA40460BF0EDFAE88420
:109B000040460BF0E9FA0C2E28857EF6B4AAD8F868
:109B100000301A46591CC8F8001012F8021BA97729
:109B2000C8F800205B7885F8203040460BF0D4FA66
:109B3000102EA8847EF69FAAD8F800305A1CC8F8C8
:109B400000201B78EB7240460BF0AEFAD8F80030DC
:109B5000E8605A1CC8F800201A782A74162E7EF67F
:109B60008AAA9A1CC8F800205B7885F82130012564
:109B70002B46FEF7CABA5A1CC8F80020544A1B7874
:109B8000137001252B46FEF7C0BA5A1CC8F80020F6
:109B90004E4A1B785375FEF76EBA5A1CC8F800205F
:109BA0001878060600F1DC844A4B1B78DD073EF589
:109BB00062AA032828BF002001250DF023FE2B46B2
:109BC000FEF7A3BA5A1CC8F80020404693F800904C
:109BD0000BF06AFA074640460BF066FA0546404627
:109BE0000BF062FA064640460BF076FA40460BF060
:109BF00073FAD8F800300133C8F80030B9F1000F1B
:109C000000F07884B9F1100F7EF435AA324B1F6052
:109C10005D600EB1314B9E603149324B0222081F0C
:109C200001251A7026F000FB2B46FEF76EBAC6F32C
:109C30004706122E3FF6ECACB6B10EAB0DF1120991
:109C400003EB46054F46263D40460BF045FA27F804
:109C5000020FBD42F8D1244B39F8022F23F8022F0E
:109C60004F45F9D1112E09D8204A7300023B134405
:109C70000021223223F8021F9A42FBD11C4A012301
:109C80001D461370FEF741BA1A46591CC8F8001059
:109C9000184912F8020BC870C8F8002016495A7803
:109CA0000A70DA1CC8F80020144A9B78D37001258A
:109CB0002B46FEF72ABA00BF943800200B5D002027
:109CC000647E0020107C0020753700200C5D002091
:109CD00028220020B455002088250020A41C002044
:109CE0008C250020DA450020D67E0020D87E00207A
:109CF000FC7E0020407E0020507E0020587E002008
:109D000040460BF0E9F940460BF0E6F940460BF00F
:109D1000E3F9D8F80030BF4D9A1C2F68C8F800202E
:109D20005A7887F82F20DA1CC8F800209A7887F82C
:109D30003A201A1DC8F80020DA7887F83B2007334C
:109D4000C8F8003040460BF0C7F9F88740462F6846
:109D50000BF0C2F9112EB88700F2E083286815F0E5
:109D6000F9FBFEF788B95A1CC8F80020A94DAA4F84
:109D70001B78D5F800907B7140460BF0ADF9A9F83F
:109D800020004046D5F800900BF0A6F9052EA9F862
:109D9000220000F28D830DF057FD19F073FF286843
:109DA000012515F0EBFC2B46FEF7AFB99B4B1B785A
:109DB000D9073EF560A99A4B4FF4C87201251A8065
:109DC0002B46FEF7A2B91A46591CC8F80010924E4D
:109DD00012F8021BB170C8F8002092495A780A7034
:109DE000DA1CC8F80020904D9A782A711A1DC8F81C
:109DF0000020DB78092BA8BF09234046AB700BF08D
:109E00006BF9D8F80030D8F804202880D11A01293D
:109E100007DD40460BF060F9D8F80030D8F8042090
:109E200068829A4240F0BE830DF00EFDD8F80030F3
:109E3000D8F804209A423EF41EA95A1CC8F8002003
:109E40001B78EB7001252B46FEF75FB940460BF0FF
:109E500043F9054626F0D2FAFF283EF40CA9B5F5E1
:109E60007A7F80F088830DF13809002309F8243DBA
:109E7000EE08494603A88DF80C3001361FF098FB18
:109E80009DF80C30F6B205F00705B34205F1010567
:109E900003D19DF81430AB4203D02946304626F05A
:109EA00099FAD8F80030D8F80420D21A012A7EF79F
:109EB000E2A85A1C0EA8C8F8002000221D7800F85D
:109EC0002C2D1FF069FB9DF80C30AB420AD0574B8C
:109ED0001B683BB19A79AA4204D31B681B690BB17A
:109EE00028469847D8F800305A1CC8F80020484641
:109EF00000221D788DF814201FF042FB9DF81430CD
:109F0000AB423EF4B8A8494B1B68002B3EF4B3A803
:109F10001B685B69002B3EF4AEA828469847FEF705
:109F2000AAB8434A1278012A3EF6A5A819465A1C37
:109F3000C8F800203F4A11F8020B9070C8F80010D2
:109F400059781170D91CC8F800109B7853700125FE
:109F50002B46FEF7DAB85A1CC8F800201E78112EDE
:109F60003FF656AB9A1CC8F80020334D5B7805F8D5
:109F7000163040460BF0B0F840F6CA039842A8BF2E
:109F8000184640F2EE23984205EB4601B8BF18464A
:109F90000125A0F2EE222B46192092FBF0F24A7026
:109FA000FEF7B3B81D4B1B78D8073EF564A8012512
:109FB0000DF0A6FE0DF0C8FC2B46FEF7A6B8174B19
:109FC0001B78DA073EF557A81C4A1378012543F0A1
:109FD000040313702B46FEF798B80E4A1068DA1C7B
:109FE00001462133951EC8F8005012F8035C0D702D
:109FF000551EC8F8005012F8025C4D70C8F80020D9
:10A0000012F8015C8D700332934201F10301E9D132
:10A01000A5E600BF48200020E8480020B4550020F5
:10A0200068860020347E002018580020406E0020F2
:10A030007D8400207E840020BC810020721E0020D0
:10A040005A1CC8F800201A78BE49002A00F02C8259
:10A050000A7842F00202981C0A70BB4DC8F8000052
:10A060005B782B7040460BF01FF8686040460BF0A1
:10A070001BF8A86040460BF02FF8A88140460BF073
:10A080002BF8B24A68821378012543F0020313705B
:10A090002B46FEF73AB8092E7FF6BAAAAC4F1A46FD
:10A0A000591C3D68C8F8001012F8021B2970C8F846
:10A0B00000205A78AA70DA1CC8F800209A78642A1E
:10A0C00003F10401A8BF64226A71C8F80010DA78AD
:10A0D000642A03F10501A8BF6422AA71C8F8001020
:10A0E0001A79EA719A1DC8F800205A79642A28BFA3
:10A0F0006422D91D2A72C8F800109A79EA7003F117
:10A100000802C8F80020DB792B7140460AF0E4FF12
:10A110000A2E688140F0138201251CF02FFB2B468C
:10A12000FDF7F3BF00231B7AFFDE23685A1C226071
:10A130001970298820460BF023F82368EA78591C07
:10A1400021601A7023682A79591C21601A702368CB
:10A15000AA79591C21601A7023686A79591C2160F8
:10A160001A70FFF7E9B81A46591CC8F80010794D63
:10A1700012F8021B6970C8F800205A782A70DA1C9D
:10A18000C8F800209B78AB7040460AF0A5FFD8F8CD
:10A190000030E880591C1A46C8F8001012F8021B5B
:10A1A0002971C8F800205B786B714FF0FF352B46A2
:10A1B000FDF7ABBF5A1CC8F800201B780A2B00F033
:10A1C000BC80502B7FF424AA40460AF085FF624EE3
:10A1D000308040460AF080FF4FF0FF3570802B46FC
:10A1E000FDF793BFDFF898B14FF000084FF0080A71
:10A1F00008F10108B8F1240F1BD0C8F120020AFAB7
:10A2000002F22BFA08F6A8F1200316432AFA03F308
:10A210001E4306F0010200231343E9D05FFA88F0E1
:10A220001CF034FA0028E3D0414648460BF02AFBE4
:10A23000DEE74A4B1B78DF0700F102810026484F1A
:10A24000B04602E00136242E0ED0314638460BF0DF
:10A2500029FB0028F6D0314648460BF023FB0028A6
:10A2600054D108F10108EDE73E4B3F4EB3F85010D2
:10A2700020460AF085FF002120460AF081FF3B4B73
:10A280001A68530103F02001C2F340030B43C2F3E9
:10A29000800143EA4103C2F3C00143EA8103C2F3F0
:10A2A000401143EAC10102F01002114320460AF0B6
:10A2B00067FF03A9042220460AF01AFF23683178B9
:10A2C0002B4A581C2060197011886429A8BF64218A
:10A2D00020460AF055FF962D00F0B7800021204659
:10A2E0000AF04EFF2168B8F1190348BFA8F1120324
:10A2F000A3F3C4034A1C226020460B701A4604A92B
:10A3000001250AF0F5FE2B46FDF7FFBE414603A8E6
:10A310000BF0B8FAA5E72368B178164A581C2060FC
:10A32000197023681278591C21601A70FEF752BF09
:10A33000114A92E82200FEF7DABB40460AF0CCFE52
:10A340000E4E45E7721E0020741E0020D8450020E6
:10A350004C200020641E002008260020B455002058
:10A36000A41C0020600100205A84002038510020E5
:10A37000FA350020347E002084200020307E00202A
:10A3800090E33FF400C0884400C08244D9F8003014
:10A3900013F48053B4EEE88A62D0F1EE10FA11DBC8
:10A3A000B4EEC98AF1EE10FA5DD85FED0A7A1FEDBE
:10A3B0000A7A77EEC87AB4EEC78AF1EE10FAB0EEF8
:10A3C000678A50D94FF47A71B5EE408AF1EE10FAEF
:10A3D00040F2DC5308BF1946FEF7E5BD22680125AF
:10A3E000531923602B461070FDF78FBE0AEBC50989
:10A3F000404689F802100AF06FFED8F800202AF8CB
:10A4000035001346511CC8F8001013F8021B89F8D8
:10A410000310C8F80030537889F80430D31CC8F80A
:10A420000030937889F80630131DC8F800300136E3
:10A43000D27889F80520B7427FF4FFAAFDF71BBE4A
:10A44000059B43F001030593F8E623680322591C9A
:10A4500021601A7023687278591C21601A7041E7D4
:10A46000F1EE10FA1CDBF7EE007A78EE677AB6EEC2
:10A47000007AF0EE696AE7EE876A40F2E932FDEEB3
:10A48000E67A17EE901AB1F5FA6FA8BF4FF4FA61A9
:10A490009142B8BF114689B2002B3EF484AD93E7D8
:10A4A0004FF47A71FEF77FBD0A7802F0FD02D2E523
:10A4B00040460AF011FE788140460AF00DFEB88150
:10A4C0004046D5F800900AF007FEA9F8240040465F
:10A4D000D5F800900AF000FE0D2EA9F826007FF6B0
:10A4E0005AAC40460AF0F8FDF88140460AF0F4FD07
:10A4F000388250E4304B10201F605D6011F01CFE6C
:10A500002E4A137843F001031370002E3DF4B3ADCF
:10A510002B4B01259E602B46FDF7F7BDD8F8003088
:10A520002968581C1A46C8F8000012F8020B81F876
:10A530003100C8F800205B7881F832300EE4D8F89A
:10A5400000303A68591CC8F80010197851720B2E67
:10A550003FF4E2AD991CC8F800105B785370DBE55E
:10A5600000F07F00032828BF002001250EF09AFB91
:10A570002B46FDF7CABD0DF11409484625F01EFF14
:10A58000BDF81430AB423FF48CAC0E4B1B68002B73
:10A590003FF487AC1B689B69002B3FF482AC2846D4
:10A5A00098477EE45A1CC8F800201B78003318BF77
:10A5B0000123F37138E400BF84200020721E0020C4
:10A5C000A41C0020406E00202DE9F04FA34CDFF8C2
:10A5D000C09294F85C312DED028B83468FB0002B36
:10A5E00040F05A8194F8DD31002B39D0D4F8E031B5
:10A5F0009B4AABEB0303934200F2348494F8486225
:10A60000002E00F0B780D4F850324BB3D4F8583253
:10A6100040F6B732ABEB0303934221D994F854329E
:10A62000002B00F061858F4F013BDBB284F8543280
:10A63000002B00F06985D4F8505294F85C2215F88C
:10A64000011B94F85D323868C4F850520A44013353
:10A6500084F85C2284F85D320CF078FBC4F858B2C0
:10A6600094F85E32D9F8005043B17F4E306828B17B
:10A6700094F85F32013B012B40F2F38494F8A0334D
:10A6800053B17A4E33683BB1D9F80070D4F8A43393
:10A69000FB1A632B00F22A8294F8DC33022B00F0C1
:10A6A000D482734D95F87430032B00F0488794F8EA
:10A6B000F8336BB1D4F8FC3353B10CF0F9F8D4F89B
:10A6C000003444F61F62C31A9342074600F2E88240
:10A6D00094F87A35002B40F08B8194F88B3533B1A8
:10A6E000D4F88C3503F5C333A0339B4578D294F866
:10A6F000C235BBB15F4D2E46D4F8C4050CF022FB29
:10A7000080B1D4F8C4050CF019FB94F8C83507469D
:10A710005A1E63B1D4F8C40584F8C8250CF012FBA6
:10A720000028EED10FB0BDEC028BBDE8F08F032204
:10A730005149284629F066FF94F8CC3594F8CD2588
:10A7400084F8CF7583F47F4383F0FF039B1ABFB275
:10A750009BB2B7EB132FCFD194F8CE25DBB29A4240
:10A76000CAD1304624F09CFE94F8C835184484F8C9
:10A77000C805C1E73B4F38680CF0E4FAC0B20128C5
:10A780000FD902283A4D40F0CE842B78002B41F0AF
:10A79000A087D4F84C32ABEB0303B3F57A6F81F0AA
:10A7A0009A85D4F85032002B3FF45AAF94F84832CF
:10A7B000002B7FF42BAF314B1B689B7801211E3B94
:10A7C00000228B4284F8481284F85C2241F2D2873E
:10A7D00038680221043024F089FF94F8543223E7CA
:10A7E00094F89035264AC4F88CB502EB8302526C7B
:10A7F00042B3244F244E0EADFB1C45F8203D07F11B
:10A80000150300210793A523318084F89435802116
:10A81000152384F89635284684F8951590472846E0
:10A8200031880AF0ADFC069DED1B152DA8BF15253E
:10A830002A46394607F1180029F0D9FE94F89035D8
:10A8400084F8C155114A013382FB0312A2EBE37273
:10A8500002EB42029B1A84F8903548E7B01C0020B6
:10A860003F0D0300F88200209C820020F08200202F
:10A87000000000207C2200207D220020FC8200209D
:10A88000AC490308442200207086002056555555D7
:10A89000E075002000007A44D4F86031D9F8002037
:10A8A000D31A7C2B7FF69EAE94F864311FED078A95
:10A8B000C4F86021013384F8643104F5CE7724258F
:10A8C000284624F08BFFB4F87831F7EC016A07EEE4
:10A8D000103AF8EEE66AB8EEC77A0135C6EE877A26
:10A8E000EDB267EE887AFDEEE77ACDED007ABDF93C
:10A8F0000060F0B224F048FFC6F3072024F044FFC4
:10A90000272DDDD1302024F069FFD94E002024F01E
:10A910003BFF002024F038FF30685E210CF016FA6F
:10A9200094F8643113F0030528D1D4F8602141F282
:10A9300088339A4201F2C987142024F04FFFCD4A90
:10A94000B4F9B031DD1782FB0323C5EBA3052DB2AB
:10A95000E8B224F019FFC5F3072024F015FF1C20EE
:10A9600024F03CFF002024F00FFF002024F00CFF17
:10A970005E2130680CF0EAF994F8643113F00705B1
:10A9800001F02E85282B7FF42DAE00251720D9F855
:10A99000008084F8645124F021FF284624F0F4FE5E
:10A9A000B54BB64FA3FB08239B0BA7FB0312520921
:10A9B000C2EB0212A3EB8203D8B224F0E5FE18200A
:10A9C00024F00CFFAE4BA3FB08239B09A7FB03124B
:10A9D0005209C2EB0212A3EB8203D8B224F0D4FED8
:10A9E000284624F0D1FE30685E210CF0AFF9F9E57D
:10A9F000A44D2A7832B1A449D4F87C050CF072F940
:10AA000000232B70D4F8803503F5C333A0339B4566
:10AA1000FFF463AE94F88935C4F880B5234493F805
:10AA20008455E80701F10B86A90701F1CD856A0776
:10AA300001F191852A074DD5944B07930EAA104634
:10AA4000A3F1210240F8202DA3F124020646009034
:10AA5000002003F8240C1125022355709370D4F8BC
:10AA6000C81130460AF04EFB3046D4F8CC110AF03B
:10AA700049FBB4F8D6317F4903EBC3039B00053390
:10AA800081FB0321DB17C3EBA10189B230460AF039
:10AA900051FBB4F8D83103EB8303590089B2304637
:10AAA0000AF048FB94F8C231009D9B0743BFB4F8FD
:10AAB000D01101F57A7189B24FF47A7128460AF003
:10AAC00039FB069B94F8C421591C069128461A703C
:10AAD00026F02AFD94F8893594F88A15013393FB02
:10AAE000F1F201FB123384F88935F6E5412024F0B8
:10AAF000ADFD604DB4F9AE31DFF8A08185FB0320D8
:10AB0000DB17C3EBA00080B224F084FDB4F9AC31B4
:10AB100085FB0320DB17C3EBA00080B224F07AFD95
:10AB2000B4F9B03185FB0320DB17C3EBA00080B282
:10AB300024F070FD98F8001030680CF007F994F8D4
:10AB4000A85315F0010200F0B585514B1B689A0619
:10AB500068D594F8C2319B0701F1B58301254720E0
:10AB600024F074FDD4F8C80124F020FDD4F8CC0101
:10AB700024F01CFD474AB4F8D6313068A2FB032309
:10AB8000C3F3471A51460CF0E1F8B4F8D02198F815
:10AB90000030642000FB02F08AEA030388F80030EA
:10ABA00024F004FD94F8C431306845EA8305EDB221
:10ABB00029460CF0CBF898F8003030685D40294603
:10ABC00088F800500CF0C2F894F8A85355BB4F20F9
:10ABD00024F03CFDD4F8D40324F0E8FCD4F8D803E6
:10ABE00024F0E4FC284624F0E1FC012130680CF05C
:10ABF000ADF894F8C25198F80030306805F00105BE
:10AC0000294683F0010388F800300CF09FF898F88B
:10AC1000003030685D40294688F800500CF096F806
:10AC200094F8A8531C4AC4F8A4736B1CDBB2A2FBB3
:10AC30000312D20802EB8202A3EB420384F8A8338A
:10AC400094F8DC33022B7FF42CAD0BF031FED4F8FA
:10AC5000E06340F6B833861B9E4201F24E8294F8C0
:10AC6000EC333A2B01F03A85002384F8DC331EE5FF
:10AC7000008300206766666673B2E7458988888826
:10AC8000D34D6210BC860020988600209886002054
:10AC9000385100201F85EB51CDCCCCCCF482002064
:10ACA00094F80634002B40F0CB846A4B1B6848F6BE
:10ACB000034113F0080F49F607464FF0190208BF89
:10ACC0000E46580784F8062403D546F4005646F08D
:10ACD0000806990648BF46F4804694F8B85148BF24
:10ACE00046F02006C6F30908002D41F01B8394F8B6
:10ACF000B931002B41F024861D4664204FF0FF3A05
:10AD00004FF0000C06960796ADF82650CDF820803F
:10AD1000ADF828A08DF83600ADF824C0ADF82AC0F3
:10AD2000ADF82CC0ADF82EC0ADF830C0ADF832C0D3
:10AD3000ADF834C00DF1180EBEE80F00464E354692
:10AD40000FC59EE80F0007C525F8023B180C01212E
:10AD5000FE221F23287084F8531084F84E2084F8B4
:10AD60004F3094F8162484F851C05118C82084F844
:10AD7000161484F85020311F84F852004FF6FF75E6
:10AD800001E011F8013B6B4083EA0313DBB21A09BF
:10AD900082EA152242EA03228E4282EAC305F0D1FA
:10ADA0002D49A4F84C5001F11F0011F8013B6B40F4
:10ADB00083EA0313DBB21A0982EA152282EA03222C
:10ADC00082EAC3031BB29DB28142A4F84C50ECD17D
:10ADD00083F07C0383EA0313DBB21A0982EA1522AB
:10ADE00082EA032282EAC3031BB29AB24FEA122C10
:10ADF0005FFA83FE194EA4F84C2084F874C084F8DE
:10AE000073E004F14E0804F16E0AD8F80000D8F897
:10AE10000410D8F80820D8F80C3035460FC508F1D2
:10AE20001008D0452E46F0D1D8F8000028600C4D0F
:10AE300098F80430337105F1270684F865E484F846
:10AE400066C415F8011FD4F8FC030BF07FFFAE4277
:10AE5000F7D1F8E338510020041D0020F020002035
:10AE6000EF200020D94ADA4BD07AD9F80010D4F874
:10AE700010221B88891A4FF47A7202FB00F2DDB2AD
:10AE800000201B0A914284F8025284F8F85184F899
:10AE9000033284F8F93184F8E60184F8E80181F09E
:10AEA000F480CC4BCC491A689B6894F8C20181FBB2
:10AEB000026581FB0361D217DB17C2EBA502C3EB6E
:10AEC000A10315121912F42684F80022012284F835
:10AED000015284F80432302584F8051284F8FE61AA
:10AEE0007521782384F8FF21860794F8C42184F81B
:10AEF000065284F8071284F8083284F8322241F1AD
:10AF0000BF80D4F8C851B549D4F8CCC1B448B54BCA
:10AF1000DFF8E8A281FB0567EE1781FB0CE1C6EBC9
:10AF2000A7564FEAEC77C7EBA15100FB065707EB9A
:10AF300047077F0000FB01C083FB07E800EB4000F0
:10AF400040004FEAA848052A4FEAD5754FEAE77254
:10AF500001EB810183FB00E301EB810106EB860637
:10AF600084F82152A8EB02054FEAA34E00912A462D
:10AF70004FEAE0716DB206EB860605EB8606B4F883
:10AF8000D631AEEB010529464FEADC7C0AFB127292
:10AF900003EBC303944FDFF868E284F826C24FFA4C
:10AFA00081FC00990AFB15054FEA8303B4F8D00130
:10AFB0000CEB81018EFB03CE87FB028C4FEAE27221
:10AFC00087FB0587C2EB6C12B6B289B24FEAE37316
:10AFD000B4F844C284F8226200F5FA704FEAE575CD
:10AFE0004FEA112AC3EBAE1EC5EB67154FEA1623D5
:10AFF00080B24FEA222884F828A284F823324FEA4C
:10B00000252784F82712CEF307264FEA102184F86B
:10B01000242234BF4FF0320A4FF0330A4FEA1C2289
:10B02000B4F8463284F8258284F8295284F82A72CA
:10B0300084F81FE284F8206284F82D0284F82E122E
:10B0400084F833A284F82BC284F82C2284F834329A
:10B0500094F84862C4F8E0B1002E7FF4D4AAFFF758
:10B0600089BB624F4FF0010A4FF0000808E01B2B2C
:10B0700000F07B820D2B00F0878187F801A03068FB
:10B080000BF060FE00285BD030680BF057FE83B2F7
:10B090007E2BD9F800204CD07A78002AEFD194F892
:10B0A00060120029E3D07D2B00F0468294F864E220
:10B0B000BEF1000F04D080F02003DBB284F86422DC
:10B0C0004A1CD2B2092A635484F8602200F02A8212
:10B0D000082AD4D8B4F86222134403EB132303F0F4
:10B0E000FF03A4F86232CAE7C4F8503284F8483249
:10B0F00024F030FB94F854323D4F013BDBB284F82E
:10B100005432002B7FF497AA94F85C1294F85D32C5
:10B1100038684A1C013384F85C2284F85D320BF0F5
:10B1200015FEFFF79BBA24F005FB01232B70FFF7F8
:10B1300038BB84F8608284F8618287F801809EE7DA
:10B1400094F865322BB1637884F86502302B01F0F6
:10B15000398394F86122274B274FDFF8A8E0DFF806
:10B160006CC00126002A3FF489AAD9F80000401BD0
:10B17000012825D894F87883B8F1000F40F00682B2
:10B1800094F890A303EB4A00008900283CD184F88E
:10B19000906338688106E5D594F8C2018007E1D54F
:10B1A000B4F8D62110494FF4F36303FB02F381FB9B
:10B1B0000321DB17C3EB61114FF4036024F07CFA29
:10B1C000002384F86132FFF759BA00BF888200205B
:10B1D000A0820020A4820020676666666BCA5F6B4F
:10B1E000806967FF83DE1B431F85EB510000002051
:10B1F000F8820020AC4903083851002040420F007B
:10B20000D34D6210386E00200AF1010A5FFA8AFA03
:10B21000B0F5E06F84F890A300F099801AD8B0F5EB
:10B22000047F00F0318136D8B0F5887F00F00981C5
:10B23000B0F5007F00F0EF80B0F5807F92D13968E3
:10B2400049078FD5002124F037FA002384F86132B2
:10B25000FFF714BAB0F5026F00F001816CD8B0F5B9
:10B26000E46F00F08380B0F5006F00F09380B0F5DC
:10B27000E26F7FF477AFD4F8A021B4F8781164239B
:10B2800003FB02F393FBF1F124F016FA002384F898
:10B290006132FFF7F3B9B0F5826F00F02481B0F5A9
:10B2A000C06F00F01081B0F5806F7FF45BAF94F851
:10B2B00091330133DBB2032B00F2628142F2107151
:10B2C00084F8913301FB03F1B4F89233002B40F082
:10B2D00055810131D24B1B78DF07B4F8943348BF56
:10B2E0000431DD0748BF0A31980748BF14311A06F8
:10B2F00048BF2831DF0548BF28315D0748BF6431AA
:10B30000180748BFC8319A0548BF01F5C8719F06A4
:10B3100048BF01F57A71DD0648BF01F5FA615806AC
:10B3200048BF01F57A614FF4806024F0C5F900232D
:10B3300084F86132FFF7A2B9B0F5046F19D0B0F507
:10B34000116F4DD0B0F5036F7FF40CAF21E7D4F847
:10B350009C21B4F87811642303FB02F393FBF1F111
:10B3600024F0AAF984F86182FFF788B9D4F8A421FF
:10B37000EFE7B4F9B01101EB8101490024F09CF929
:10B3800084F86182FFF77AB984F860A22370A4F888
:10B39000621274E6386881067FF5E4AE94F8C20163
:10B3A00080077FF5DFAE1AF0010F40F07887D4F800
:10B3B000C8219C4982EAE273A3EBE27303EB5303D7
:10B3C000A1FB0331C908002AB8BF41F080414FF406
:10B3D000006024F071F9002384F86132FFF74EB960
:10B3E00094F8B80100283FF4BDAE8F4908780028D2
:10B3F0003FF4B8AE8D4B1B8803EB830359008046A6
:10B400004FF4116091FBF8F124F056F9002384F811
:10B410006132FFF733B994F8B90100283FF4A2AEC6
:10B42000834B84491B6881FB0321DB17C3EBA1011C
:10B430004FF4007024F040F9002384F86132FFF7E4
:10B440001DB9386841077FF58DAE00214FF4887033
:10B4500024F032F9002384F86132FFF70FB939681C
:10B4600089067FF57FAE94F8C2A11AF0020F3FF46F
:10B4700079AEB4F8D031642101FB03F124F01CF95A
:10B4800084F86182FFF7FAB894F8B80100283FF415
:10B4900069AE6549087800283FF464AE664B5B7B73
:10B4A000002B01F04982614B198891FBF0F101EB0F
:10B4B000810149004FF4047024F0FEF8002384F861
:10B4C0006132FFF7DBB894F8B90100283FF44AAEC7
:10B4D000574B4FF4C060996824F0EEF8002384F8CD
:10B4E0006132FFF7CBB83868810640F1F18594F8F6
:10B4F000C22194F8C41112F0020F0CBF00234FF4C4
:10B500007A7312F0010F0CBF00224FF4FA62134459
:10B5100019444FF4826024F0CFF8002384F861329C
:10B52000FFF7ACB8B4F86222C2F1FF0293427FF495
:10B53000A4AD84F865A2A0E584F864A29FE5D4F8E0
:10B54000F40303685B69984700283FF4B0A8D4F877
:10B55000F403036801219B6998470222002385F8C0
:10B56000742084F8DC33FFF7A2B830680BF0EAFBF4
:10B5700000287FF482AD84F861A280E50231A9E65B
:10B58000012384F8913342F210719DE6D4F86832B9
:10B590002A4E94F88E23B34201F0B081511C94F8E6
:10B5A0008F03D4F86C7284F88E1302F00F028DF8BA
:10B5B00018200DF11902F91A002941F3008306A998
:10B5C00000910DF11E0502E0002E40F3A08501332D
:10B5D000C4F8683213F8011C02F8011BAA42A7EB59
:10B5E000030680EA0100EFD384F88F0301F0E182C3
:10B5F000531CAB42107038BF002203D203F8012B5A
:10B60000AB42FBD10099322024F03AF84FF0000809
:10B61000002384F8788384F86132FFF72FB800BFE5
:10B62000B45500201F85EB51DF820020A08200204E
:10B63000A48200206766666688820020281F00209A
:10B64000013B84F8063494F80734002B40F09580D1
:10B6500094F84815D9F800E00A2284F80724002954
:10B6600000F059850129B4F854A541F2218302293B
:10B67000B4F8568501F06A810329B4F858C501F081
:10B680004283B4F85A250092042901F03783052932
:10B69000B4F85C5501F02E830629B4F85E0501F07C
:10B6A00026830729B4F8602500F03D85B4F862359B
:10B6B00000F039BDB4F89433D80513D4D90601F19C
:10B6C000EF809D0601F14981580601F16F8219074B
:10B6D00001F17B82DD0701F1D78213F0020F0CBF6D
:10B6E00004220C22B24994F8AF3391F800A00AF07A
:10B6F000010A0BB14AF0020A5320009223F0A6FF80
:10B70000AC4B1B8803EB830303EB8303980080B2ED
:10B7100023F080FF002023F07DFFB4F8D033A6494A
:10B720003068C3EBC3135B0081FB03211944DD17B1
:10B73000C5EB6125EDB229460BF008FB98F8003007
:10B74000009A306842EA0A0A5D40002188F80050F9
:10B750000BF0FCFA514630680BF0F8FA98F800301C
:10B7600030688AEA0303DBB2194688F800300BF030
:10B77000EDFA94F8A853FFF729BA013B84F807348F
:10B7800094F80A34002B40F06E848C4B1B6819220D
:10B7900084F80A249A0640F11A8294F8C2319B0771
:10B7A00000F1B88501260BF083F8B4F8D811B4F88D
:10B7B000D051D4F8C831069001EB810101934900C2
:10B7C0004FF47A70ADF83210D4F8CC21B4F8D681A9
:10B7D00094F8C4C101998DF8346000FB05F04FF076
:10B7E000000E06AB4FF6FF75ADF830808DF835C012
:10B7F000CDF81CE00A9008910992ADF82C50ADF8F4
:10B800002E5098460093B8E80F006D4EB446ACE851
:10B810000F0098E80F00ACE8070094F81624ACF885
:10B82000003084F851E0A6F1040A02F1010E18205C
:10B83000FE211E234FF0C80CD04684F8502084F817
:10B8400016E484F8530084F84E1084F84F3084F8DE
:10B8500052C001E018F8013B6B4083EA0313DBB2EE
:10B860001A0982EA152242EA0322464582EAC30502
:10B87000F0D1534AA4F84C5002F11E0112F8013BDA
:10B880006B4083EA0313DBB2180980EA152080EAD3
:10B89000032080EAC3031BB29DB28A42A4F84C5035
:10B8A000ECD183F0180383EA0313DBB21A0982EAAE
:10B8B000152585EA032282EAC3031BB29AB2DBB2E2
:10B8C0004FEA122E019384F87230DFF800C1A4F819
:10B8D0004C2004F16E0384F873E004F14E060293E9
:10B8E000F36830687168B26865460FC5029B103610
:10B8F0009E42AC46F4D13068CCF80000314D9DF842
:10B90000043084F8643484F865E42E4616F8011F88
:10B91000D4F8FC030BF01AFA2B4BB342F6D10AF021
:10B92000C7FFB4F9B011DFF8A8E0B4F8D061069011
:10B930008EFB010EC9174FF47A7000FB06F0D4F8A5
:10B94000C821D4F8CC31009E0990C1EBAE014FF074
:10B95000000EADF82CE0ADF82EE0ADF830E0ADF81B
:10B9600032100A90079208930FCE04F1540CACE801
:10B970000F0096E8070021231C268CE8070084F8B6
:10B980005330C8226FF0010384F851E084F84E3040
:10B9900084F84F6084F8522094F8163484F85030BC
:10B9A0005A1C84F8162433464FF6FF7E564613E0A1
:10B9B000B4550020A08200200308208038510020C8
:10B9C000041D0020EF20002015210020F020002081
:10B9D0006766666616F8013B83EA0E0383EA031383
:10B9E000DBB21A0982EA1E2242EA0322B04582EA49
:10B9F000C30EEFD1D248A4F84CE000F11C0110F8BE
:10BA0000013B83EA0E0383EA0313DBB21A0982EADD
:10BA10001E2282EA032282EAC3031BB21FFA83FEBC
:10BA20008842A4F84CE0EAD183F0680383EA031368
:10BA3000DBB21A0982EA1E2282EA032282EAC303E7
:10BA40001BB29AB2DBB2110A019384F87030DFF8AE
:10BA500000C3029104F16E03A4F84C2084F8711025
:10BA600004F14E080393D8F80C30D8F80000D8F849
:10BA70000410D8F80820E646AEE80F00039B08F152
:10BA800010089845F446EED1B8F80030AEF8003012
:10BA90009DF8043084F862349DF8083084F86334EB
:10BAA000A84618F8011FD4F8FC030BF04FF9A54B7A
:10BAB0004345F6D1D4F8D433D4F8D82306934FF0C5
:10BAC000000E009BCDF820E0079293E8070004F1F8
:10BAD000540383E8070094F8162484F851E03120D9
:10BAE00002F1010EFE210C2384F85020C82284F8B4
:10BAF00016E484F8530084F84E1084F84F3084F82C
:10BB000052204FF6FF7E01E01AF8013B83EA0E0354
:10BB100083EA0313DBB21A0982EA1E2242EA0322F5
:10BB2000564582EAC30EEFD18549A4F84CE001F1F5
:10BB30000C0011F8013B83EA0E0383EA0313DBB226
:10BB40001A0982EA1E2282EA032282EAC3031BB296
:10BB50001FFA83FE8142A4F84CE0EAD183F0270368
:10BB600083EA0313DBB21A0982EA1E2E8EEA032E41
:10BB70008EEAC30EA2460FFA8EFE1FFA8EF65AF810
:10BB80004E0FDFF8CCC1A4F84C604FEA16285FFADC
:10BB90008EFE84F860E084F86180DAF80410DAF848
:10BBA0000820DAF80C30BAF810A0ACE80F0004F264
:10BBB0005346ACF800A084F8538484F852E415F896
:10BBC000011FD4F8FC030BF0C1F8AE42F7D194F892
:10BBD0000E64002E40F0BE80B4F9AC21B4F9AE3151
:10BBE0009FED596AD9F80010069106EE902AB4F933
:10BBF000B021534D84F851605B4207EE102A07EEE6
:10BC0000903AF8EEE66AF8EEE77AB8EEC77A67EEB1
:10BC1000867A66EE866A27EE067A0022CDED087AED
:10BC2000CDED076A8DED097A0A920B920C920DF117
:10BC3000180EBEE80F002E460FC69EE8070094F8C7
:10BC400016C486E807004FF00508FE20C8214FF013
:10BC50001E0E1C230CF1010284F84E0084F85210D1
:10BC600084F80E8484F853E084F84F30291F84F858
:10BC700050C04FF6FF7084F8162401E011F8013B24
:10BC8000434083EA0313DBB21A0982EA102242EA34
:10BC900003228D4282EAC300F0D1294DA4F84C0062
:10BCA00005F11C0115F8013B434083EA0313DBB2A5
:10BCB0001A0982EA102282EA032282EAC3031BB233
:10BCC00098B28D42A4F84C00ECD183F0270383EAAC
:10BCD0000313DBB21A0982EA102282EA032282EA03
:10BCE000C3031BB29AB24FEA122C5FFA83FEDFF84D
:10BCF0006080A4F84C2084F871C084F870E004F1EE
:10BD00004E0604F16E0930687168B268F368454602
:10BD10000FC510364E45A846F5D10C4D3388A8F80E
:10BD2000003005F1240684F862E484F863C415F851
:10BD3000011FD4F8FC030BF009F8AE42F7D10CE078
:10BD4000041D00201321002088C3E43AEF200020C6
:10BD5000F0200020731E84F80E3494F80F34019301
:10BD6000002B40F08481D24B1B6805229D0684F88D
:10BD70000F2400F18382DFEDCF7AB0EE677AB4F959
:10BD80005A35B4F9B011CC4DCC48CDED077AB3F5A6
:10BD9000FA6FA8BF4FF4FA63B3F57A7FB8BF4FF4D8
:10BDA0007A73A3F57A72642303FB02F385FB032500
:10BDB00080FB0120DB17CA170026C3EBA51306A9D9
:10BDC000C2EBA0028DED087AADF82A30ADF828203C
:10BDD000069609960D4600910FCDDFF8E4E22E6835
:10BDE00094F816C484F850C075460FC54A212E60D9
:10BDF000AEF1040800250CF10100FE22142384F8A2
:10BE00005310C82184F85150464684F8160484F82B
:10BE10004E2084F84F3084F852104FF6FF7501E041
:10BE200016F8013B6B4083EA0313DBB21A0982EA7E
:10BE3000152242EA0322B64582EAC305F0D1A049A1
:10BE4000A4F84C5001F1140011F8013B6B4083EA57
:10BE50000313DBB21A0982EA152282EA032282EA7C
:10BE6000C3031BB29DB28142A4F84C50ECD183F0C5
:10BE7000140383EA0313DBB21A0982EA152282EA69
:10BE8000032282EAC30325461BB21FFA83FC55F83E
:10BE90004E0FDFF838E2A4F84CC0DBB24FEA1C2AA0
:10BEA00084F869A084F8683069680293AA68EB682E
:10BEB000AEE80F00286969692B8BAEE8030004F235
:10BEC0003F45AEF800309DF8083084F85BA4A946E1
:10BED00084F85A3404F25B4A19F8011FD4F8FC03C1
:10BEE0000AF034FFCA45F7D1764A94F878351278CB
:10BEF000013BDBB212F0010214BFC0214021172B1D
:10BF00009BBF71481B184FF0000E93F82CE0B4F85B
:10BF10009433980706BF0120019041F0100113F4FB
:10BF2000027F019818BF022013F0100F18BF0620DF
:10BF300013F0200F0CBF034610230193002A40F09A
:10BF4000B2840322019B069303234FF0000C8DF86B
:10BF50002030009B8DF81CE08DF81E108DF81F20FE
:10BF60008DF81DC093E80700DFF854E184F853C052
:10BF7000AEE8030094F816148EF8002001F1010ACF
:10BF80004FF0FE090923C82084F851C084F85010EE
:10BF900084F816A484F84E9084F84F3084F8520048
:10BFA0004FF6FF7E01E018F8013B83EA0E0383EAB7
:10BFB0000313DBB21A0982EA1E2242EA0322464533
:10BFC00082EAC30EEFD13E49A4F84CE001F109002A
:10BFD00011F8013B83EA0E0383EA0313DBB21A096B
:10BFE00082EA1E2282EA032282EAC3031BB21FFAFC
:10BFF00083FE8142A4F84CE0EAD183F0320383EA65
:10C000000313DBB21A0982EA1E2282EA032282EAC1
:10C01000C303A6461BB21FFA83FC5EF84E0F2B4EDD
:10C02000A4F84CC0DBB24FEA1C2884F85D3084F8D9
:10C030005E80DEF80410DEF8082007C6BEF80C109B
:10C040009EF80E203180B27004F58A6684F8508420
:10C0500084F84F3415F8011FD4F8FC030AF076FE7B
:10C06000AE42F7D108E0013B84F80A34AFE5019B0A
:10C0700003F1FF3984F80F94C4F80074FEF728BB6D
:10C080002D2384F83332FEF7E3BF94F81432D9F845
:10C090000020C4F81022013B012B3EF602AF102213
:10C0A000022384F8E62184F8E831FEF7FABE00BFE7
:10C0B0003851002000000000D34D621067666666AC
:10C0C000041D0020B4550020AC490308F0200020D6
:10C0D000DEF80000000600F1CC839CF80C0000287C
:10C0E0003FF440A894F89613032900F2B485DFE8E2
:10C0F00011F05F01550146012F01B4F8E43300222D
:10C100000133A4F8E43384F8DC23FEF7D0BA84F8D2
:10C110008F03FFF76DBA0A4608460D4600918C461C
:10C1200088468A460B46B4F8D013A64ECDF818E0E0
:10C13000C1EB012186FB016E8E44C917C1EB6E2154
:10C14000BDF80060ADF81E804FF0000EADF820C0C5
:10C15000ADF82260ADF824508DF82CE0ADF81CA0AD
:10C16000ADF82600ADF82820ADF82A308DF82D1056
:10C1700006AD0FCD944E84F851E0B646AEE80F0000
:10C1800095E8030094F816C44EF8040B23250CF12F
:10C190000108FE201623C822AEF8001084F8535080
:10C1A00084F850C084F8168484F84E0084F84F3028
:10C1B000311F84F852204FF6FF7501E011F8013B62
:10C1C0006B4083EA0313DBB21A0982EA152242EAC2
:10C1D00003228E4282EAC305F0D17B49A4F84C5079
:10C1E00001F1160011F8013B6B4083EA0313DBB247
:10C1F0001A0982EA152282EA032282EAC3031BB2E9
:10C200009DB28142A4F84C50ECD183F0F40383EA50
:10C210000313DBB24FEA131E8EEA152E8EEA032EAD
:10C220008EEAC30E25460FFA8EFE1FFA8EF855F8D9
:10C230004E0F664EA4F84C805FFA8EFE4FEA182C23
:10C2400084F86AE084F86BC06968AA68EB680FC676
:10C2500028696969AA6904F23F4507C604F25D4688
:10C2600084F85DC484F85CE415F8011FD4F8FC037D
:10C270000AF06CFDAE42F7D1FFF782BAB4F8D631BE
:10C28000DFED536A07EE903AB4F8D031F8EEE77A72
:10C2900007EE103A67EEA67AB8EE477A6FE5D4F863
:10C2A000CC214C4982EAE273A3EBE27303EB530324
:10C2B000A1FB0331C908002AACBF41F0004141F0A5
:10C2C0004041FFF784B894F8C431042B8CBF032598
:10C2D0000225FEF744BC012338682B700AF02EFDBE
:10C2E000054638680AF02AFD6D067EF45AAA8A28A7
:10C2F00000F09F848E287EF454AA94F84832002BD4
:10C300007EF481A9344BC4F850322D2384F8543282
:10C31000FEF751BA94F8C431042B8CBF03260226D1
:10C32000FFF741BA2D4B94F8B9211B8803EB830327
:10C3300003EB83039D00ADB2002A40F0B1844FF0BF
:10C34000FF330FFA83FA0CF0C1FC40B2FEF7D8BC01
:10C35000D4F89C2353799079D17903F1407303EB9E
:10C36000002303EB0141002384F896334FF48260ED
:10C3700023F0A2F9002384F86132FEF77FB9D4F8E4
:10C380009823137A507992781B0403EB002313440B
:10C390004A1C84F8962303EB0161E7E7D4F898235D
:10C3A000D379107952781B0403EB00231344EFE791
:10C3B000D4F898239379D07812781B0403EB0023E8
:10C3C0001344E5E703082080041D0020F02000202E
:10C3D0000AD7233C1F85EB51941E0020A082002029
:10C3E000022023F0FBF9FF2022F0DCFF0378FF2B73
:10C3F00000F0D58390F90100C517EDB2C0B223F06B
:10C40000C3F9284623F0C0F9032023F0E7F9FF2001
:10C4100022F0C8FF0378FF2B00F05783B0F90850D3
:10C42000E8B2C5F3072523F0AFF9284623F0ACF9AD
:10C4300094F8B831002B40F09382D24B1B689806D9
:10C4400040F1398294F8C231990700F16D830025DB
:10C450002F46012023F0C2F9384623F095F92846EB
:10C4600023F092F9092023F0B9F9002023F08CF988
:10C47000002023F089F9B4F8DA2194F8C451B2F518
:10C48000967F0AD994F8643103F00F03072B04D880
:10C4900042F20F75954228BF1546BB4F052023F089
:10C4A0009DF93B7A002B00F0BD83A5F1200307EE38
:10C4B000903A9FEDB67AF8EEE77AF6EE006A67EE0C
:10C4C000877ABEEE007AF5EEC07AF1EE10FA58BF28
:10C4D000B0EE667A77EE877AFDEEE77ACDED007AF8
:10C4E000BDF90050E8B223F04FF9C5F3072023F05F
:10C4F0004BF994F8C221002304930593930700F1AC
:10C50000BD8294F8DC31012B00F0B882B7F900301D
:10C51000DFED9F6A07EE103AB7F9023007EE903A66
:10C52000B8EEC77AF8EEE77A27EE267A67EEA67AB3
:10C53000BDEEC77AFDEEE77A06A88DED067ACDED61
:10C54000077A23F05DF95E2130680AF0FFFB94F86A
:10C550006431FEF717BA8F4B0793A3F1240600222C
:10C560002121A3F1210703F8242CB17072700697E2
:10C570001AF07EF8884B8949B4F89423002814BF38
:10C5800099468946530500F1B481D00700F198829D
:10C59000910740F10683DFF828924FF003084246E6
:10C5A00049467F4828F023F807EB08030EA87D4A88
:10C5B000013340F8203D9B1A002207F808207370D1
:10C5C00024F0B2FFFEF736BA724B774907930EAEEE
:10C5D000A3F1210046F8200D0A2003F8230C0027C0
:10C5E000082003F8220C03F8247C3046098808F060
:10C5F000A1FD6E4B6E491B6881FB0321DB17C3EB6A
:10C60000A101304689B208F095FD0CF05FFB069B56
:10C61000B4F8BA21591C06911F70069B110A5F1CC1
:10C6200006971970069B591C06911A70069B5A1C96
:10C6300006921870304624F077FFFEF7F8B9B4F987
:10C64000AE319FED5C8A534A079207EE903AF8EEBE
:10C65000E77A0EAE67EE887AA2F12101FDEEE77A65
:10C6600046F8201DA2F124030020CDED007A02F847
:10C67000240C1E2208209A70BDF800105870304615
:10C6800008F058FDB4F9AC3107EE903AF8EEE77ACD
:10C69000304667EE887AFDEEE77ACDED007ABDF898
:10C6A000001008F047FDB4F9B03107EE903AF8EE0B
:10C6B000E77A304667EE887AFDEEE77ACDED007ACC
:10C6C000BDF8001008F036FD304624F02DFFFEF7CF
:10C6D000ABB9C4F84CB22E70FEF763B894F8EA0315
:10C6E000C0B10138C0B2344D01302844002215F8E1
:10C6F000013B534083EA0313DBB2120AD90042EA3A
:10C700000322A84281EA131382EA0302EFD1002A2E
:10C710007EF4AAAA244B294D244AD4F8F4031B889A
:10C720001168EB619268036BE962EA640021B4F876
:10C73000E423EE66E963EA65002B00F09D825B6806
:10C74000816C8B423BBFC2685B1A5B1A9B18002B43
:10C750007DF4A8AF036802219B699847042394F8ED
:10C76000EB0385F8743022F03DF9032384F8DC33C1
:10C77000FDF798BF022138680AF0D4FA94F85432D1
:10C78000FDF752BF3851002088820020E4380E3F68
:10C790000050C34798860020647003085C7003084B
:10C7A0007786002075860020A0820020A4820020C9
:10C7B0006766666658A08B41982000200000002024
:10C7C00074700308A3785E09012E40F0648103F0C1
:10C7D0000F0E13F0100300F07B81C64AE37827792F
:10C7E000A4F88603D11887EA0300C4F87C23134613
:10C7F00084F86662C4F88013073A84F88C03A4F8BE
:10C80000847394F88C03BC4F0CE012F8011BC4F83D
:10C810007C63BA4280EA0100197007D2D4F8801311
:10C82000D4F87C33994203F10106EED1BA4284F880
:10C830008C0300F03982127894F88C339A4200F01D
:10C84000C781AE4BC4F8683201330122B4F88413B7
:10C85000C4F86C3200204FF6F67384F86602A4F830
:10C86000701284F8782284F87823A4F87232FEF7E4
:10C8700070BC102300250422184606A98DF8183034
:10C880008DF819208DF81A508DF81B508DF81C501A
:10C890008DF81D5022F0F4FE84F86152FDF7EEBED3
:10C8A0003422FEF71FBF94F8AF33002B0CBF0422D5
:10C8B0000522FFF747BB924B93E8030006AB83E8E2
:10C8C0000300184622F09CFF3DE6102022F086FF70
:10C8D000284622F059FF284622F056FF212022F058
:10C8E0007DFF284622F050FF284622F04DFFFEF73C
:10C8F00023B84FF00308DFF8289250E6B4F972121B
:10C90000D4F86C72501C02F00F0242F010020029A1
:10C91000B8BF42F0200284F88E0394F870028DF8BC
:10C920001820BA1B5040C0B28DF8192084F88F032C
:10C930000DF11A02FEF73FBE724B1988FEF7B7BD24
:10C94000714B6420B3F900A0FEF7DAB91A46184615
:10C950001D4600939C46FFF7E6BB2422FEF7C2BEAD
:10C960006A4F97F80080B8F1000F3FF466ADDFF82A
:10C9700094A1B4F8C051BAF800302D016422ADB2D0
:10C9800002FB03834FEA4802B3FBF2F345EA0325B7
:10C99000ADB2C3F303231D43062022F01FFFE8B20C
:10C9A00022F0F2FE280A22F0EFFEB4F8C031584916
:10C9B000BAF8005001339BB293FBF8F208FB123334
:10C9C0004A7AA4F8C031012A00F087816E23514AC7
:10C9D000497B03FB05F382FB0302DB17C3EBA203D6
:10C9E000002940F075814C4D9FB2A5FB07356D09BC
:10C9F0003A201FFA85F822F0F1FE5FFA88F022F063
:10CA0000C3FE4FEA182022F0BFFE3B2022F0E6FED4
:10CA1000642303FB15739BB24048053380FB03205E
:10CA2000DB17C3EBA000C0B222F0AEFE002022F064
:10CA3000ABFE354F394D282022F0D0FE3B6885FBF8
:10CA40000325DB17C3EBA505E8B222F09DFEC5F375
:10CA5000072022F099FE042022F0C0FEB4F8BA317B
:10CA6000002B40F01481BD6885F31005E8B222F078
:10CA70008BFEC5F3072022F087FEDEE40121D4F807
:10CA8000C821D4F8CC3184F8DC1104A804920593B1
:10CA900022F0B6FE57E5194B84F866025E1C4FF68D
:10CAA000F6710122A4F8700284F87802C4F86832A2
:10CAB000C4F86C62A4F8721284F87823FEF749BBBC
:10CAC0004FF00408DFF85C9069E500252846AAE4E9
:10CAD00094F86622002A3EF43CAB94F88D23013290
:10CAE00002F00F02724500F0C18084F86632FEF752
:10CAF00030BB00BFBC1C0020B81C0020281F002039
:10CB0000AC490308A0820020A4820020DF8200201C
:10CB100088820020310CC3301F85EB516766666642
:10CB2000687003086C700308112022F057FEB4F8F7
:10CB3000D621784D4FF4F36707FB02F285FB0235EF
:10CB4000D217C2EB6535E8B222F01EFEC5F307200E
:10CB500022F01AFE192022F041FEB4F8D6316E4AB6
:10CB600007FB03F382FB0301DB17C3EB611382FBBB
:10CB70000321DA17C2EB6112642101FB1233D8B230
:10CB800022F002FE002022F0FFFD94F8C231B4F83A
:10CB9000D0519A077FF55BACEFB22D0A59E42846D5
:10CBA0002DE4484624F046FD8046F8E41022FEF7C6
:10CBB00099BD0099322022F063FDFEF729BD06AB36
:10CBC00000930DF11E05FEF713BD2022FEF78ABD6E
:10CBD000524BD4F87C23C4F88023002703F55B7202
:10CBE00003F51B76C4F86C2203F5177103F55C702E
:10CBF0003A46C4F86862C4F87C3384F86672A4F8D4
:10CC00007072A4F87272FBF7FBF9013058D0D4F8B7
:10CC10006832C4F86C320123C4F8686284F878334F
:10CC2000FEF797BAE8B222F0AFFD280A22F0ACFD79
:10CC30005FE43B4B1B6898067DF5B3AD94F8483232
:10CC4000002B7DF4E0AC374BC4F850322D2384F830
:10CC50005432FDF7B0BD4B1CDBB2042B84F8963385
:10CC60004FEA01613FF47FABFFF780BBD4F880133C
:10CC7000D4F87C332C4AC4E5C269036A9A423CBFAB
:10CC8000C1685218D31A62E50822FEF72BBD0CF0DA
:10CC90001DF822F079FD002022F076FDFFF7CDBBD4
:10CCA000224B1B68FFF74DBB84F88DE3FEF751BAAA
:10CCB0001A4618461D4600939C469846FFF733BA1D
:10CCC000D4F868320222591CC4F868121A709EE720
:10CCD0009BB23A7893FBF2F385E6392022F07EFD91
:10CCE000E8B222F051FD280A22F04EFDA1E61A46D4
:10CCF000FFF719BA1A461846FFF715BA1A4618462A
:10CD00001D46FFF710BA1A4618461D460093FFF756
:10CD10000ABA00BF89B5F8141F85EB51BC1C00206E
:10CD200038510020C81E0020B31C0020A48200201F
:10CD30002DE9F04FDFF808B12DED0C8B9BF800309A
:10CD40009BB0012B099002F04083394C94F80021EC
:10CD5000002A41F04983072B364D02F0318300232E
:10CD600005936B683348984700286ED0B5F8A870D3
:10CD7000002285F84920002F40F09182B5F9260065
:10CD80002A6BB5F92460E96AB5F92830DFF8B49068
:10CD9000821A686BEA63711A1B1AA963264895F810
:10CDA0004A102B6415F054FAD9F8003013F00053F0
:10CDB00002F0F880D5ED0F5AD5ED0E7A1F4A94EDAA
:10CDC000676AD4ED686A94ED697AD4F8A83112687C
:10CDD000B8EEE58AD5ED105AF8EEE77AF8EEE58A76
:10CDE000013377EE867A38EE268A78EE878A934288
:10CDF000C4ED677A84ED688AC4ED698AC4F8A83105
:10CE000001F040869BF80070142F03F0BD820023D0
:10CE1000D4F8B0610693062E02F26E83DFE816F0B6
:10CE2000F019BA180B136A19CF184818C01700BFA9
:10CE300094220020FC480020344900203C5100206E
:10CE4000F1810020386E0020069C9BF80090B9F11B
:10CE5000070F00F0DB8294F8B831002B40F0E3823A
:10CE6000CF4B5B79002B40F0158201239BF800200B
:10CE700084F8B831072A02F0698400230C93C94B67
:10CE8000D4ED709A93ED007AC74AC84B12680692A7
:10CE9000F7EE007A37EEE9CAC54A07922CEE07CAC8
:10CEA000C44AD4ED6F8ADFF88493DFEDC3AA9FED07
:10CEB000C39A9FEDC3BADFEDC3CA9FEDC3AADFEDEE
:10CEC000C3BADFF86C83DFF86CA3C14F0B93B4EEE9
:10CED000E7CA0025F1EE10FA089288BFB0EE67CAE3
:10CEE00005932E46BB4B2B44D3ED007ABA4BF5EE9F
:10CEF000407A2B44F1EE10FA93ED008A17D0B74B2D
:10CF00002B4493ED007A78EE476AB0EEE66AF4EED1
:10CF1000C67AF1EE10FA08D5F5EEC06AF1EE10FA15
:10CF2000CCBF37EE878A37EE678A83ED008A079B8E
:10CF30001888810700F07F82022E05F06180069933
:10CF4000A74B91F8322006EE902A33F916202B4495
:10CF500007EE102A13ED096A91F83130B8EEC77A5E
:10CF6000F8EEE66A5A4207EE902AA6EE867A71003B
:10CF7000F8EEE77AB4EEE77AF1EE10FA0AD407EEAB
:10CF8000903AF8EE677AF4EEC77AF1EE10FA88BFBD
:10CF9000F0EE477ADFF8A0C2924A0A920CEB010346
:10CFA000515EB3F90A30CA1A07EE102AB8EEC77AF2
:10CFB000C207E7EE497A40F1ED828B4890ED008A96
:10CFC00027EE888A94F8D001E0B18748D4F8D421BC
:10CFD00090ED008A85485B1A07EE903A099B01683C
:10CFE00028EE098AF8EEE77A981A884228EE278A0E
:10CFF00000F36782F7EE007AF4EEE79AF1EE10FAAA
:10D0000000F12B827A4B2B44D3ED007A059BD3EDB4
:10D0100001DA68EEA77A38EE6DDA67EE8D7ACAED3E
:10D02000007A089BD9ED007A93ED007A714BD7ED29
:10D03000006A67EE277A2B4427EE8C7AD3ED007ACC
:10D0400067EE277AB0EE667AA7EE8D7AF0EE477A31
:10D0500094ED706AB7EE007AB4EEC76AF1EE10FA9A
:10D06000ACBF0123002343B1F0EEE66AB0EEE77AED
:10D07000B4EEE67AF1EE10FA01D5C7ED007A022E91
:10D0800004F03C875C4A5D4B52F826001B68B0EE0A
:10D090006D0A98475A4A5B4B52F826001B6898471E
:10D0A000069B93F83A30632B04D8079B1B88002B10
:10D0B00001F06D81B0EE6C8A534B99ED007A38EE39
:10D0C000400A2B4493ED008A83ED000A069B30EE64
:10D0D000480A93F84830C0EE077ADBB1B7EE007A21
:10D0E000F4EEC79AF1EE10FA14DB484B93ED007A98
:10D0F000F0EEE76AF4EEC76AF1EE10FA0ADD444B8F
:10D1000093ED007AB0EECDDAB4EEC7DAF1EE10FAB4
:10D1100001F370823F4B94F8E0212B4493ED007AA9
:10D1200028EE877A67EE277AC8ED007A2AB9CAED29
:10D1300000CAC7ED00CAC8ED00CA059B0435043318
:10D140000C2D06F1010608F104080AF1040A07F1A2
:10D15000040705937FF4C6AE9BF80030072B02F05E
:10D160005581012B02F0F782002305932A4B0E4ACA
:10D170001B68126892F82F1013F48052069200F088
:10D1800087822648264F0278264D274EED8896ED59
:10D19000037A12F0010F3A8B08BFA4F8E8214DE0A2
:10D1A000E84800206C3A0020482000202051002050
:10D1B000442000207800002000009642CDCCCC3DD9
:10D1C000AE47813F000000000000C842610BB63B43
:10D1D0000C440020603A00209823002058240020AE
:10D1E000242400205C1E0020443A0020703A0020D5
:10D1F000183A0020243A0020883A0020843A00207F
:10D20000EC3A0020E83A00206C240020803A00200C
:10D210007C3A0020303A0020386E0020B4550020BF
:10D220000C5D002068400020E08200205C3A002075
:10D230001844002000440020407E0020A2EB050E90
:10D2400007EE90EAF8EEE77AB4EEE77AF1EE10FA3C
:10D2500042F26981561906EE906AF8EEE66AB4EE7B
:10D26000E67AF1EE10FA81F2E183B4F8E82196450E
:10D2700083F24686B54AB64DD2ED004AD5ED003A66
:10D28000B44AC4ED7B3AC4ED7C4AD2ED006ADFEDCE
:10D29000B27A16E2B14B1B78013BDBB2E6E5B04B4C
:10D2A000B0490B9391F801A01B68DFF8E0829BF86E
:10D2B0000090B8F906004FF47A71B1FBF3F3C3EBB9
:10D2C000431603EB8603DE00B6B2B74203F0E280FA
:10D2D000E96FB5F924E02B6E4A1C07EE90EA73441F
:10D2E000012AEA672B66F8EEE77A03F0DD80D5EDD8
:10D2F0001B5AD5ED1D6A07EE102A37EEE56AB8EE27
:10D30000C75A012F86EE057A37EE257A77EEC77A6F
:10D3100085ED1C7AE6EE276A85ED1B7AF0EE667ADB
:10D32000C5ED1E6AC5ED1D6A03F04886D5F890105C
:10D33000B5F926E06B6E4A1C07EE90EA7344012AA9
:10D34000C5F890206B66F8EEE77A03F0C580D5ED5E
:10D35000205AD5ED226A07EE102A37EEE56AB8EEBC
:10D36000C75A012F86EE057A37EE257A77EEC77A0F
:10D3700085ED217AE6EE276A85ED207AF0EE667A71
:10D38000C5ED236AC5ED226A03F04E86D5F8A410D8
:10D39000B5F928E0AB6E4A1C07EE90EA7344012A07
:10D3A000C5F8A420AB66F8EEE77A03F0AE80D5EDC1
:10D3B000255AD5ED276A07EE102A37EEE56AB8EE52
:10D3C000C75A012F86EE057A37EE257A77EEC77AAF
:10D3D00085ED267AE6EE276A85ED257AF0EE667A07
:10D3E000C5ED286AC5ED276A03F01186A8F8060086
:10D3F000013F9BF80090A5F8A8700B990023B9F1A4
:10D40000070F4B608B60CB607FF425AD09F050FABD
:10D41000059BDFF87881C01A94F8B831A8F80000AD
:10D42000002B3FF41DAD013B84F8B8311BB0BDECBF
:10D430000C8BBDE8F08F94F8D031002B45D0022E34
:10D4400004F09A85DFF848C1474A0A920CEB46037C
:10D4500032F91610B3F90A30B7E50A9B4349B3F91C
:10D460000000BCF90A300968C21A82EAE273A3EB31
:10D47000E2738B42BFF6C6AD0A9BBCF90C20B3F930
:10D4800002309A1A82EAE273A3EBE27399427FF7C1
:10D49000B9AD0B99364BD1ED017A93ED007AF0EEF0
:10D4A000E77AF4EEC77AF1EE10FA7FF5ABADD1ED85
:10D4B000027AF0EEE77AB4EEE77AF1EE10FA7FF74F
:10D4C000A1AD002384F8D0319CE52A4B2B4493ED89
:10D4D000000A059BD3ED01DA28EE800A38EE6DDAFA
:10D4E000022E20EE0D0A8AED000A7FF49AAD224A40
:10D4F000224B10681B689847089B99ED007AD3ED82
:10D50000007A1F4BD7ED006A1A781E4B83ED020A92
:10D510001D4B67EE277A2B4467EE8C7A93ED006AF9
:10D5200067EE867AB0EE667AA7EE8D7A012AF0EE83
:10D53000477A02D0192A7FF48BADB4EEEADAF1EE25
:10D5400010FACCBF012300238DE500BF604000200E
:10D55000247E00207840002000000000347E00205F
:10D5600020510020E84800205C1E0020743A002072
:10D57000783A0020183A00204C3F0020603F0020FD
:10D58000AC38002000440020243A0020F481002020
:10D59000407E0020D4ED5E6A94ED5F7A0A9AB4EE84
:10D5A000E67AF1EE10FAB2F90200B2F900E00D905D
:10D5B0004BBFB7EE007AF7EE006A77EE665A76EE6A
:10D5C000C75A8EEAEE720028A2EBEE72B8BF404254
:10D5D000824200F3CF870D9A2948002AD8BF5242D1
:10D5E00007EE102A0078B8EEC77A27EE097A0028ED
:10D5F00000F0D287234890ED005AB5EEC05AF1EE04
:10D6000010FA41F3F7862048D0ED004AF5EEC04A03
:10D61000F1EE10FA41F3EE8634EEC77AB7EE006A07
:10D62000C7EE246A75EEC65AF4EEC66A65EE8A5AEB
:10D63000F1EE10FA85EE857A88BFF0EE466AF5EED7
:10D64000C06AF1EE10FA37EE067AB8BFF0EE6C6AF7
:10D6500066EE876AF4EEC66AF1EE10FA88BFF0EE65
:10D66000466AF5EEC06AF1EE10FAB8BFF0EE6C6AE9
:10D67000064890ED007A67EE877AA7EEA68AA1E4C5
:10D68000503A00204C3A0020543A0020483A0020FA
:10D69000E14FE24A788B92ED037AE14A07EE900A75
:10D6A000E048D2ED003AE04AD0ED004AD2ED006AFF
:10D6B000DE48C4ED7C4AF8EEE77AC4ED7B3A77EEBB
:10D6C000677AC7EEA65ADA4DDA4A95ED005ADA4D76
:10D6D0009FEDDA7A95ED003AD94D9FEDDA6A95ED36
:10D6E000004AD2ED006AF7EE007AF4EEE75A35EE22
:10D6F000035AF1EE10FA88BFF0EE675A35EE045A7D
:10D70000F4EEC75AF1EE10FA25EE065AB8BFF0EE65
:10D71000475AB1EE667A33EEE43AB4EEC75AF1EE08
:10D7200010FAC4ED7D5A84ED7F3A00F17184B4EEB5
:10D73000E65AF1EE10FA88BFB0EE665ABC4A9FED89
:10D74000C16AD2ED017ABC4AD2ED012ABC4A77EE19
:10D75000A27A92ED014A77EE847A67EE867AB4EE89
:10D76000E77AF1EE10FA08DCF4EEE76AF1EE10FA6F
:10D770008CBFB0EE677AB0EE667AAD4A9FEDB16AC3
:10D78000D2ED027AAC4A92ED024AAF4A77EE847A41
:10D79000D2ED006A67EE867AB1EE664AF4EEC47A9C
:10D7A000F1EE10FA08D4F4EEE67AF1EE10FA8CBF3E
:10D7B000B0EE664AB0EE674A002941F0F081B7EE5C
:10D7C000002AA24AA24E527894F80012002AFFEED4
:10D7D000002AB7EE006A327814BFF0EE467AF0EE17
:10D7E000627A002914BFF0EE626AF0EE466A002AFF
:10D7F00002F0F486B4EEC62AF1EE10FA24EE274ABF
:10D80000944941F30D8291ED026A91ED011AD1ED37
:10D81000037ADFED8A1A27EE066A62EE262AA1EE67
:10D82000056AA7EE846A26EE226AB4EEE16AF1EE9A
:10D8300010FAB4BFF0EE617AF0EE467A8DED0E6A22
:10D8400088BFB0EE616A012A00F0BE81D1ED066AA0
:10D85000D1ED051A91ED072A67EE266AE1EE856A99
:10D86000E2EE046A66EEA26AF4EEC66AF1EE10FA1F
:10D87000F4EEE76A8CBFB0EE462AB0EE662AF1EE0F
:10D8800010FA98BFB0EE426AA8BFF0EE667A022A9C
:10D89000CDED0F6A00F09881D1ED0A6AD1ED091A39
:10D8A00091ED0B2A67EE266AE1EE856AE2EE046AE4
:10D8B00066EEA26AF4EEC66AF1EE10FAF4EEE76ADA
:10D8C0008CBFB0EE462AB0EE662AF1EE10FA98BF91
:10D8D000B0EE426AA8BFF0EE667A032ACDED106A78
:10D8E00000F07281D1ED0E6AD1ED0D1A91ED0F2A83
:10D8F00067EE266AE1EE856AE2EE046A66EEA26AE7
:10D90000F4EEC66AF1EE10FAF4EEE76A8CBFB0EE00
:10D91000462AB0EE662AF1EE10FA98BFB0EE426ADF
:10D92000A8BFF0EE667A042ACDED116A00F04C81B2
:10D93000D1ED126AD1ED111A91ED132A67EE266A24
:10D94000E1EE856AE2EE046A66EEA26AF4EEC66A69
:10D95000F1EE10FAF4EEE76A8CBFB0EE462AB0EEB4
:10D96000662AF1EE10FA98BFB0EE426AA8BFF0EE58
:10D97000667A052ACDED126A00F02681D1ED166A8D
:10D98000D1ED151A91ED172A67EE266AE1EE856A48
:10D99000E2EE046A66EEA26AF4EEC66AF1EE10FAEE
:10D9A000F4EEE76A8CBFB0EE462AB0EE662AF1EEDE
:10D9B00010FA98BFB0EE426AA8BFF0EE667A062A67
:10D9C000CDED136A00F00081D1ED1A6AD1ED191A7C
:10D9D00091ED1B2A67EE266AE1EE856AE2EE046AA3
:10D9E00066EEA26AB4EEE66AF1EE10FAF4EEE67ABA
:10D9F0008CBFB0EE662AB0EE462AF1EE10FA58BFA0
:10DA0000B0EE426AB8BFF0EE667A072ACDED146A2E
:10DA100000F0DA8020E000BF0C5D0020E0820020F2
:10DA2000247E00208C7C002070400020B455002013
:10DA300000440020643F00200C440020000000004F
:10DA4000184400206F12833A683F002028220020EB
:10DA50006C710020A03F0020D1ED1E6AD1ED1D1A8F
:10DA600091ED1F2A67EE266AE5EE216AE4EE026A6E
:10DA700066EEA26AF4EEC66AF1EE10FAF4EEE76A18
:10DA80008CBFB0EE462AB0EE662AF1EE10FA98BFCF
:10DA9000B0EE426AA8BFF0EE667A082ACDED156AAC
:10DAA00000F09280D1ED226AD1ED211A91ED232A66
:10DAB00067EE266AE5EE216AE4EE026A66EEA26A85
:10DAC000F4EEC66AF1EE10FAF4EEE76A8CBFB0EE3F
:10DAD000462AB0EE662AF1EE10FA98BFB0EE426A1E
:10DAE000A8BFF0EE667A092ACDED166A6CD0D1EDAA
:10DAF000266AD1ED251A91ED272A67EE266AE1EE16
:10DB0000856AE4EE026A66EEA26AF4EEC66AF1EE97
:10DB100010FAF4EEE76A8CBFB0EE462AB0EE662A41
:10DB2000F1EE10FA98BFB0EE426AA8BFF0EE667A46
:10DB30000A2ACDED176A47D0D1ED2A6AD1ED291A0C
:10DB400091ED2B2A67EE266AE1EE856AE2EE046A21
:10DB500066EEA26AF4EEC66AF1EE10FAF4EEE76A37
:10DB60008CBFB0EE462AB0EE662AF1EE10FA98BFEE
:10DB7000B0EE426AA8BFF0EE667A0B2ACDED186AC5
:10DB800022D0D1ED2E1A91ED2D2AD1ED2F6A27EE5C
:10DB9000217AA2EE057AA6EE847A27EE227AB4EEF6
:10DBA000C67AF1EE10FAF4EEC77A8CBFF0EE466A50
:10DBB000F0EE476AF1EE10FA8DED197AA8BFB0EEDB
:10DBC000666AB8BFF0EE477A77EEC67AF7EE006A7B
:10DBD000F4EEE67AF1EE10FAC4ED707A43F37A814E
:10DBE00086EEA77A012ADDED0E7A67EE877ACDED13
:10DBF0000E7A55D0DDED0F7A67EE877A022ACDEDE9
:10DC00000F7A4DD0DDED107A67EE877A032ACDEDDD
:10DC1000107A45D0DDED117A67EE877A042ACDEDD2
:10DC2000117A3DD0DDED127A67EE877A052ACDEDC7
:10DC3000127A35D0DDED137A67EE877A062ACDEDBC
:10DC4000137A2DD0DDED147A67EE877A072ACDEDB1
:10DC5000147A25D0DDED157A67EE877A082ACDEDA6
:10DC6000157A1DD0DDED167A67EE877A092ACDED9B
:10DC7000167A15D0DDED177A67EE877A0A2ACDED90
:10DC8000177A0DD0DDED187A67EE877A0B2ACDED85
:10DC9000187A05D0DDED197A27EE877A8DED197A9D
:10DCA000DD49096811F0805100F05F84F6EE005AFA
:10DCB000C4ED7D5A0078002A02F0AB84DFF870933F
:10DCC000D64DDFF870A3DFF870C394F8F8E17F8BCE
:10DCD0000797FDEEE37AD9ED006A9AF80380B5F96B
:10DCE00006909CF800C003F0100700F0010003F458
:10DCF000800317EE905ABEF1000F40F09F81002F75
:10DD000000F01C85002843F09480B8F1000F43F028
:10DD10001E81C349DDED0E7A91ED007AC14BE7EE2D
:10DD2000257ABDEEE47A17EE100AB0EE647AA3EE1F
:10DD3000277AFDEEC77A17EE90EA17EE907AAE4595
:10DD4000A8BF2F467045C8BF074607EE907AF8EE89
:10DD5000E77A012AC3ED007A00F04D8191ED047A53
:10DD6000DDED0F7AE7EE257AB0EE647AA3EE277A3E
:10DD7000FDEEC77A17EE90EA17EE907AAE45A8BF8F
:10DD80002F468645B8BF074607EE907AF8EEE77A49
:10DD9000022AC3ED017A00F02E8191ED087ADDEDC3
:10DDA000107AE7EE257AB0EE647AA3EE277AFDEEDC
:10DDB000C77A17EE90EA17EE907AAE45A8BF2F46C5
:10DDC0008645B8BF074607EE907AF8EEE77A032A51
:10DDD000C3ED027A00F00F8191ED0C7ADDED117A3E
:10DDE000E7EE257AB0EE647AA3EE277AFDEEC77AE5
:10DDF00017EE90EA17EE907AAE45A8BF2F468645FB
:10DE0000B8BF074607EE907AF8EEE77A042AC3ED2A
:10DE1000037A00F0F08091ED107ADDED127AE7EEF2
:10DE2000257AB0EE647AA3EE277AFDEEC77A17EE74
:10DE300090EA17EE907AAE45A8BF2F468645B8BF48
:10DE4000074607EE907AF8EEE77A052AC3ED047AE2
:10DE500000F0D18091ED147ADDED137AE7EE257AAA
:10DE6000B0EE647AA3EE277AFDEEC77A17EE90EA59
:10DE700017EE907AAE45A8BF2F468645B8BF074635
:10DE800007EE907AF8EEE77A062AC3ED057A00F0FD
:10DE9000B28091ED187ADDED147AE7EE257AB0EED6
:10DEA000647AA3EE277AFDEEC77A17EE90EA17EEB2
:10DEB000907AAE45A8BF2F468645B8BF074607EE05
:10DEC000907AF8EEE77A072AC3ED067A00F093809D
:10DED00091ED1C7ADDED157AE7EE257AB0EE647AE5
:10DEE000A3EE277AFDEEC77A17EE90EA17EE907A46
:10DEF000AE45A8BF2F468645B8BF074607EE907AC5
:10DF0000F8EEE77A082AC3ED077A74D091ED207A0B
:10DF1000DDED167AE7EE257AB0EE647AA3EE277A85
:10DF2000FDEEC77A17EE90EA17EE907AAE45A8BFDD
:10DF30002F468645B8BF074607EE907AF8EEE77A97
:10DF4000092AC3ED087A56D091ED247ADDED177ACF
:10DF5000E7EE257AB0EE647AA3EE277AFDEEC77A73
:10DF600017EE90EA17EE907AAE45A8BF2F46864589
:10DF7000B8BF074607EE907AF8EEE77A0A2AC3EDB3
:10DF8000097A38D091ED287ADDED187AE7EE257A16
:10DF9000B0EE647AA3EE277AFDEEC77A17EE90EA28
:10DFA00017EE907AAE45A8BF2F468645B8BF074604
:10DFB00007EE907AF8EEE77A0B2AC3ED0A7A1AD0C8
:10DFC00091ED2C7ADDED197AE7EE257AE3EE274A1A
:10DFD000FDEEE47A17EE901A8D42A8BF0D468842F6
:10DFE000D8BF284607EE900AF8EEE77AC3ED0B7A21
:10DFF000002A00F0A48192000B490A4826F0F7FAA3
:10E000000A4B1B68002B00F09F8110F03FFE9BE144
:10E01000B0EE475AFFF792BB047E00200422002096
:10E02000A03F002044440020703F0020143A00200C
:10E030006C3F00205C20002040580020002F40F062
:10E04000FD82E049DDED0E7A91ED007ADE4BE7EEE0
:10E05000257AB1EE433AB0EE637AA3EE277AF0EE7A
:10E06000477ABCF1000F41F09983B8F1000F43F0FB
:10E070006882FDEEE77ABDEEE47A17EE90CA17EEFD
:10E0800090EAAC4517EE107AA8BFAE466745C8BF08
:10E09000BE4607EE90EAF8EEE77A012AC3ED007A71
:10E0A00000F04A8191ED047ADDED0F7AE7EE257AF2
:10E0B000B0EE637AA3EE277AFDEEC77A17EE90CA28
:10E0C00017EE90EAAC45A8BFAE46BC45B8BFBE4609
:10E0D00007EE90EAF8EEE77A022AC3ED017A00F043
:10E0E0002B8191ED087ADDED107AE7EE257AB0EE1E
:10E0F000637AA3EE277AFDEEC77A17EE90CA17EE81
:10E1000090EAAC45A8BFAE46BC45B8BFBE4607EED8
:10E1100090EAF8EEE77A032AC3ED027A00F00C8168
:10E1200091ED0C7ADDED117AE7EE257AB0EE637AA7
:10E13000A3EE277AFDEEC77A17EE90CA17EE90EAA3
:10E14000AC45A8BFAE46BC45B8BFBE4607EE90EA98
:10E15000F8EEE77A042AC3ED037A00F0ED8091ED42
:10E16000107ADDED127AE7EE257AB0EE637AA3EE4F
:10E17000277AFDEEC77A17EE90CA17EE90EAAC4503
:10E18000A8BFAE46BC45B8BFBE4607EE90EAF8EE63
:10E19000E77A052AC3ED047A00F0CE8091ED147A77
:10E1A000DDED137AE7EE257AB0EE637AA3EE277AF7
:10E1B000FDEEC77A17EE90CA17EE90EAAC45A8BFFD
:10E1C000AE46BC45B8BFBE4607EE90EAF8EEE77A29
:10E1D000062AC3ED057A00F0AF8091ED187ADDEDE7
:10E1E000147AE7EE257AB0EE637AA3EE277AFDEE95
:10E1F000C77A17EE90CA17EE90EAAC45A8BFAE46B4
:10E20000BC45B8BFBE4607EE90EAF8EEE77A072AAB
:10E21000C3ED067A00F0908091ED1C7ADDED157A61
:10E22000E7EE257AB0EE637AA3EE277AFDEEC77AA1
:10E2300017EE90CA17EE90EAAC45A8BFAE46BC45B3
:10E24000B8BFBE4607EE90EAF8EEE77A082AC3EDBB
:10E25000077A71D091ED207ADDED167AE7EE257A16
:10E26000B0EE637AA3EE277AFDEEC77A17EE90CA76
:10E2700017EE90EAAC45A8BFAE46BC45B8BFBE4657
:10E2800007EE90EAF8EEE77A092AC3ED087A53D050
:10E2900091ED247ADDED177AE7EE257AB0EE637A18
:10E2A000A3EE277AFDEEC77A17EE90CA17EE90EA32
:10E2B000AC45A8BFAE46BC45B8BFBE4607EE90EA27
:10E2C000F8EEE77A0A2AC3ED097A35D091ED287A7B
:10E2D000DDED187AE7EE257AB0EE637AA3EE277AC1
:10E2E000FDEEC77A17EE90CA17EE90EAAC45A8BFCC
:10E2F000AE46BC45B8BFBE4607EE90EAF8EEE77AF8
:10E300000B2AC3ED0A7A17D091ED2C7ADDED197A3C
:10E31000E7EE257AE3EE273AFDEEE37A17EE901A60
:10E320008D42A8BF0D468F42D8BF2F4607EE907A88
:10E33000F8EEE77AC3ED0B7A00283FF459AE234B91
:10E340001B68002B7FF461AE214B1B7893B13078B2
:10E3500068B11D4FDFF88C800025E8B2D8F8003096
:10E36000B7EC010A9847307801358542F5DB194B47
:10E370001B6898479BF80030072B01F03F80012372
:10E3800084F800311BB0BDEC0C8BBDE8F08F124B54
:10E39000124A2B4493ED007AD2ED007A104B67EECF
:10E3A000277AF7EE006AF4EEE67AF1EE10FA93EDD2
:10E3B000007A88BFF0EE667A67EE877A27EE888A61
:10E3C000FEF77ABEA03F002044440020143A00200B
:10E3D000A85C00203C5800200C240020403A00207B
:10E3E0003C3A002034580020072B02F06E850023B1
:10E3F0000593DFF84093C04DD9F800305F0501F177
:10E400000981DFF834A3DAF8008018F0080F41F032
:10E41000A680BA4B1B78002B40F0F480B84F94F8DC
:10E42000126126B1B74B1B889B0742F0EE8294F82D
:10E430001811FB7F002941F02981BE7F002E00F0DA
:10E440000D86022E02F0AE80032E01F09784AE4AB4
:10E4500052880233DBB2002902F09880002A02F0D1
:10E460009580AA480668B2FBF6F216B2A4F8486195
:10E47000002B03F0188307EE906AF8EEE77AF7EEC8
:10E48000006A86EEA77AA24A012BD4ED576AD2ED34
:10E49000007A77EEE67A67EE877AC4ED537A21D078
:10E4A000D2ED017AD4ED586A77EEE67A022B67EE68
:10E4B000877AC4ED547A15D0D2ED027AD4ED596A38
:10E4C00077EEE67A032B67EE877AC4ED557A09D0AA
:10E4D000D2ED037AD4ED5A6A77EEE67A67EE877A60
:10E4E000C4ED567A9BF80000092803F0A783002E9C
:10E4F00040F3BA8593B3D4ED577A94ED537A77EE1F
:10E50000877A012BC4ED577AC2ED007A21D0D4ED81
:10E51000587A94ED547A77EE877A022BC4ED587AC4
:10E52000C2ED017A15D0D4ED597A94ED557A77EE93
:10E53000877A032BC4ED597AC2ED027A09D0D4ED63
:10E540005A7A94ED567A77EE877AC4ED5A7AC2ED0C
:10E55000037A013B022BB8BF0223DBB200290CBFB8
:10E560009E464FF0020E00F081BD5D023FF59EAB6E
:10E57000FFF7A0BBBEF1000FD6BFCEF1000207EE41
:10E5800010EA07EE102A6348B8EEC77A007827EE43
:10E59000097A00287FF42EA85F4890ED006AB4EE57
:10E5A000CB6AF1EE10FA40F1D587B7EE005A35EE9E
:10E5B000465ADFED5A6A5A4836EEC77A25EE2B5A8C
:10E5C000D0ED006AA5EE076A26EE267AB5EEC07A8F
:10E5D000F1EE10FA40F20E87CAEE076AB7EE006A53
:10E5E00035EEC67AF0EE465AE7EE265AF0EE656A48
:10E5F000FFF730B80123099AC4F8D42184F8D03148
:10E60000FEF788BD474B3E4FB3F906207B8B9A42FD
:10E610003FF705AF444B1B78012B01F0A287192B64
:10E6200001F09F870E2B3FF4FAAE082B3FF4F7AEB4
:10E63000374A00239360C4F80C31F0E6002842F01A
:10E640002182BCF1000F41F02E83FDEEE47A0DF142
:10E65000380C17EE90EAFDEEE67A0CEB8203069397
:10E660004FFA88F188F00103DFF8C0A0DFF8C0900E
:10E67000089417EE907AB1EE433A079218460C468A
:10E68000534693ED007AFCEC017AE7EE257A0AF125
:10E69000100AB0EE637AA3EE277AFDEEC77A17EE82
:10E6A000903A17EE902AAB42A8BF2A469F42CCBFB1
:10E6B000002108F00101002914BF114639469E458A
:10E6C000CCBF002300F0010307EE901A002B14BF0B
:10E6D00013467346B8EEE77A07EE903A069BF8EEDB
:10E6E000E77A002C18BFF0EE477A6345E9EC017A2F
:10E6F000C6D1079A089C7BE4FC480020F004002067
:10E700000C5D002044200020F821002078440020E7
:10E71000E0820020503A0020583A002000003443A4
:10E720004C3A00200422002028220020A03F002094
:10E7300044440020386E002038510020CC49DDEDE3
:10E740000E7A91ED007ACB4BE7EE257AB8F1000F07
:10E7500042F00A82BDEEE47A17EE107AB0EE647AE7
:10E76000A3EE277AFDEEC77A17EE90CA17EE90EA6D
:10E77000AC45A8BFAE466745C8BFBE4607EE90EAA7
:10E78000F8EEE77A012AC3ED007A3FF4D5AD91EDBA
:10E79000047ADDED0F7AE7EE257AB0EE647AA3EE27
:10E7A000277AFDEEC77A17EE90CA17EE90EAAC45CD
:10E7B000A8BFAE466745C8BFBE4607EE90EAF8EE72
:10E7C000E77A022AC3ED017A3FF4B6AD91ED087AFB
:10E7D000DDED107AE7EE257AB0EE647AA3EE277AC3
:10E7E000FDEEC77A17EE90CA17EE90EAAC45A8BFC7
:10E7F000AE46BC45B8BFBE4607EE90EAF8EEE77AF3
:10E80000032AC3ED027A3FF497AD91ED0C7ADDED6A
:10E81000117AE7EE257AB0EE647AA3EE277AFDEE60
:10E82000C77A17EE90CA17EE90EAAC45A8BFAE467D
:10E83000BC45B8BFBE4607EE90EAF8EEE77A042A78
:10E84000C3ED037A3FF478AD91ED107ADDED127AE5
:10E85000E7EE257AB0EE647AA3EE277AFDEEC77A6A
:10E8600017EE90CA17EE90EAAC45A8BFAE46BC457D
:10E87000B8BFBE4607EE90EAF8EEE77A052AC3ED88
:10E88000047A3FF459AD91ED147ADDED137AE7EE99
:10E89000257AB0EE647AA3EE277AFDEEC77A17EEFA
:10E8A00090CA17EE90EAAC45A8BFAE46BC45B8BFCB
:10E8B000BE4607EE90EAF8EEE77A062AC3ED057A3F
:10E8C0003FF43AAD91ED187ADDED147AE7EE257A52
:10E8D000B0EE647AA3EE277AFDEEC77A17EE90CAFF
:10E8E00017EE90EAAC45A8BFAE46BC45B8BFBE46E1
:10E8F00007EE90EAF8EEE77A072AC3ED067A3FF4CE
:10E900001BAD91ED1C7ADDED157AE7EE257AB0EEC0
:10E91000647AA3EE277AFDEEC77A17EE90CA17EE57
:10E9200090EAAC45A8BFAE46BC45B8BFBE4607EEB0
:10E9300090EAF8EEE77A082AC3ED077A3FF4FCACD8
:10E9400091ED207ADDED167AE7EE257AB0EE647A65
:10E95000A3EE277AFDEEC77A17EE90CA17EE90EA7B
:10E96000AC45A8BFAE46BC45B8BFBE4607EE90EA70
:10E97000F8EEE77A092AC3ED087A3FF4DDAC91EDB1
:10E98000247ADDED177AE7EE257AB0EE647AA3EE0D
:10E99000277AFDEEC77A17EE90CA17EE90EAAC45DB
:10E9A000A8BFAE46BC45B8BFBE4607EE90EAF8EE3B
:10E9B000E77A0A2AC3ED097A3FF4BEAC91ED287AD2
:10E9C000DDED187AE7EE257AB0EE647AA3EE277AC9
:10E9D000FDEEC77A17EE90CA17EE90EAAC45A8BFD5
:10E9E000AE46BC45B8BFBE4607EE90EAF8EEE77A01
:10E9F0000B2AC3ED0A7A3FF49FAC91ED2C7ADDED42
:10EA0000197AE7EE257AE3EE274AFDEEE47A17EE6F
:10EA1000901A8D42A8BF0D46B942A8BF2F4607EEF7
:10EA2000907AF8EEE77AC3ED0B7A85E407EE902A48
:10EA3000F8EEE77A104EDFF848C0D6ED004ADCED7C
:10EA4000003A0E4EC4ED7B3A77EE677A06EE905AA6
:10EA5000BCEEC77AF8EEE66A17EE102A77EEE67A91
:10EA6000C4ED7C4AA4F8E821D6ED006AFEF729BE81
:10EA7000A03F002044440020604000207840002057
:10EA8000247E002007EE103A9BF80030DFF88881E2
:10EA9000C4F8A871B8EEC77AF7EE006A132B86EEB9
:10EAA000879AB8F90400B4F8AC6195ED080A01F052
:10EAB0007C84534B534A93ED001AD3ED093A93EDFE
:10EAC000162A93ED1F3AD3ED0B1AD3ED144A93EDAA
:10EAD000016A93ED0A4A93ED0C7AD3ED155AD3ED02
:10EAE000172AD3ED206A93ED045AD3ED030A69EE99
:10EAF000277A69EE288A29EE088AE7EE813A02EB46
:10EB000086070021A2EE283AC4F89C11C4F8A0118F
:10EB1000E1EE884AA7EE864AE8EE075A93ED1A7AA4
:10EB200093ED0F6A93ED021AD3ED0E1AC7ED003A7A
:10EB3000E2EEA86A25EE635A27EE437A93ED0D2A9A
:10EB4000D3ED192AC7ED204AA3EEE04A26EE646A07
:10EB5000D3ED183A83ED094AA7EE815AF0EE477AD1
:10EB6000E1EEE45AA8EE026AE2EEC36AE3EEA87AA6
:10EB700083ED0A5AC3ED145A83ED156A87ED403AC6
:10EB8000C3ED1F6AC3ED207AC4F8A411731C03F00F
:10EB90001F03A4F8AC31A8F80400FEF733B91A4AF1
:10EBA000117900293EF40BAE1849097800293EF48A
:10EBB00006AE1278DFED162A07EE902A154AF8EE17
:10EBC000676A128807EE901A06EE102AF8EEE77AC6
:10EBD000B8EE466A66EEA77AF7EE006A87EE862AF6
:10EBE000B4EEE22AF1EE10FA88BFB0EE622AB4EE7B
:10EBF000E62AF1EE10FAB8BFB0EE662AFEF7E1BDE4
:10EC0000FC53002060510020641E0020DF820020A1
:10EC1000713DAA3FA0820020F48100200000000086
:10EC200091ED026A91ED012AD1ED037A5FED052A9B
:10EC300027EE066AA5EE026AA7EE846A26EE266A29
:10EC4000B4EEE26AF1EE10FAB4BFF0EE627AF0EEE2
:10EC5000467A8DED0E6A88BFB0EE626A012A3EF4F4
:10EC6000B3AFD1ED062AD1ED051A91ED072A67EE73
:10EC7000222AE5EE212AE2EE042A62EEA62AF4EE2A
:10EC8000C62AF1EE10FAF4EEE72A8CBFB0EE462A5F
:10EC9000B0EE622AF1EE10FA98BFB0EE426AA8BF59
:10ECA000F0EE627A022ACDED0F2A3EF48DAFD1ED5F
:10ECB0000A2AD1ED091A91ED0B2A67EE222AE5EE18
:10ECC000212AE2EE042A62EEA62AF4EEC62AF1EE2A
:10ECD00010FAF4EEE72A8CBFB0EE462AB0EE622AB4
:10ECE000F1EE10FA98BFB0EE426AA8BFF0EE627A79
:10ECF000032ACDED102A3EF467AFD1ED0E2AD1EDF7
:10ED00000D1A91ED0F2A67EE222AE5EE212AE2EE96
:10ED1000042A62EEA62AF4EEC62AF1EE10FAF4EE08
:10ED2000E72A8CBFB0EE462AB0EE622AF1EE10FA66
:10ED300098BFB0EE426AA8BFF0EE627A042ACDED29
:10ED4000112A3EF441AFD1ED122AD1ED111A91ED05
:10ED5000132A67EE222AE5EE212AE2EE042A62EE69
:10ED6000A62AF4EEC62AF1EE10FAF4EEE72A8CBFDA
:10ED7000B0EE462AB0EE622AF1EE10FA98BFB0EE7D
:10ED8000426AA8BFF0EE627A052ACDED122A3EF45F
:10ED90001BAFD1ED162AD1ED151A91ED172A67EEAA
:10EDA000222AE5EE212AE2EE042A62EEA62AF4EEF9
:10EDB000C62AF1EE10FAF4EEE72A8CBFB0EE462A2E
:10EDC000B0EE622AF1EE10FA98BFB0EE426AA8BF28
:10EDD000F0EE627A062ACDED132A3EF4F5AED1EDBF
:10EDE0001A2AD1ED191A91ED1B2A67EE222AE5EEB7
:10EDF000212AE2EE042A62EEA62AF4EEC62AF1EEF9
:10EE000010FAF4EEE72A8CBFB0EE462AB0EE622A82
:10EE1000F1EE10FA98BFB0EE426AA8BFF0EE627A47
:10EE2000072ACDED142A3EF4CFAED1ED1E2AD1ED46
:10EE30001D1A91ED1F2A67EE222AE5EE212AE2EE45
:10EE4000042A62EEA62AF4EEC62AF1EE10FAF4EED7
:10EE5000E72A8CBFB0EE462AB0EE622AF1EE10FA35
:10EE600098BFB0EE426AA8BFF0EE627A082ACDEDF4
:10EE7000152A3EF4A9AED1ED222AD1ED211A91ED49
:10EE8000232A67EE222AE5EE212AE2EE042A62EE28
:10EE9000A62AF4EEC62AF1EE10FAF4EEE72A8CBFA9
:10EEA000B0EE462AB0EE622AF1EE10FA98BFB0EE4C
:10EEB000426AA8BFF0EE627A092ACDED162A3EF426
:10EEC00083AED1ED262AD1ED251A91ED272A67EEE2
:10EED000222AE5EE212AE2EE042A62EEA62AF4EEC8
:10EEE000C62AF1EE10FAF4EEE72A8CBFB0EE462AFD
:10EEF000B0EE622AF1EE10FACDED172A98BFB0EE0F
:10EF0000426AB8BFF0EE672A0A2A02F0E984D1ED1E
:10EF10002A7AD1ED291A91ED2B2A67EE277AE1EEB4
:10EF2000857AE2EE047A67EEA67AF4EEC67AF1EE1E
:10EF300010FAF4EEE27A8CBFB0EE462AB0EE672A01
:10EF4000F1EE10FACDED187A98BFB0EE426AB8BF74
:10EF5000F0EE627A0B2A3EF437AED1ED2E2AD1EDD7
:10EF60002D1A91ED2F2A67EE222AE5EE212AE2EEF4
:10EF7000042A62EEA62AB4EEE26AF1EE10FAF4EE8A
:10EF8000E27A8CBFB0EE627AB0EE467AF1EE10FA19
:10EF9000CDED192A58BFB0EE476AB8BFF0EE627ADD
:10EFA000FEF712BED44A0B920026CA46D34FDFF8B2
:10EFB0006C83DDF82C9006943446B7EC018AD5EDCD
:10EFC000087AB8EEC88A28EE278A002C02F06E87ED
:10EFD0006BBB9BF80030082B39D006F5D260B0EE41
:10EFE000480A2844D5F88C36984706F5E360D5F8EA
:10EFF0001437284498479BF80030032BB0EE408A22
:10F0000020D0D5F8AC30D7F84406B0EE480A98477F
:10F0100009EB84030134032C06F12C0683ED010A6D
:10F020003DF412AFDAF8003003F00053C5E706F5FF
:10F03000F460B0EE480A2844D5F89C379847B0EE03
:10F04000408AC6E723F0E0F928F81400D9E7B0EECB
:10F05000480A23F0D9F928F81400BEE7A4F848615B
:10F06000002900F08D81A64A4FF0020EA54BDFED7E
:10F07000A66A19689BF800C00B78887807EE903A6A
:10F08000F8EEE77AB0EE007A67EEA67AF4EEC77A89
:10F09000F1EE10FA40F3448237EEC77ADFED9B6A57
:10F0A000B0EE676AA7EE266AB0EE467A9FED986AE0
:10F0B000D2ED006A66EE866AB0EEE66AC4ED5B6A7F
:10F0C00084ED5E6A98B105EE900AB8EEE55ADFED80
:10F0D0008E5A66EEA64A25EE255AF7EE005A75EED0
:10F0E000C55A64EE864AE5EE245A66EEA56ADFED5F
:10F0F000895A4B7927EE257A27EE267ACBB1DFEDB8
:10F10000826ADFED855A26EE266A06EE903AF8EE20
:10F11000E66A66EE866AF4EEE56AF1EE10FA00F34E
:10F12000BE85F7EE005A75EEE66A85EEA66A27EE12
:10F13000067ABCF10C0F9FED7B8ADFED7B6A00F055
:10F140007685B4EEC87AF1EE10FA98BFB0EE478A31
:10F15000B4EEE68AF1EE10FAB8BFB0EE668A84ED3E
:10F16000418ABEF1000F00F0FD80B0EE007AF4EEAF
:10F17000C77AF1EE10FA05DD37EEC77ADFED636A84
:10F18000E7EE267A92ED017ADFED616A27EE267AC4
:10F19000B0EEC76A84ED5C7A84ED5F6A98B106EEE2
:10F1A000900ADFED595AF8EEE66A27EE075A66EE46
:10F1B000A56AF7EE005A75EEE65A25EE065AE6EE17
:10F1C000855A27EE257ADFED536A8B7967EEA67AAA
:10F1D00067EE877AABB107EE103AB8EEC77ADFED8B
:10F1E0004A5ADFED4D6A27EE067A27EE257AB4EE0D
:10F1F000E67AF1EE10FA40F34485DFED496A67EEF6
:10F20000A67ABCF10C0F00F0F084DFED466A9FEDAA
:10F21000467AF4EEE67AF1EE10FA88BFF0EE667AFE
:10F22000F4EEC77AF1EE10FAB8BFF0EE477ABEF10D
:10F23000010FC4ED427A40F395804B78DFED326ADE
:10F2400007EE903AF8EEE77AB0EE007A67EEA67A2B
:10F250004B7AF4EEC77AF1EE10FA05DD37EEC77A95
:10F26000DFED2A6AE7EE267A92ED027ADFED286A70
:10F2700027EE267AB0EEC76A84ED5D7A84ED606A87
:10F280009BB106EE903ADFED205AF8EEE66A27EEE3
:10F29000075A66EEA56AF7EE005A75EEE65A25EEB5
:10F2A000065AE6EE855A27EE257ADFED1A6ACB7903
:10F2B00067EEA67A67EE877AE3B307EE103AB8EE08
:10F2C000C77ADFED115ADFED146A27EE067A27EED2
:10F2D000257AB4EEE67AF1EE10FA27DCB5EEC07AC4
:10F2E000F1EE10FA01F14481B7EE006A36EE477A8A
:10F2F000C6EE076A1CE000BF205100203449002000
:10F30000E08200204C2000200AD7233CD7A368418C
:10F310006F12033B00004843A4707D3FF48100203E
:10F320000000C84200C0F94400C0F9C45FED046A9F
:10F3300067EEA67ABCF10C0F00F04D845FED076A12
:10F340001FED077AF4EEE67AF1EE10FA88BFF0EEE0
:10F35000667AF4EEC77AF1EE10FAB8BFF0EE477AAB
:10F36000C4ED437ABCF1090F00F0298497F82160BD
:10F37000002E40F0DC830023DAF8008084F8183196
:10F3800018F0200F09D0A84B1B8803F0300323B1DD
:10F39000A64B1B78DA0701F17086A54B1B7823B9C1
:10F3A000A44EB378002B41F038819BF80030072B36
:10F3B00000F05B840022072B84F800217DF4CFACA1
:10F3C00007F076FA0590FDF7CCBC9B4B9B4C1A6876
:10F3D0009B4BDFF8788294F80001D2691B88A8F86B
:10F3E0000020A8F8023000287FF401A80590954D70
:10F3F000FDF7B7BCDFED946AFEF73AB907F058FAAB
:10F40000059A924B801AD880FEF7B9BF07F050FAE0
:10F410009BF800300C9ADFF83482801A012BA8F890
:10F42000020000F09A81072B7DF49EAE07F040FAAF
:10F430000590FDF79BBEDFF850A2D4ED017A94ED64
:10F44000006ABAF80000DAF8143077EEA77AF0EE26
:10F45000006AB0EE677AA6EE267A013804EBC002A5
:10F46000D6EE267A083A1033F6EE003A27EE237AE3
:10F4700067EEA37A84ED207AC4ED217A6F4CA6461C
:10F4800004F1800192ED027A92ED036ADEED036AE7
:10F49000DEED027A53ED014A13ED025A37EE674A68
:10F4A00076EEC65A77EE277AE4EE845A0138A2F156
:10F4B0000802E5EE047A0EF1080E03F1080336EEB9
:10F4C000267A01F10801E4EE877AE5EE475A67EE05
:10F4D000A37A25EEA37AC1ED007A81ED017AD1D12C
:10F4E000142F09D107F0E4F9069BDFF86081C01AF8
:10F4F000A8F80200D4F8B061554B0B93554AD9F8DF
:10F500000030013682FB06129119F217C2EBA102FC
:10F51000C2EBC202B61AC4F8B06103F0005343E56F
:10F52000B0EE677AC2E54C4D4C4E4D4AD5ED004ADF
:10F53000D6ED003A4B4D1278C4ED7B3AC4ED7C4ACF
:10F54000D5ED006A12B1012284F8F821D4ED7D7A5C
:10F55000FEF7B7B8444890ED007AFFF737B8434A52
:10F56000D2ED027AB2EE0E7AF0EEE76AF4EEC76AF6
:10F57000F1EE10FA41D52C4B1B885E073DD53C4B74
:10F580003C49B3F904303C4881FB03610088DB1738
:10F59000C3EBA1031B1A9BB219B211F1B30FBCBF8D
:10F5A00003F5B47319B2B329C4BFA1F5B47319B28A
:10F5B000324B1E481B790078002B4FF6FF7318BFA3
:10F5C000012300077EF525AF2D48006811FB03F3EA
:10F5D000017E2C489BB211FB03F380FB030119440D
:10F5E000DB17C3EB211307EE103AB8EEC77A77EEBC
:10F5F000C77AC2ED027AFEF70CBF1D4B1D4AB3F964
:10F6000004301D4982FB0302DB17C3EBA2030B800E
:10F61000FEF7FFBEAB68002B3EF4F3AE05F14401EC
:10F6200028469847FEF7EDBE44200020721E0020B9
:10F630007C8400207E840020E44800209422002066
:10F64000FA350020FC48002000000000F481002072
:10F6500020510020932449928C7C0020644000209B
:10F6600040580020744000204C3A0020E0820020E6
:10F670005C1E002067666666E4460020387E002037
:10F680004820002089888888485100203B483C4A0F
:10F69000D0F8EC00126844F62066B042A8BF3046AD
:10F6A000B0F57A7FB8BF4FF47A7080B212F0100FC5
:10F6B000A4F81A01D9F8002001F01D84D20400F149
:10F6C0006783304A12680792B2F936C02E4A2F4E2D
:10F6D000D2ED037AD4F81C21A6FB0006B6096420FB
:10F6E00090FBF6F01428BDEEE77A04EB420EA8BFBB
:10F6F0001420013282428DED067AC4F81C21A8BF85
:10F700000022BDF81860A8BFC4F81C2104EB420217
:10F71000AEF82061B2F9202107EE102AB8EEC77AC0
:10F7200077EEC77AFDEEE77ACDED067ABDF91800DF
:10F7300080EAE072A2EBE072624502F3A581144A0E
:10F7400010464FF07E520260FEF777BE07F0B0F829
:10F750000C90FDF794BBDFF8408007F0A9F80D4A44
:10F76000D4F8E43112680590C31A9A1AC4F8E40177
:10F77000A8F80430A8F80620FDF7F8BC60010020C6
:10F78000047E002048200020E0820020D34D62103B
:10F790007800002078440020F4810020B8F1000FA8
:10F7A0003EF467ACF4EEE47AF1EE10FAB8BFF0EE96
:10F7B000667AFDEEE77ABDEEE67A17EE90EA17EE8E
:10F7C00090CAAE4517EE107AA8BFAC467745C8BFC1
:10F7D000BC4607EE90CAF8EEE77A012AC3ED007A3C
:10F7E0003EF4AAAD91ED047ADDED0F7AE7EE257ACD
:10F7F000B0EE637AA3EE277AB4EEE47AF1EE10FA73
:10F80000F0EE477AB8BFF0EE667AFDEEE77A17EED3
:10F8100090EA17EE90CAAE45A8BFAC46BE45B8BF49
:10F82000BC4607EE90CAF8EEE77A022AC3ED017AE9
:10F830003EF482AD91ED087ADDED107AE7EE257A9F
:10F84000B0EE637AA3EE277AB4EEE47AF1EE10FA22
:10F85000F0EE477AB8BFF0EE667AFDEEE77A17EE83
:10F8600090EA17EE90CAAE45A8BFAC46BE45B8BFF9
:10F87000BC4607EE90CAF8EEE77A032AC3ED027A97
:10F880003EF45AAD91ED0C7ADDED117AE7EE257A72
:10F89000B0EE637AA3EE277AB4EEE47AF1EE10FAD2
:10F8A000F0EE477AB8BFF0EE667AFDEEE77A17EE33
:10F8B00090EA17EE90CAAE45A8BFAC46BE45B8BFA9
:10F8C000BC4607EE90CAF8EEE77A042AC3ED037A45
:10F8D0003EF432AD91ED107ADDED127AE7EE257A45
:10F8E000B0EE637AA3EE277AB4EEE47AF1EE10FA82
:10F8F000F0EE477AB8BFF0EE667AFDEEE77A17EEE3
:10F9000090EA17EE90CAAE45A8BFAC46BE45B8BF58
:10F91000BC4607EE90CAF8EEE77A052AC3ED047AF2
:10F920003EF40AAD91ED147ADDED137AE7EE257A17
:10F93000B0EE637AA3EE277AB4EEE47AF1EE10FA31
:10F94000F0EE477AB8BFF0EE667AFDEEE77A17EE92
:10F9500090EA17EE90CAAE45A8BFAC46BE45B8BF08
:10F96000BC4607EE90CAF8EEE77A062AC3ED057AA0
:10F970003EF4E2AC91ED187ADDED147AE7EE257AEB
:10F98000B0EE637AA3EE277AB4EEE47AF1EE10FAE1
:10F99000F0EE477AB8BFF0EE667AFDEEE77A17EE42
:10F9A00090EA17EE90CAAE45A8BFAC46BE45B8BFB8
:10F9B000BC4607EE90CAF8EEE77A072AC3ED067A4E
:10F9C0003EF4BAAC91ED1C7ADDED157AE7EE257ABE
:10F9D000B0EE637AA3EE277AB4EEE47AF1EE10FA91
:10F9E000F0EE477AB8BFF0EE667AFDEEE77A17EEF2
:10F9F00090EA17EE90CAAE45A8BFAC46BE45B8BF68
:10FA0000BC4607EE90CAF8EEE77A082AC3ED077AFB
:10FA10003EF492AC91ED207ADDED167AE7EE257A90
:10FA2000B0EE637AA3EE277AB4EEE47AF1EE10FA40
:10FA3000F0EE477AB8BFF0EE667AFDEEE77A17EEA1
:10FA400090EA17EE90CAAE45A8BFAC46BE45B8BF17
:10FA5000BC4607EE90CAF8EEE77A092AC3ED087AA9
:10FA60003EF46AAC91ED247ADDED177AE7EE257A63
:10FA7000B0EE637AA3EE277AB4EEE47AF1EE10FAF0
:10FA8000F0EE477AB8BFF0EE667AFDEEE77A17EE51
:10FA900090EA17EE90CAAE45A8BFAC46BE45B8BFC7
:10FAA000BC4607EE90CAF8EEE77A0A2AC3ED097A57
:10FAB0003EF442AC91ED287ADDED187AE7EE257A36
:10FAC000B0EE637AA3EE277AB4EEE47AF1EE10FAA0
:10FAD000F0EE477AB8BFF0EE667AFDEEE77A17EE01
:10FAE00090EA17EE90CAAE45A8BFAC46BE45B8BF77
:10FAF000BC4607EE90CAF8EEE77A0B2AC3ED0A7A05
:10FB00003EF41AAC91ED2C7ADDED197AE7EE257A08
:10FB1000E3EE273AF4EEE34AF1EE10FAD4BFF0EE4A
:10FB2000637AF0EE667AFDEEE77AFEF7F7BB1E2108
:10FB3000D04805F0B7FE00283FF41DACCE4B1B8823
:10FB400059063FF518AC94F88431B34241F0D3879D
:10FB5000CA4BD4ED627A93ED017A94ED435ADFED0E
:10FB6000C85A9FEDC86A67EEC56A67EE887AE7EE05
:10FB7000086AE5EE077AF4EEE56AF1EE10FA8CBF5A
:10FB8000B0EE657AB0EE667AB4EEC67AF1EE10FAAF
:10FB9000F4EEE57AB8BFB0EE467AF1EE10FA88BF1F
:10FBA000F0EE657AF4EEC67AF1EE10FAB8BFF0EE38
:10FBB000467A84ED417AC4ED437AFFF7DCBBFDEE73
:10FBC000C87ADFF8E08217EE903AA8F80460A8F847
:10FBD0000630FFF7CBBBBDEEE77ADFF8C88217EE41
:10FBE000103AA8F80430FFF7A9BB9FEDA57ADFED26
:10FBF000A56ADFF8B082F4EEC77AF1EE10FA98BF8A
:10FC0000B0EE677AFDEEE77AB4EEE67AF1EE10FA3E
:10FC100017EE903AB8BFB0EE667ABEF1010F84EDF0
:10FC2000427AA8F802303FF708ABFFF79FBBB4EE6B
:10FC3000C87AF1EE10FA98BFB0EE478ABDEEC77AE7
:10FC4000B4EEE68ADFF85C82F1EE10FA17EE103AB5
:10FC5000B8BFB0EE668A84ED418AA8F80030BEF1E4
:10FC6000000F7FF482AAFFF781BB06F021FE059A00
:10FC7000DFF830829BF80030801AA8F80400FFF704
:10FC800099BBB5EEC07AF1EE10FA00F17584B7EECB
:10FC9000006A36EE477AC6EE076AFFF7B0BA9FED04
:10FCA0007A6AFFF744BAFDEEE47A0EA817EE90EAFE
:10FCB000FDEEE67A00EB820306934FFA88F188F0B6
:10FCC0000103DFF8E491DFF8E4C1089417EE907ABD
:10FCD000B1EE433A07921C468A464B4693ED007AB2
:10FCE000F0EC017AE7EE257A08F0010309F110093A
:10FCF000B0EE637AA3EE277AF4EEC74AF1EE10FA7B
:10FD0000D8BF0023002BF0EE477A18BFB0EE667A1A
:10FD1000BDEEC77AFDEEE77A17EE102A17EE901ABD
:10FD2000AA4217EE103AA8BF2B469742CCBF00223A
:10FD300008F00102002A08BF3B46A94217EE902AAC
:10FD400007EE103AA8BF2A468E45CCBF002304F028
:10FD50000103002B08BF724607EE902AB8EEC77A5F
:10FD6000F8EEE77A069BBAF1000F18BFF0EE477A7B
:10FD70009842ECEC017AB0D1FEF7BBBC97F820209A
:10FD8000C2EB421002EB8002D20092B2FEF761BBDE
:10FD90003E4A12680792B2F836C04FEA5C0C95E40E
:10FDA0003B4BD4F8B4810B93B4F8ACA1CAF1200357
:10FDB000D8B2384B0AEB481E03EB8E0E830801F0D5
:10FDC000388701331B013449344A07930EEB030C87
:10FDD0000EF1100313ED024A13ED035A13ED016AFD
:10FDE00013ED047A51ED024A51ED035A51ED016AC7
:10FDF00051ED047A64EE244A65EE255A66EE266AD1
:10FE000067EE277A1033634542ED024A42ED035A0A
:10FE100042ED016A42ED047A01F1100102F1100293
:10FE2000D8D1079B1E49A3F11002964401EB020CA6
:10FE3000224410F0030309D0BEEC017AFCEC017AF5
:10FE400067EE277A013BE2EC017AF5D1BAF1000FB7
:10FE500041F0D284142F7FF451AB06F029FD069BAC
:10FE6000DFF84080D4F8B061C01AA8F80200FFF7AC
:10FE700045BB00BF047E0020442000207800002005
:10FE800000C0F94400C0F9C40000C8424820002066
:10FE90002051002060510020F0520020A4220020B8
:10FEA000E0520020F4810020A03F002044440020C4
:10FEB000D4F8B4A1C44AC54B0B9203EBCA03126831
:10FEC00007929DED077A9B88DFEDC17AC14AF8EE73
:10FED000478A09EE103A643BC82BA8BFC82368EED6
:10FEE000A78AF8EE497A782BB8BF782368EEA78AFC
:10FEF00007EE903A4FF02C08B0EE680A08FB0A288B
:10FF0000B8EEE78A22F0CCFAB8EEC99AF0EE409A41
:10FF1000B0EE680A22F026FA38EE097A79EE487ACD
:10FF200028EE098A67EE877AB7EE006A88EE277AAC
:10FF3000142FF8EE007A77EE076A60EE277A89EEE2
:10FF4000A67A77EE065A36EE477AC6EE256A67EE4F
:10FF5000A67A27EE267AC8ED006A88ED047AC8ED05
:10FF6000026AC8ED017AC8ED037A01F099869A4BCE
:10FF70009BF800700AF1010A83FB0A38A8EBEA78C3
:10FF800008EB48080136AAEB0808C4F8B061C4F8C9
:10FF9000B48109E7DFF85CA29048DAF80820BAF8E3
:10FFA0000C1021F0E7FA9BF80070142F01F06C861A
:10FFB000D4F8B0610136C4F8B061FFF73EBA884B9F
:10FFC0001A78D4F8B4E181489FED867A4FEACE0CD6
:10FFD00000EB0C0383ED007A002A7CD07F49B0EE61
:10FFE000476AF0EE476A0023F1EC017A013367EECD
:10FFF000A77A05EE903AB4EEE77AF1EE10FAF8EE51
:020000040801F1
:10000000E55AB8BFB0EE677A934276EEA76AA7EEDC
:10001000A56AE9D1F5EEC06A00EB0C03F1EE10FA27
:1000200083ED007A57DDC6EE265A6F4B6F4A128871
:10003000F7EE007A75EEE75AD3ED007A65EEA77A0F
:10004000FDEEE77A17EE903A812B41F394809342CC
:10005000A8BF134607EE903AF8EEE77A644B2C21DE
:1000600001FB0E3393ED097AD3ED003A93ED0A6A62
:1000700093ED014AD3ED046AD3ED034A93ED025A9E
:10008000A3EEA77AA4EE276A66EEC76AA7EE646AB3
:10009000BDEEC77AE5EE276A17EE101A812983EDC7
:1000A000096AC3ED0A6A41F363808A42A8BF0A461F
:1000B00007EE902AF8EEE77AFCEEE77ACDED077AC4
:1000C000BDF81C3000EB0C029380BEF1000F02D192
:1000D000132F01F0F884152F7FF402AA6044DFF893
:1000E0001881838828F81E30374BD4F8B0610B9301
:1000F000FFF704BADFF8E8A09AF800205FEA920858
:1001000001F06286DFF8F4C008F1010040010CEB59
:10011000000E0CF12003ACF1700113ED076A53EDF2
:10012000056A13ED037A53ED017A53ED025A13ED8C
:10013000084A53ED064A13ED045A26EE066A66EEA7
:10014000A66A27EE077A67EEA77AA4EE046A203340
:100150007345E4EEA46A01F11001A5EE057AE5EE1F
:10016000A57AF1EEC65AB1EEE66AF1EEC76AB1EED3
:10017000E77A41ED085A01ED076A41ED066A01EDA3
:10018000057ACAD12038844404EB081112F0030325
:1001900018BF0CF1080C0FD05CED017A1CED027A4F
:1001A00067EEA77A013BE7EE077A0CF1080CB1EE97
:1001B000E77AA1EC017AEFD1142F01F07F850136A7
:1001C000C4F8B061FDE600BF20510020605300205C
:1001D00027D4D2369C5000205655555594220020E5
:1001E00042510020000000004451002040510020F6
:1001F0007853002048510020F4810020142300206F
:10020000DFF8CCA3BAF80070DAF804E04FEA570C34
:100210004FEA8C0204EB8708FF0804EB020300F0AE
:100220009F8010320137E34803EB07174244103335
:100230000EF1100608F1100151ED032A51ED043AB8
:1002400010ED043A10ED032A51ED026A11ED016A36
:1002500010ED020A10ED018A12ED044A12ED035A64
:1002600053ED044A53ED035A13ED027A53ED017A2C
:1002700052ED020A12ED011A73EE238A72EE221A6F
:1002800040ED048A40ED031A70EE268A78EE061AD5
:1002900040ED028A40ED011A74EE848A75EE851AEB
:1002A00043ED048A43ED031A77EE208A77EE811A34
:1002B00043ED028A43ED011A73EE633A75EE655A17
:1002C00016ED035A32EE623A74EE644A65EE631A32
:1002D00016ED044A23EE052A64EE652AE3EE041ABD
:1002E0001033BB4224EE843AA3EE842A00F11000BE
:1002F00006F11006A5EE853A01F1100102F1100297
:10030000E4EE852A41ED071A01ED082A02ED073ACD
:1003100042ED082A56ED055A16ED065A70EE666A49
:1003200038EE466A30EEC77A71EE677A26EE253AE5
:1003300065EEE63A25EE674A67EE054AE6EE053ACF
:10034000A6EE853AA7EE254AE7EEA54A01ED063A64
:1003500041ED053A02ED064A42ED054A7FF46CAFE5
:100360001FFA8CF67246314693481BF09DFD3146CC
:10037000DAF8042040461BF097FD9BF80030142B60
:100380007FF4B8A8FFF7AEB806F092FA9BF80070B9
:100390000690142F05BFDFF83C82D4F8B061D4F882
:1003A000B061A8F80060FCF736BD844FDFF828A2E2
:1003B00097ED004A97ED097AD7ED014A97ED0A6A61
:1003C000D7ED046A97ED035AD7ED025A69EE277A02
:1003D0000AEB8603A4EE277AA7EEA46A66EEC76A44
:1003E000A7EE456AE7EEA56A27EE000A87ED096ADF
:1003F000C7ED0A6A83ED007A29EE088A22F004F834
:1004000069EE288AD7ED145AD7ED1F6A97ED0B1ABB
:10041000D7ED161A97ED155A97ED207A97ED0C2A1D
:10042000D7ED172A97ED0F6AD7ED1A7A97ED0E3AA6
:10043000D7ED0D3A97ED194AD7ED184AE1EE085A73
:1004400000220AEB8603E8EEA16A00B2C4F89C2100
:10045000A8EE025AC4F8A021C4F8A421A8EEA27AFA
:1004600026EE656A67EEE67AA5EEC35AA3EE886AC1
:10047000A6EEC47AE8EEA47A87ED145AC3ED205AAA
:1004800087ED156AC3ED406A87ED1F7AC7ED207AC4
:10049000FEF77CBBB5F92430EA6207EE903A012200
:1004A000F8EEE77A2B66EA670023012FC5ED1C7A88
:1004B000C5ED1B7A6B6701F0FD82B7427CF436AF65
:1004C000B5F926306B6607EE903A00220123F8EE6C
:1004D000E77A2A63C5F890300023012FC5ED217A11
:1004E000C5ED207AC5F8883001F0E082B7427CF48F
:1004F0004DAFB5F92830AB6607EE903A00220123E4
:10050000F8EEE77A6A63C5F8A4300023012FC5ED41
:10051000267AC5ED257AC5F89C307CF467AF9FED4F
:10052000288AB9F1030F2BD0BAF1000F09D007EEDA
:1005300090AAF8EEE77AF4EEC87AF1EE10FA01F13B
:100540003D84204AAB6E1268A8F80600002103EB38
:10055000560393FBF6F66E6391621163D162FCF76A
:1005600047BF194B9B7B002B3EF462A8FDF757BF9A
:10057000F7EE006AFEF7DCBEF7EE006AFEF73FBE5C
:10058000B0EE480A21F040FF00B2CDE7B4F8486170
:10059000013E36B2002EA4F848617EF761AD0B4AE9
:1005A000FDF7A8BFB4F81A2102F57A7292B2FDF7EE
:1005B00050BF00BFA422002094220020FC53002042
:1005C00000000000E448002044570020E0820020A2
:1005D00048510020F481002060510020CD49DFED1A
:1005E000CE7A0968C4ED707A11F0805100F0A184D0
:1005F000B7EE007A77EE677AF4EEE57AF1EE10FA6C
:1006000088BFF0EE657AF0EE675AC4ED7D7AFDF7AB
:1006100051BB00F00100FDF78FBEC04F3A78013AA0
:100620000A2A1CD8DFE812F00A01E601B701960198
:100630005D0140012B011801E600D1000B00B84A12
:10064000B84952680968C8328A4203D31BF002F8DD
:1006500028B1B378032B01F07A8401233B70F3783F
:10066000002B3EF4A2AED9F80030D80441F19A83B1
:10067000AD4B9B8807EE903AF8EEE77AAB4A92EDE5
:10068000012AD2ED022A92ED033AD2ED043A92ED1C
:10069000054AD2ED064A92ED075AD2ED085A92ED7C
:1006A000096AD2ED0A6A92ED0B7AB4EE672AF1EE8E
:1006B00010FAF4EE672A14BF01230023F1EE10FABA
:1006C000B4EE673A18BF43F00103F1EE10FAF4EE0E
:1006D000673A18BF43F00103F1EE10FAB4EE674A2F
:1006E00018BF43F00103F1EE10FAF4EE674A18BFA9
:1006F00043F00103F1EE10FAB4EE675A18BF43F06D
:100700000103F1EE10FAF4EE675A18BF43F001034B
:10071000F1EE10FAB4EE676A18BF43F00103F1EE90
:1007200010FAF4EE676A18BF43F00103F1EE10FA15
:10073000B4EE677A18BF43F00103F1EE10FA18BF68
:1007400043F00103002B41F0C98292ED007AB4EE30
:10075000677AF1EE10FA41F0C182DFF8C881D4F86F
:100760009821D8F800309A4201F2BF823B78012BE1
:100770003EF41BAE94F89421002A3EF416AE0B2BE7
:1007800018D801229A4040F6030112EA010617D157
:1007900012F4C06F0ED0093B012B0BD845201AF084
:1007A0007DFFFF201AF07AFF61481AF063FF3046A0
:1007B0001AF074FF5A4BD8F800205A600B233B7094
:1007C000002384F89431FEF7F0BD5A4B1B78002BC0
:1007D00001F09F821A2015F059FF002841F09982FC
:1007E00094F89431002B41F0948209233B701CF063
:1007F000FFFA34E71A2015F049FF0028F7D04E4BD6
:100800001B88002BF3D14D4B4520D3F800801AF004
:1008100045FF0E201AF042FF40461BF0B9FFDDF8FD
:10082000248040461BF0B4FF454A4FF480510A2310
:10083000404611803B701BF0BDFFD8E7414803786C
:10084000DB077FF50CAF802018F012FF08B109F02C
:1008500081F911F043FA02E71AF0DAFE1CF0E2FA2D
:1008600000283FF4FCAE1AF0F5FE00283FF4F7AE86
:10087000334A4FF480510A2311803B70EFE61AF09F
:10088000C7FE314B002105208DE80300A3F10802CB
:10089000029153201CF078FF00287FF4E0AE204A3C
:1008A000082310603B70DAE61AF0B2FE274A029283
:1008B000A2F10C034FF007080193CDF80080A2F1DC
:1008C00008030021143A47201CF05EFF00287FF443
:1008D000C6AE134B87F800804FF0FF3283E8050067
:1008E000BDE61AF095FE1A4B002102208DE80300A8
:1008F000A3F10802029148201CF046FF00287FF473
:10090000AEAE074B4FF0FF310622186059603A70C7
:10091000A5E600BF047E0020000000807D8400204A
:10092000287E0020E075002068400020703F0020F5
:10093000D8700308CC440020707C0020807C00200C
:10094000227E0020B4550020AC4C0308644C030800
:10095000484C03081AF05CFE774A0292A2F10C039D
:10096000282101930091A2F10A035021163A49204F
:100970001CF00AFF00287FF472AED9F8003013F0A3
:10098000800301F0C2826D4B4FF0FF3105221860E9
:1009900059603A7063E6DFF8A4811AF039FE684ABC
:1009A000D8F80430126864339342BFF458AE402044
:1009B0001AF012FE00287FF452AED8F800306149D8
:1009C0004FF0400A0FE006911AF068FE0699D8F839
:1009D00000300A680133013ABAF1010A0A60C8F826
:1009E000003001F09B82584AD35C1846002BEAD1B4
:1009F00001F099BA524B514A1B6853605149002388
:100A0000136003220B603A7029E6504BDFED507AF9
:100A100093ED080AB4EEE70AF1EE10FA40F24287CD
:100A200021F088FDD4ED457A20EE270A21F0ECFC78
:100A3000B0F5617F00F33A8707EE900AF8EEE76AB7
:100A4000DFED447A66EEA76A07EE906AB8EEE77AC1
:100A5000FDEEE67A17EE903A2033402B41F25E81AC
:100A60009FED3D0A21F0D0FC00B207EE900AB8EEEF
:100A7000E77A3A4AD2ED037A77EE877AC2ED037AC3
:100A8000FDF7D5BC0698002800F02E87FDEEE47A2D
:100A90000EA901EB820217EE90EAFDEEE67A91468E
:100AA0002346424664462E482E4F17EE90AAB1EEDA
:100AB000433A9C46C84613E0FDEEC77A17EE903ADB
:100AC000734503DBAB42A8BF2B46994607EE909ACD
:100AD000F8EEE77A4145E7EC017A00F1100027D003
:100AE00090ED007AF1EC017AE7EE257AF146B0EE6E
:100AF000637AA3EE277AF0EE477A002ADCD05346D9
:100B000034B1B4EE647AF1EE10FA48BFF0EE667AD2
:100B1000FDEEE77A17EE909AD14504DBA94517EE72
:100B2000903AA8BF2B4607EE903AF8EEE77AD1E765
:100B30006446FDF704BC00BF764A0308287E002007
:100B4000E0750020D0730020004A03081037002011
:100B50008FC2753CD06D393A00000000E082002061
:100B6000A03F002044440020BDEEE67A17EE107A44
:100B7000B0EE647AA3EE277AF0EE477ABCF1000F6C
:100B800040F01C83FDEEC77A17EE90CA17EE90EA8C
:100B9000AC45A8BFAE466745C8BFBE4607EE90EA63
:100BA000F8EEE77A012AC3ED007A3DF4C5AB91ED8A
:100BB000047ADDED0F7AE7EE257AB0EE647AA3EEE3
:100BC000277AFDEEC77A17EE90CA17EE90EAAC4589
:100BD000A8BFAE46BC45B8BFBE4607EE90EAF8EEE9
:100BE000E77A022AC3ED017A3DF4A6AB91ED087ACB
:100BF000DDED107AE7EE257AB0EE647AA3EE277A7F
:100C0000FDEEC77A17EE90CA17EE90EAAC45A8BF82
:100C1000AE46BC45B8BFBE4607EE90EAF8EEE77AAE
:100C2000032AC3ED027A3DF487AB91ED0C7ADDED3A
:100C3000117AE7EE257AB0EE647AA3EE277AFDEE1C
:100C4000C77A17EE90CA17EE90EAAC45A8BFAE4639
:100C5000BC45B8BFBE4607EE90EAF8EEE77A042A34
:100C6000C3ED037A3DF468AB91ED107ADDED127AB5
:100C7000E7EE257AB0EE647AA3EE277AFDEEC77A26
:100C800017EE90CA17EE90EAAC45A8BFAE46BC4539
:100C9000B8BFBE4607EE90EAF8EEE77A052AC3ED44
:100CA000047A3DF449AB91ED147ADDED137AE7EE69
:100CB000257AB0EE647AA3EE277AFDEEC77A17EEB6
:100CC00090CA17EE90EAAC45A8BFAE46BC45B8BF87
:100CD000BE4607EE90EAF8EEE77A062AC3ED057AFB
:100CE0003DF42AAB91ED187ADDED147AE7EE257A22
:100CF000B0EE647AA3EE277AFDEEC77A17EE90CABB
:100D000017EE90EAAC45A8BFAE46BC45B8BFBE469C
:100D100007EE90EAF8EEE77A072AC3ED067A3DF48B
:100D20000BAB91ED1C7ADDED157AE7EE257AB0EE8E
:100D3000647AA3EE277AFDEEC77A17EE90CA17EE13
:100D400090EAAC45A8BFAE46BC45B8BFBE4607EE6C
:100D500090EAF8EEE77A082AC3ED077A3DF4ECAAA8
:100D600091ED207ADDED167AE7EE257AB0EE647A21
:100D7000A3EE277AFDEEC77A17EE90CA17EE90EA37
:100D8000AC45A8BFAE46BC45B8BFBE4607EE90EA2C
:100D9000F8EEE77A092AC3ED087A3DF4CDAA91ED81
:100DA000247ADDED177AE7EE257AB0EE647AA3EEC9
:100DB000277AFDEEC77A17EE90CA17EE90EAAC4597
:100DC000A8BFAE46BC45B8BFBE4607EE90EAF8EEF7
:100DD000E77A0A2AC3ED097A3DF4AEAA91ED287AA2
:100DE000DDED187AE7EE257AB0EE647AA3EE277A85
:100DF000FDEEC77A17EE90CA17EE90EAAC45A8BF91
:100E0000AE46BC45B8BFBE4607EE90EAF8EEE77ABC
:100E10000B2AC3ED0A7A3DF48FAA91ED2C7ADDED11
:100E2000197AE7EE257AE3EE274AFDEEE47AFDF73C
:100E300075BA0698002800F0B285FDEEE67A0EA994
:100E400001EB820217EE90AAFDEEE47A914623466A
:100E500042466446CA48CB4F17EE90EA9C46C846C5
:100E600014E0FDEEC77A17EE909ACE4503DCA94553
:100E70004B46A8BF2B4607EE903AF8EEE77A41457D
:100E8000E7EC017A00F110003FF452AE90ED007AE9
:100E9000F1EC017AE7EE257A7346B0EE647AA7EEBC
:100EA000837AF0EE477A002ADBD034B1F4EE474A79
:100EB000F1EE10FAC8BFF0EE667AFDEEE77A53461F
:100EC00017EE909ACA45D2DDD5E705F0F1FC059002
:100ED000FDF78FBAAC49096811F0805129D0B6EE00
:100EE000007A67EE877AF4EEE75AF1EE10FA3FF5F2
:100EF0008AABFFF77DBBD6003EF5E0ABFDF79DBAB0
:100F0000A24DA34EA34AD5ED004AD6ED003AA24D1C
:100F10001278C4ED7D7AC4ED7B3AC4ED7C4AD5ED00
:100F2000006A002A3CF4CDAB012284F8F821FCF7DA
:100F3000C8BB13F4800101D00021D0E7B6EE007ADF
:100F4000F4EEC75AF1EE10FAC9DCFCF7B3BEFDEEC1
:100F5000E67A28460EAB8A49DFF828E217EE907A47
:100F6000654603EB82088446D1ED007AB3EC017A42
:100F7000A7EEA57A1031B0EE646AA3EE076A07EE19
:100F8000907AB0EE467A35B1F4EE464AF1EE10FAB8
:100F9000C8BFB0EE667ABDEEC77A17EE100A874278
:100FA00004DC6045A8BF604607EE900AF8EEE77AD9
:100FB0009845EEEC017AD7D1FDF71AB8012A40F333
:100FC000798507EE101AB8EEC77AC7EE876AB1EED8
:100FD000E68AB9F1030F14D0BAF1000F09D007EE79
:100FE00090AAF8EEE77AB4EEE78AF1EE10FA00F391
:100FF000E5862B6E03EB560393FBF6F3EB62FFF7EC
:101000005CBAB0EE480A21F0FFF900B2E4E7012A29
:101010007FF785AA07EE101AB8EEC77AC7EE876A7F
:10102000B1EEE68AFFF77DBA012A40F33F8507EE6D
:10103000101AB8EEC77AC7EE876AB1EEE68AB9F140
:10104000030F14D0BAF1000F09D007EE90AAF8EE02
:10105000E77AB4EEE78AF1EE10FA00F3AF866B6E32
:1010600003EB560393FBF6F32B63FFF73FBAB0EEA7
:10107000480A21F0C9F900B2E4E7484B484AB3F9FD
:101080000430DFED487A82FB0312DB17C3EBA203C7
:101090001BB208EE103AB8EEC88A28EE278AB0EEE6
:1010A000480A04F027FBF0EE408AB0EE480A04F04C
:1010B000A7FA3D4BD878002800F0C9843B4AB4F920
:1010C0008E11B2F9023044F250665B1AB34200F35B
:1010D000F584374EB342BCBF03F50C43A033464200
:1010E0009E4200F305858342A8BF0346B2F9002063
:1010F000B4F98C710B4419B2D31B44F25062934281
:10110000A4F88E1100F3EF84294A9342BCBF03F583
:101110000C43A0339E4203DC9842A8BF1846064603
:10112000BB191BB207EE903A07EE101AF8EEE77AF9
:10113000F8EEC76A27EEE87A60EE277AA0EE267A04
:10114000A4F88C31E8EEA67ADFED1A6A27EE267A4B
:1011500067EEA67ABDEEC77AFDEEE77A17EE102AA3
:1011600017EE903AA4F89021A4F89231FEF715B941
:101170008223FEF7A7BFDFED107AFEF76FBF00BF37
:10118000A03F002044440020047E00208C7C0020EE
:101190006440002040580020744000205C1E002065
:1011A0006766666635FA8E3C68460020C4460020B5
:1011B000B0B9FFFFCDCCCC3D00000243B4EEE47AE1
:1011C000F1EE10FAB8BFF0EE667AFDEEE77A17EEB0
:1011D00090EA17EE90CAAE45A8BFAC467745C8BFA7
:1011E000BC4607EE90CAF8EEE77A012AC3ED007A12
:1011F0003DF4A2A891ED047ADDED0F7AE7EE257AB1
:10120000B0EE647AA3EE277AB4EEE47AF1EE10FA47
:10121000F0EE477AB8BFF0EE667AFDEEE77A17EEA9
:1012200090EA17EE90CAAE45A8BFAC46BE45B8BF1F
:10123000BC4607EE90CAF8EEE77A022AC3ED017ABF
:101240003DF47AA891ED087ADDED107AE7EE257A83
:10125000B0EE647AA3EE277AB4EEE47AF1EE10FAF7
:10126000F0EE477AB8BFF0EE667AFDEEE77A17EE59
:1012700090EA17EE90CAAE45A8BFAC46BE45B8BFCF
:10128000BC4607EE90CAF8EEE77A032AC3ED027A6D
:101290003DF452A891ED0C7ADDED117AE7EE257A56
:1012A000B0EE647AA3EE277AB4EEE47AF1EE10FAA7
:1012B000F0EE477AB8BFF0EE667AFDEEE77A17EE09
:1012C00090EA17EE90CAAE45A8BFAC46BE45B8BF7F
:1012D000BC4607EE90CAF8EEE77A042AC3ED037A1B
:1012E0003DF42AA891ED107ADDED127AE7EE257A29
:1012F000B0EE647AA3EE277AB4EEE47AF1EE10FA57
:10130000F0EE477AB8BFF0EE667AFDEEE77A17EEB8
:1013100090EA17EE90CAAE45A8BFAC46BE45B8BF2E
:10132000BC4607EE90CAF8EEE77A052AC3ED047AC8
:101330003DF402A891ED147ADDED137AE7EE257AFB
:10134000B0EE647AA3EE277AB4EEE47AF1EE10FA06
:10135000F0EE477AB8BFF0EE667AFDEEE77A17EE68
:1013600090EA17EE90CAAE45A8BFAC46BE45B8BFDE
:10137000BC4607EE90CAF8EEE77A062AC3ED057A76
:101380003CF4DAAF91ED187ADDED147AE7EE257AC8
:10139000B0EE647AA3EE277AB4EEE47AF1EE10FAB6
:1013A000F0EE477AB8BFF0EE667AFDEEE77A17EE18
:1013B00090EA17EE90CAAE45A8BFAC46BE45B8BF8E
:1013C000BC4607EE90CAF8EEE77A072AC3ED067A24
:1013D0003CF4B2AF91ED1C7ADDED157AE7EE257A9B
:1013E000B0EE647AA3EE277AB4EEE47AF1EE10FA66
:1013F000F0EE477AB8BFF0EE667AFDEEE77A17EEC8
:1014000090EA17EE90CAAE45A8BFAC46BE45B8BF3D
:10141000BC4607EE90CAF8EEE77A082AC3ED077AD1
:101420003CF48AAF91ED207ADDED167AE7EE257A6D
:10143000B0EE647AA3EE277AB4EEE47AF1EE10FA15
:10144000F0EE477AB8BFF0EE667AFDEEE77A17EE77
:1014500090EA17EE90CAAE45A8BFAC46BE45B8BFED
:10146000BC4607EE90CAF8EEE77A092AC3ED087A7F
:101470003CF462AF91ED247ADDED177AE7EE257A40
:10148000B0EE647AA3EE277AB4EEE47AF1EE10FAC5
:10149000F0EE477AB8BFF0EE667AFDEEE77A17EE27
:1014A00090EA17EE90CAAE45A8BFAC46BE45B8BF9D
:1014B000BC4607EE90CAF8EEE77A0A2AC3ED097A2D
:1014C0003CF43AAF91ED287ADDED187AE7EE257A13
:1014D000B0EE647AA3EE277AB4EEE47AF1EE10FA75
:1014E000F0EE477AB8BFF0EE667AFDEEE77A17EED7
:1014F00090EA17EE90CAAE45A8BFAC46BE45B8BF4D
:10150000BC4607EE90CAF8EEE77A0B2AC3ED0A7ADA
:101510003CF412AF91ED2C7ADDED197AE7EE257AE5
:10152000B0EE647AA7EE837AF4EEC74AF0EE477A1B
:10153000F1EE10FAC8BFF0EE667AFDEEE77AFCF73E
:10154000EDBEFDEEE77ABDEEE67A17EE90CA17EE35
:1015500090EAAC4517EE107AA8BFAE466745C8BF03
:10156000BE4607EE90EAF8EEE77A012AC3ED007A6C
:101570003CF4E2AE91ED047ADDED0F7AE7EE257AE8
:10158000B0EE637AA3EE277AFDEEC77A17EE90CA23
:1015900017EE90EAAC45A8BFAE46BC45B8BFBE4604
:1015A00007EE90EAF8EEE77A022AC3ED017A3CF4FE
:1015B000C3AE91ED087ADDED107AE7EE257AB0EE54
:1015C000637AA3EE277AFDEEC77A17EE90CA17EE7C
:1015D00090EAAC45A8BFAE46BC45B8BFBE4607EED4
:1015E00090EAF8EEE77A032AC3ED027A3CF4A4AE5F
:1015F00091ED0C7ADDED117AE7EE257AB0EE637AA3
:10160000A3EE277AFDEEC77A17EE90CA17EE90EA9E
:10161000AC45A8BFAE46BC45B8BFBE4607EE90EA93
:10162000F8EEE77A042AC3ED037A3CF485AE91ED37
:10163000107ADDED127AE7EE257AB0EE637AA3EE4A
:10164000277AFDEEC77A17EE90CA17EE90EAAC45FE
:10165000A8BFAE46BC45B8BFBE4607EE90EAF8EE5E
:10166000E77A052AC3ED047A3CF466AE91ED147A6C
:10167000DDED137AE7EE257AB0EE637AA3EE277AF2
:10168000FDEEC77A17EE90CA17EE90EAAC45A8BFF8
:10169000AE46BC45B8BFBE4607EE90EAF8EEE77A24
:1016A000062AC3ED057A3CF447AE91ED187ADDEDDC
:1016B000147AE7EE257AB0EE637AA3EE277AFDEE90
:1016C000C77A17EE90CA17EE90EAAC45A8BFAE46AF
:1016D000BC45B8BFBE4607EE90EAF8EEE77A072AA7
:1016E000C3ED067A3CF428AE91ED1C7ADDED157A57
:1016F000E7EE257AB0EE637AA3EE277AFDEEC77A9D
:1017000017EE90CA17EE90EAAC45A8BFAE46BC45AE
:10171000B8BFBE4607EE90EAF8EEE77A082AC3EDB6
:10172000077A3CF409AE91ED207ADDED167AE7EE0A
:10173000257AB0EE637AA3EE277AFDEEC77A17EE2C
:1017400090CA17EE90EAAC45A8BFAE46BC45B8BFFC
:10175000BE4607EE90EAF8EEE77A092AC3ED087A6A
:101760003CF4EAAD91ED247ADDED177AE7EE257AC7
:10177000B0EE637AA3EE277AFDEEC77A17EE90CA31
:1017800017EE90EAAC45A8BFAE46BC45B8BFBE4612
:1017900007EE90EAF8EEE77A0A2AC3ED097A3CF4FC
:1017A000CBAD91ED287ADDED187AE7EE257AB0EE33
:1017B000637AA3EE277AFDEEC77A17EE90CA17EE8A
:1017C00090EAAC45A8BFAE46BC45B8BFBE4607EEE2
:1017D00090EAF8EEE77A0B2AC3ED0A7A3CF4ACAD56
:1017E00091ED2C7ADDED197AE7EE257AE3EE273AD2
:1017F000FDEEE37AFCF792BD830001EB030C04EBF2
:10180000030EE04B03EBC8185FEA9A0300F0F9827D
:1018100001331B01079308EB03000CF1100108F1E1
:1018200010030EF1100213ED024A13ED035A13EDEB
:10183000016A13ED047A51ED024A51ED035A51ED5C
:10184000016A51ED047A64EE244A65EE255A66EE8B
:10185000266A67EE277A1033834242ED024A42ED50
:10186000035A42ED016A42ED047A01F1100102F1DE
:101870001002D8D1079B103B08EB03020CEB0301CD
:1018800073441AF0030A3EF4E5AAB2EC017AF1ECD3
:10189000017A67EE277ABAF1010AE3EC017AF4D112
:1018A000FEF7D8BA9FEDB87AFFF7E3B807EE906A73
:1018B000DFEDB66AB8EEE77A66EEA65A9FEDC55A36
:1018C0009FEDC56ADFEDC57AA5EE856A26EEA55ABD
:1018D000E5EE867AE5EE276A26EE870AFFF7C2B8BC
:1018E000F0EE627AFCF770B9FDEEE67A0EA8CDED67
:1018F000087AFDEEE47A0B94A54FDFF8C8A2CDF884
:101900002490444617EE90EADDF820800A93B1EE69
:10191000433A00EB8202CDF818C097ED007AF0EC64
:10192000017AE7EE257AB0EE637AA3EE277AF0EE3D
:10193000477ADCB9FDEEC77AF44617EE909ACE45A9
:1019400004DCA94517EE90CAA8BFAC4607EE90CAC2
:10195000F8EEE77A002900F03C829042EAEC017A46
:1019600007F11007D9D10B9CFCF7E9BC069B33B1FA
:10197000F4EE474AF1EE10FAC8BFF0EE667AFDEEDB
:10198000E77A17EE90CAE04507EE908A04DCAC4592
:10199000A8BFAC4607EE90CAF8EEE77ADAE7FDEEAC
:1019A000E47A0EA817EE90EAFDEEE67A0B94784FF3
:1019B000DFF810A2CDED087A444600EB8202CDF8A4
:1019C00024900A93CDF818C017EE908A05E0824261
:1019D000EAEC017A07F11007C5D097ED007AF0EC38
:1019E000017AE7EE257AB0EE647AA3EE277AF0EE7C
:1019F000477ADCB9FDEEC77AF44617EE909ACE45E9
:101A000003DCA945CC46A8BFAC4607EE90CAF8EE69
:101A1000E77A0029DBD10A9B002BD8D1099B9C4691
:101A2000079B9C45B8BFF0EE667AD0E7069B33B1C2
:101A3000F4EE474AF1EE10FAC8BFF0EE667AFDEE1A
:101A4000E77AC44617EE909AC845DEDCD9E7514BD9
:101A50009FED516AB3F90020B3F9023007EE902AE6
:101A600006EE903AF8EEE77AF8EEE66A27EEE87AC4
:101A700060EE277AA0EE267AE8EEA67A27EE067ABE
:101A800067EE867AFFF766BB079A9FED447A128F5E
:101A900007EE902AF8EEE77A414A67EE877AC2EDC0
:101AA000007AFCF7CABC3F4AFCF71CBD9FED368AA2
:101AB000FFF7C5BA9FED348AFFF78BBAA3F50C4345
:101AC000A03BFFF70CBB9FED380A384B0B9325EE7C
:101AD000800A20F099FCDFF8F080D4F8B061A8F813
:101AE0000600FDF70BBDA3F50C43A03BFFF712BBAF
:101AF0003346FFF7FBBA07EE906AB8EEE76ADFED10
:101B00002C7A9FED327A84F8846126EE276A76EE8D
:101B1000077AFDEEE76A16EE903A2033402B40F24A
:101B200077819FED197A1E4BFDEEC67A83ED017A1F
:101B300017EE903A2033402B00F26781DFED247AD4
:101B4000B4EEE76AF1EE10FA40F37C82DFED195A49
:101B5000DFED197A01E0B0EE666AB4EEE76AF1EE05
:101B600010FA76EE656AF6DCDFED147AF4EEE76AD9
:101B7000F1EE10FA40F16382DFED0E5A9FED106A2C
:101B800030E000BF605100200000000084F9223FD7
:101B9000A03F0020C4460020CDCCCC3D6F12833A3C
:101BA00078000020E08200200000C8422051002080
:101BB00035FA8E3CDB0FC940E4CB1641DB0F49C040
:101BC000E4CB16C144440020F4810020DB0FC93F60
:101BD000DB0F494092E741B99730083C15A82ABE6F
:101BE000F0EE676AF4EEC66AF1EE10FA76EEA57AC8
:101BF000F6D45FED0A6AF4EEE67AF1EE10FA40F3FD
:101C0000F4805FED0D6A76EEE77A67EEA75A1FED76
:101C10000F5A1FED0F6A5FED0F6AA5EE856A27EE7A
:101C2000A55AE5EE866AE5EE267AC4ED627AFDF7FE
:101C300094BFDA49DA4A8C46FEF7FBB892ED000A07
:101C400007930891069220F0DFFBDFF8A4E3DFF8AA
:101C5000A483DEF8ECE0DFF8A0C3A8F800008CFB5A
:101C60000E3C4FEAEE70C0EBAC1007EE900AF8EEB7
:101C7000E77A069A079B0899FDEEE77A17EE900A35
:101C8000A8F80200FCF733BC04F012FE069BDFF854
:101C900064839BF80070C01AA8F80200FEF788B9A8
:101CA00004F006FE069BDFF84C83D4F8B4A1D4F808
:101CB000B061C01AA8F80200FEF759B904F0F8FDA7
:101CC000069BDFF830839AF80020D4F8B0619BF8C7
:101CD0000070C01AA8F80400FEF771BAB14B1B6877
:101CE00003F59C530833C4F898313B78012B7DF4FD
:101CF0005CAB94F89431002B7DF457ABB378032B95
:101D000000F096810FF0EAFF012384F89431FDF78B
:101D10004CBB09981AF04EFDFEF769BDDFEDA27AC3
:101D2000F4EEE76AF1EE10FA40F32381DFED9F5AFB
:101D30009FED9F6A01E0F0EE676AF4EEC66AF1EE8D
:101D400010FA76EEE57AF6DCDFED9A6AF4EEE67AE2
:101D5000F1EE10FA40F16981DFED945A9FED966A39
:101D600001E0F0EE667AF4EEC67AF1EE10FA77EE64
:101D7000A56AF6D4DFED917AF4EEE76AF1EE10FA97
:101D800004DDDFED897A77EEE66A95E5DFED8C7AA2
:101D9000F4EEE76AF1EE10FA44BFDFED867A77EEF3
:101DA000E66A89E5874B1B78002B7BD1864B1B8B22
:101DB00007EE903AF8EEE77AFEF760BCA8F8060066
:101DC000A5F8A860FBF719BB754901F1800CFEF777
:101DD000DDB90A9B002B7FF4C0AD099B9C46079B95
:101DE0009C45B8BFF0EE667AB7E5DFED756AF4EEB4
:101DF000E67AF1EE10FA44BFDFED6E6A76EEE77A2E
:101E000003E77346614642463BE5DFED707A0CE737
:101E1000B4EEC76AF1EE10FA0FDDB0EE677ADFEDCF
:101E2000635ADFED636A01E0B0EE677AB4EEE67AFA
:101E3000F1EE10FA77EEE57AF6DC9FED5E7AF4EEDD
:101E4000C77AF1EE10FA0FD5B0EE677ADFED575A88
:101E5000DFED596A01E0B0EE677AB4EEE67AF1EEB2
:101E600010FA77EEA57AF6D49FED547AF4EEC77A9D
:101E7000F1EE10FA36DD9FED4C7A77EE677A67EE79
:101E8000A75A9FED535ADFED536A9FED537AE5EE63
:101E9000856A27EEA55AA5EEA67AE5EE077AB0EE9A
:101EA000677A40E6DFED497AFEF7E8BB9BF8001061
:101EB000132943D04BB106F5F460B0EE480A28442C
:101EC000D5F89C379847B0EE408A9BF80030132B2A
:101ED0007DF481A8B0EE480A20F096FAA8F8020036
:101EE000FDF77BB89FED367AF4EEC77AF1EE10FA83
:101EF00044BF9FED307A77EE677AC0E794F8E0311F
:101F0000002B7BF429A9FBF712B9344A4FF0FF31BB
:101F10001360072351603B70FEF7A1BB304AD35CCE
:101F2000002B7EF49CAB00234FF0FF32C8F800304A
:101F30000423C8F804203B70FEF791BBB0EE480ABA
:101F4000079320F061FA079BA8F80000B2E7DFF8DA
:101F5000AC80D8F8000007F0D7FD224B1B78002298
:101F6000022BC8F800207EF478AB07F09DF9FEF74D
:101F700074BBF0EE667AE7E60B9BD3ED03DA1A4BFF
:101F800093ED020A194B38EE6DDA28EE800A20EE46
:101F90000D0A83ED020AFBF7AABA00BFE052002047
:101FA00094220020E0750020DB0F4940DB0FC94080
:101FB000E4CB1641DB0F49C0E4CB16C1DB0FC93FB0
:101FC000DB0FC9BF40580020185800200000000057
:101FD00092E741B99730083C15A82ABE287E002018
:101FE000004A030874440020183A002000440020EE
:101FF00060010020F4810020D34D6210D4730020D2
:1020000094F8D031002BB7D1104B2B4493ED000A3C
:10201000059BD3ED01DA28EE800A38EE6DDA20EE6A
:102020000D0A8AED000AFBF762BAF0EE676AA1E6D4
:10203000802017F01DFB00287DF4B7A962E6F0EEC2
:10204000667AD6E5F0EE466A8EE500BF183A0020C3
:102050002DE9F04F2DED028BBC4ABD49137895B0A8
:102060000446089000F59C4020300A900860002B40
:1020700000F06E86B74909688C4240F28582B64905
:102080000491D1F80090B54DB549B64C0291013B91
:10209000137009F480530793002B40F08382B24BF6
:1020A00005931E7806F00106029B5B7D002B40F035
:1020B0008A8219F4004F40F0CD8719F4807F0BD04D
:1020C000AA4B089ADFF8DCB29A429BF8023001F280
:1020D000BE81002B41F0BF81B4F90630A44F19F442
:1020E000805840F0E785029AB2F81AA05345B4BF71
:1020F0004FF0000A4FF0010A9E4B1B6813F080530B
:1021000000F08182002E00F0828202999A4A898C26
:1021100092ED037A039207EE901AF8EEE77AB4EEA6
:10212000E77AF1EE10FA81F27A80BAF1000F40F00E
:10213000778295F8A420002A40F072828F4A904955
:10214000106890F8300000220A604A608A60002817
:1021500040F066828B4A1070002E40F0678238781B
:10216000029AB4F900C0518B928BB4F902606145B8
:10217000B4BF4FF0800E4FF0000E4EF040036245AA
:10218000D8BF73469B0843F0800EB142B8BF734678
:1021900043F0400EB242C8BF73469B08B4F904E056
:1021A000B4F9066043F0800C8E45C8BF634643F027
:1021B000400C9645B8BF63469B0843F0800E8E42A4
:1021C000C8BF734643F0400E95F8A6C09642B8BF0C
:1021D00073469C4500F06086002285F8A63085F89D
:1021E000A720002800F0A387049B1A6802F00402CD
:1021F000002A40F00F850DF14808634E0022C8F810
:10220000042006F1500A129240F6330B4FF01909E0
:1022100040F2833702E00436564520D0B278F37896
:102220009A4219FB0270F6D27178043119FB0372DD
:1022300034F911305B45A8BF5B46B3F5617FB8BF89
:102240004FF461739842E6DA9A42E4DB317823294D
:10225000E1D84046043603F015FB5645DED14B4A23
:10226000444B177898E8030083E80300002F00F040
:102270005984474B06933F48012103F013FB002884
:1022800040F05583049B1B68D90500F14B83414EF8
:10229000DFF814813748B8F8007027F00107BFB2A3
:1022A0000221A8F8007003F0FDFA002840F05C87D6
:1022B00027F00207BFB2A8F80070374BDFF8ECA098
:1022C0001978DAF804000793BF0708BF81F002010C
:1022D000C1F3400104F0A8FF366816F00A0F40F081
:1022E000B082B8F80070B60600F1D8820C212148FF
:1022F00003F0D8FA002800F00683284B1B7847F437
:102300008077082BA8F8007000F007830E2B00F0F0
:102310000483049B1B685E0579D5214B1B79002B38
:1023200000F0AF811421134803F0BCFA002840F0FC
:10233000AD8110F0E9F8012009F072FE002866D0A6
:10234000DFF86C9000254FF0CC0B36E0C87F002002
:10235000D47E0020C47F0020386E0020A0240020FE
:102360000C5D002004220020B4550020404B4C009E
:10237000F0040020047E0020E0820020482000209D
:102380000C440020742400207C4400207C84002025
:102390004C200020385100205886002028220020A0
:1023A000888200205C200020442000205C860020E1
:1023B000486E0020DDB2022D29D80BFB05F76B1CFF
:1023C00059F80760002EF5D1C378BB4A90F9020096
:1023D00052F823300196032200920121324608F080
:1023E0000FFE034605EB450000EB0010089353B1C8
:1023F000314609EB8000CC2222F01EF9089B49F8F7
:1024000007300135EDB21AF031F90028D3D1059B20
:102410001D7815F0010500F0F382A84B01221A7017
:10242000069BB4F906101B68A5485A8901269142FB
:10243000067080F25D83A34B4FF07E521A60A24A71
:10244000029BB4F900E01E8B92F9043057781078A3
:10245000002BAEEB060314BF01224FF0FF32002B1E
:1024600040F33A83B3F5FA7FC0F23C834FF4FA733A
:102470001B1A07EE903AF8EEE77A039B7645C3ED18
:10248000007A03DDF1EE677AC3ED007AB4F902E079
:10249000AEEB0603002B40F36F82B3F5FA7FC0F278
:1024A00071824FF4FA731B1A07EE903AF8EEE77A4E
:1024B000039B7645C3ED017A03DDF1EE677AC3ED48
:1024C000017AB4F90400831B002BD8BF331AB3F58B
:1024D000FA7F80F24D82BB42D8BF002700F34A82C8
:1024E00002FB07F207EE902A039A049BF8EEE77AC4
:1024F000B042C2ED027ABCBFF1EE677AC2ED027A59
:102500001A6812F4805200F01E82B1F5FA6FA8BF6B
:102510004FF4FA61B1F57A7FB8BF4FF47A71A1F543
:102520007A746A496A4881FB0437E317C3EB67137F
:102530005F1C6FF0630E30F9177030F913000EFB5B
:1025400003433C1A03FB04F381FB0341DB17C3EB9A
:10255000611303441BB207EE903A039BB8EEE78A7F
:1025600083ED038A002A40F07883B8F800305806DB
:1025700000F1CC80002D40F057811EF023FF15B0F4
:10258000BDEC028BBDE8F08F524B0493D3F8009062
:10259000514B029309F48053504D514C0793002B3B
:1025A0003FF47DAD00214F4803F07CF94E4B0028ED
:1025B00001F008811E780593029B5B7D06F0010601
:1025C000002B3FF476AD029A013BD27D34F91330F3
:1025D000002A40F0D285A3F57A73B3F57A7FA8BFBD
:1025E0004FF47A7323EAE37307EE903A9FED3F7A54
:1025F000F8EEE77A67EE877A3D4AFCEEE77A17EE67
:10260000903A138059E519F4800F7FF47BAD0022D6
:1026100085F8A420374A0392BAF1000F3FF48EAD3B
:10262000354A01211170002E3FF499AD19F0100FB9
:102630003FF495AD314A1278D2063FF590ADB8F12E
:10264000000F7FF48CAD002B7FF489AD19F4800F5F
:102650007FF485AD3878002801F02685284B9B78DB
:10266000BAF1000F41F08C853BB1264A264B126827
:102670001B689B1A002BC1F27385012385F8A530D6
:102680006EE5059B1B78DD077FF553AE3C2016F009
:10269000EFFF00283FF4BBAE07F05CFA3C2016F0D9
:1026A00093FF00283FF4B3AE07F054FA3C2016F035
:1026B0008BFF0028F0D1AAE668630308B555002017
:1026C000AC23002050240020387E00201F85EB51D1
:1026D000B8550020386E00200C5D0020A02400209A
:1026E00004220020047E0020B4550020AAF1823F7D
:1026F00080200020E082002074240020721E002030
:10270000647E0020E0750020C0300020A04BA14A6C
:10271000B3F90430A049DFEDA16A09889FEDA07AE2
:1027200082FB0302DB17C3EBA2035B1A1BB207EEAB
:10273000903AF8EEE77A67EEA67A77EE876ABDEE12
:10274000E66A16EE103A2033402B40F27B87BDEE4E
:10275000E77ADFED946A17EE103A2033402B00F24F
:10276000F2879FED917AF4EEC77AF1EE10FA41F319
:102770006C83DFED8E5A9FED8E6A01E0F0EE477AB2
:10278000F4EEC67AF1EE10FA37EEE57AF6DCDFED1C
:10279000897AB4EEE77AF1EE10FA41F15A83DFED6F
:1027A000835A9FED856A01E0B0EE677AB4EEC67A8F
:1027B000F1EE10FA77EE257AF6D49FED797AF4EE01
:1027C000C77AF1EE10FA00F33A859FED7C7AF4EEC9
:1027D000C77AF1EE10FA44BF9FED767A77EE677A0A
:1027E00067EEA75A9FED765A9FED766A9FED767A4F
:1027F000A5EE856A27EEA55AA5EE867AE5EE077A5C
:10280000039A92ED016AD2ED005A27EEC67A65EE80
:10281000A77AA5EEA67AE6EE267A82ED007AC2EDD8
:10282000017A002D3FF4A9AE079BDAF80000197871
:1028300001F0010104F0F8FC15B0BDEC028BBDE81D
:10284000F08F0521614803F02DF8B8F800700028DA
:1028500000F066847A0740F1E48606215B4803F0C5
:1028600021F8002800F055847B0640F1D48607212A
:10287000564803F017F800283FF435AD444B454A5D
:10288000B3F904304449B8F8007082FB0302DB1747
:10289000C3EBA203B6060B807FF528AD4C4B1B782B
:1028A000980704D54B4E3378042B01F23D8017F086
:1028B000300F3FF41BAD102009F03EFC202009F042
:1028C0003BFC454BB8F8007000221A704349444A5B
:1028D0004448454D00230B604449036000260E60C8
:1028E0004B608E604E618B61CE612B605360936153
:1028F000166096605661D6610C21344802F0D2FF12
:1029000000287FF4FAAC3A4B1B7827F48077BFB2EB
:10291000082BA8F800707FF4F9AC27F04007A8F85E
:102920000070F6E4334BDB78002B3FF4B0AC324E52
:1029300033689A077FF5ACACDFF8C080B8F8007058
:1029400047F00107B4E4029B588B8142C0F2F38246
:10295000B1F5FA6FD4BFC0EB0101C0F5FA614FF4D5
:102960007A7303FB01F3C0F5FA60B3FBF0F4D8E52A
:102970004FF4FA73DF1BB3E5A6EB0E03B3F5FA7F52
:10298000BFF68FAD9842FFF68EADDFED067A8FE58C
:102990005C1E002067666666BC30002035FA8E3CFF
:1029A000DB0FC93F00000000DB0F4940DB0FC940CF
:1029B000E4CB1641DB0F49C0E4CB16C1DB0FC9BF26
:1029C00092E741B99730083C15A82ABE047E002042
:1029D000721E0020741E0020DA450020C44600202C
:1029E0007446002020240020242400209C4600203F
:1029F000282200205C2000203851002044200020A4
:102A0000BA4B1B780893002B7FF40AADDFF830B384
:102A1000DFF830931BF8030C99F800705946ABF1BE
:102A2000030613F0FBFD002800F08D82089B002FA9
:102A30004FD106F10801707913F0F0FD002841F044
:102A40003582AB49B07A13F0E9FD002800F08E82A0
:102A5000022F41F02E82A749F07B13F0DFFD002802
:102A600041F02A82A449307D13F0D8FD002800F0FF
:102A70008E82042F41F02382A049707E13F0CEFD98
:102A8000002841F01F829E49B07F13F0C7FD002847
:102A900000F08E82062F41F018829A4996F82300A2
:102AA00013F0BCFD002840F07D87974996F8280078
:102AB00013F0B4FD002800F08E82082F40F08387C9
:102AC000924996F82D0013F0A9FD00283FF4A8AC18
:102AD00009231A4600F068BFA6EB0E03B3F5FA7F90
:102AE000BFF6C4AC9842FFF6C3ACDFED897AC4E40C
:102AF000B1F5FA6F80F22182187A8B1A03FB00F38A
:102B0000C2F5FA6293FBF2F3C3F1640307EE903A65
:102B1000F8EEE77A9FED7F7A7F4B67EE877AC3ED19
:102B2000007A8CE4DFF820A2DFF820820AF15A064E
:102B30004FF0010951461AF8010C13F06FFDF8B17E
:102B40009AF804009AF802309AF803E000EB40018A
:102B500005EB8101013BD1F8B42003EB430343446F
:102B600093420DD095F8E02081F8B0E009FA00F02A
:102B700022EA0000C1F8B430C1F8B87085F8E0006E
:102B80000AF1060AB245D5D1644B654A0693194647
:102B9000644BD2F800A009681B78634E0891D146B7
:102BA000079300274FF0010BA246736853B31C78BC
:102BB00044B3B168A9EB010100290ADB95F8E010E4
:102BC0000BFA07F021EA000109F5FA7085F8E01028
:102BD000B060079AB2B1317858780431C9B2002890
:102BE00040F02283029A3AF91110108B00F1C80EBE
:102BF000714540F36C8695F8E0109B783941CA071F
:102C000040F1C6860137042F06F10C06CDD154469B
:102C1000FFF731BB95F8AB3053B1059B1B78D90753
:102C200006D5029BB4F906205B8B9A4200F3A2867C
:102C300011213E4802F036FE002800F0B48295F8DB
:102C4000AE302BB995F8A93013B93223A5F8AC30C2
:102C5000012385F8AE30FFF7CEBA1D21334802F0CC
:102C600021FE00283FF481AC314BDB78002B7FF450
:102C70007CACDFED307A304938EE678AC6F5FA630E
:102C8000FDEEC87A1BB2CDED027ABDF90820120321
:102C900081FB0201D217C2EBA11203FB02F343F343
:102CA0000F33334407EE903A039BF8EEE77AC3ED17
:102CB000037A5AE41D211D48039302F0F3FD039BA0
:102CC00000287FF410AA1D49029AB1F806A0128BC1
:102CD000A2EB0A018B4240F3238652449342B4BFD5
:102CE0004FF0000A4FF0010AFFF706BAB555002071
:102CF000683800206D3800207238002077380020B6
:102D00007C38002081380020863800208B38002055
:102D1000000000000AD7233C502400204C20002053
:102D2000E0750020D844002050250020047E0020BB
:102D30005C20002000007A44D34D621068400020DF
:102D40005E3800208000002076370020CC4C03083D
:102D5000A74DA84B2E780293DFF89C82002E00F03E
:102D60001682B6B1DFF8E092DFF8E0B2A24FCA46B1
:102D70000024072C3846E1B2D8F8043041F37081C2
:102D8000984700B20134A6422BF8020F0AF1040A58
:102D9000EFD19A4B04931A46994BD2F80090089AB7
:102DA000A3FB023E42F2010319EA03034FEA9E1E0F
:102DB000059300F0E8819348934A944B0078944936
:102DC000039012781A70039B087023B18F4B1B7805
:102DD00083F0010303938F4A029912788E4B0E926F
:102DE000104698F800200692A3FB00B30A465B0841
:102DF000148D91F822C00C9403EB4303148BC98CFF
:102E00002E781194C31A95F829400991DBB20F94DA
:102E10000F220CF1040C0B93804F814CDFF830A291
:102E20000998CDF8409009F480535FFA8CFCDDF8E6
:102E30003C9085F82820B3460D9207930021099510
:102E4000CDF83C8036B9069B9C458DBF1E46E346B7
:102E50006646B346B14280F28582039B002B00F0A8
:102E60001982704B33F911201FFA82F880454FEA1E
:102E7000410303D30C9DA84540F258825AF8212003
:102E8000964580F01082E25E059D002D40F027827D
:102E9000E25201310637D5E795F8A790B9F1F90F5D
:102EA00000F2B78109F101095FFA89F985F8A79065
:102EB00085F8A630002800F03B81B9F1140F7FF4AB
:102EC00093A95F2B40F048810598027812F0010128
:102ED00000F0C3875449897802F0FE02027000298D
:102EE00041F08C80049A1268520700F1BA813A7856
:102EF000002A40F0BB810021BB2B129101F0218000
:102F0000B72B01F00380BE2B01F06F80BD2B01F0C9
:102F1000D6809E2B01F0E6809D2B01F0DB80AE2B4E
:102F200001F0E780AD2B7FF45FA9FF21002012F0B4
:102F300029FCFFF759B9134615E51B7AC3F1640361
:102F400007EE903AE4E50BF10501707913F066FBAA
:102F500000283FF476AD012F40F0A88706F10D015F
:102F6000B07A13F05BFB002840F0A3872F49F07B79
:102F700013F054FB00283FF475AD032F40F09C87FD
:102F80002B49307D13F04AFB002840F098872949EF
:102F9000707E13F043FB00283FF475AD052F40F021
:102FA00091872549B07F13F039FB002840F08D87C9
:102FB000224996F8230013F031FB00283FF475AD49
:102FC000072F40F0EF841E4996F8280013F026FBE7
:102FD000002840F0F8841B4996F82D0013F01EFBE2
:102FE00000283FF41DAA092F3FF41AAA70E500BF7C
:102FF000A02400200C5D0020F8210020386E002065
:10300000D34D6210B07E0020C41A0020C51A0020E3
:10301000D8440020C97F0020ABAAAAAACC24002053
:1030200004220020A42400207E8400206D3800208B
:1030300072380020773800207C380020813800204A
:10304000863800208B38002088810020A2240020B0
:10305000CC7F0020D5F88C30089AD31A002BFFF6CD
:103060002CA8B54A95F89030517CB44A029F32F8AA
:1030700011200A98B97DC5F88C00013303F00F03C5
:1030800085F890302B4492B292FBF1F283F89420B1
:1030900095F8940095F8951095F8962095F8973046
:1030A00001440A4495F8980095F89910134418447F
:1030B00095F89A2095F89B3001440A4495F89C00B5
:1030C00095F89D101344184495F89E2095F89F306C
:1030D00001440A4495F8A00095F8A110134418443F
:1030E00095F8A23095F8A32001440B441A4442F30A
:1030F0000B12642AF97DA8BF642213B209B1C2F190
:10310000640307EE903A9FED8E7AF8EEE77AFFF7C8
:1031100071BA27F04007BFB2A8F80070FFF7A7BB4D
:1031200027F00407BFB2A8F80070FFF796BB8146EE
:103130000021844802F0B6FB002846D0002385F821
:10314000A83006F04BFF95F8A730142B7FF44CA85D
:103150003B78002B41F00080059B1B7803F00103B6
:10316000002B7FF441A83BE0BB073FF5A6A847F042
:103170000207A8F80070FFF7A0B8C3F53B63083357
:103180001BB2FFF728BA704B1B7803931DE693F828
:10319000223098F800600433DBB2B3428EBF2E7049
:1031A0002B701E46DDE595F8A930002B3FF423A8CF
:1031B000059B1B7813F001037FF41DA8012285F8FD
:1031C000A93085F8AA20FFF716B8059B5F4A1B783F
:1031D0001060DB0700F17A85B9F1140F7FF404A8C1
:1031E00095F8A630572B00F08F85049A126812F0DC
:1031F00004022AD05A2B28D195F8A930002B40F090
:10320000618795F8AB3083F0010385F8AB30FEF7AA
:10321000EFBF85F8A6C000288AD0FEF7E5BF0122DF
:1032200085F8A420FFF7FCB9012800F0A38595F8E4
:10323000E0100BFA07F30B4385F8E030E2E49FED72
:10324000447A77EE677AFFF7CBBA5D2B00F0E3851F
:103250005B2B00F09F835E2B00F00386562B00F063
:1032600049863A782AB16F2B00F03286374A00211E
:103270001160972B00F03486A72B7FF43CAE3549C4
:10328000049B1A680B7843F004030B7002F00402ED
:10329000FEF7AEBF002847D05AF8212096454FEAE6
:1032A0004103FFF4F0AD2C4A2B4DD25C05EB030833
:1032B000002A00F04C82022A40F0A18198F80120F7
:1032C00002EB820202EB820202F2EE2292B20329A8
:1032D00040F3B480059D12B2002D3FF4D9AD0B9D93
:1032E00003EB0108A844099D05EB4808A8F82C2029
:1032F000B9F1000F03D10E9D022D7FF6C9ADB7F8CD
:1033000002903A88B7F804804A449044134A0FFA6E
:1033100088F882FB0852124DA2EBE87225F8038070
:1033200012B24FF00109B3E502464B000EF5967854
:103330004AF82180A8E500BFE87500200476002047
:1033400014AE2341047E0020D8440020C430002065
:10335000DB0F4940721E0020BC8100205655555598
:10336000142500200D99099DBC4BDDF83C8085F8A3
:1033700000B04A460F2985F829200CBF01220022FF
:10338000DDF8409085F828101A7006D11B21B4484A
:1033900002F088FA002800F01E85B248B24AB34B0A
:1033A00011688268C1608A1A012119704368B04FA0
:1033B0009A42029A397088BF002392F8227088BF1F
:1033C00080F82130079B98F80000B2F818C0B2F8D6
:1033D00026800437FFB2002B00F0C6818742A54A41
:1033E00040F25182A44F964600210EB9834606460C
:1033F000B1421ADA12F8113093B1022B0ED19EF8B5
:10340000013003EB830303EB830303F2EE239BB250
:1034100027F8023B01310EF1020EE6E73B88F7E7A1
:10342000CBB2032BFAD86346F2E785F800B00E9BC7
:10343000924A01331370079BFEF72EBE012505FA51
:1034400001F80D9D25EA080512B20D951CE513B98A
:1034500001238BF802301B2013F018F9884F9BF8DA
:1034600021A09BF82030DFF83082DFF8FC91039038
:10347000052B00F2AF80DFE803F0948855182A404E
:1034800013F030F9012800F0F584039B002B70D075
:103490007C4B1B79002B6CD00BF07AFA03224FF493
:1034A0007A738BF82020CBF81C30B8F8003043F04A
:1034B0000203A8F8003007F00DFAD9F80020DBF875
:1034C0001C3013440422CBF818308BF82020BAF1BA
:1034D000010F40F08E84D9F80030DBF818209A42B2
:1034E00078D2387818B913F0D1F8002872D1B8F82A
:1034F000003023F00203A8F80030624BD9F8002016
:10350000DB88642101FB03234FF480600022CBF8A9
:1035100010308BF820208BF8032008F00DFE9BF86C
:103520002030A5E7BAF1010F04BF05238BF8203046
:10353000002E5AD0029BD9F800E0B3F91800514B85
:10354000002160F30F0160F31F41B3F902302160E5
:103550000022DBF8141060F30F0263F31F42714581
:10356000626044D3BAF1010F40F001869BF820302D
:103570007EE7BAF1010F2DD0D9F80030DBF810202A
:103580009A423ED301238BF82030BAF1010FB4D018
:103590003C4B1B7A012B34D00BF0FAF99BF820300E
:1035A00066E7002E7FF46CAF039B4FF48060002B26
:1035B00000F0058108F0C8FD059B1E78049BD3F838
:1035C00000900023CBF8103006F00106B4F9063065
:1035D000FEF785BD059B1E78049B06F00106D3F817
:1035E0000090B4F90630FEF77ABDD9F8003047F202
:1035F00030520323CBF81C208BF8203055E7E25AD9
:1036000065E60BF0C5F9032240F6B8338BF82020AD
:10361000CBF81C3049E747F04007A8F80070FFF7E7
:1036200026B9194B194AB3F90430194982FB030230
:10363000DB1747F00407C3EBA203A8F800700B8068
:10364000FFF70BB9F4EEC77AF1EE10FA40F30C84F1
:10365000DFED135A9FED0F6A34E000BFD94400201C
:10366000047E00205C200020E0750020C41A0020A9
:10367000C51A0020BC81002004220020C97F002040
:10368000F0040020943800205C1E00206766666607
:10369000E4460020E4CB164142200020DB0F49C065
:1036A000DB0FC940E4CB16C1DB0FC93FDB0F49403C
:1036B00092E741B99730083C15A82ABE00000000E7
:1036C000F0EE476AF4EEC66AF1EE10FA36EEE57AED
:1036D000F6DC5FED0E6AB4EEE67AF1EE10FA40F138
:1036E000C6835FED115A1FED116A01E0B0EE667AF4
:1036F000B4EEC67AF1EE10FA77EE256AF6D41FED35
:10370000167AF4EEC76AF1EE10FA40F389801FEDE5
:10371000197A77EE666A66EEA65A1FED1B5A1FED00
:103720001B6A1FED1B7AA5EE856A26EEA55AA5EE4B
:10373000867AE5EE076ABDEEE77A17EE103A203397
:10374000402B7FF60EA85FED237AFFF759B8CAB277
:10375000022A40F2B882032A7FF451AF119A079DE2
:10376000002D08BF0246B2E587421946B64A63D823
:10377000B64896460EB9BB463E468E427FF755AEDA
:1037800012F8113093B1022B0ED19EF8013003EBE9
:10379000830303EB830303F2EE239BB220F8023B87
:1037A00001310EF1020EE5E70388F7E7CBB2022BF9
:1037B00003D9032BF8D14346F0E76346EEE708F060
:1037C000BBFCF9E61F4605931B7813F001063EF497
:1037D0006BAC9F498E7803F0FE033B70002E3EF4E5
:1037E00063ACDFF8908298F800200B2A0DD80121F5
:1037F000914040F603060E4040F02F8411F4C06F54
:1038000003D0093A012A40F2D384924A92491268BD
:103810004A600B2203F0010688F80020FEF744BC42
:103820009FED8E7AF4EEC76AF1EE10FA44BF9FED79
:103830008C7A77EE666A6EE7844F96460EB98346B9
:103840000646B142BFF6F1AD12F8113093B1022B2A
:103850000ED19EF8013003EB830303EB830303F2E5
:10386000EE239BB227F8023B01310EF1020EE5E791
:103870003B88F7E7CBB2022B03D9032BF8D14346A1
:10388000F0E76346EEE77148964600210EB9BB4665
:103890003E468E427FF7C9AD12F8113093B1022B2C
:1038A0000ED19EF8013003EB830303EB830303F295
:1038B000EE239BB220F8023B01310EF1020EE5E748
:1038C0000388F7E7CBB2032BFAD86346F2E7C83890
:1038D000814242DA95F8E0109B783941C8073FF5FC
:1038E00091A9C3F10008611E162900F2A980DFE842
:1038F00011F09E01B2018701FF00C601D7017401DA
:1039000061014C0137012201A700FF000F01D7011F
:1039100074016101EB00D700C300970081006D00C6
:103920004FF0010AFEF7E8BB0A2012F0AFFE814615
:10393000002800F07382F90640F1068395F8F090B4
:10394000B9F1000F7EF4D2AC012385F8F030B9F163
:10395000000F7EF4BBAFFEF7C9BC95F8E0300BFA60
:1039600007F123EA010309F5FA7185F8E030B16047
:10397000FFF748B900213B4801F094FF00287FF48D
:1039800057A9322385F8AB00A5F8AC30FFF750B942
:103990009846A8E7344B0121344E35483170036016
:1039A000FEF726BC07231A4602EB8202164489F86A
:1039B0000030B17870781CF00DFD059B1D7805F086
:1039C0000105FEF72DBD08231A46EDE7D5F8E40002
:1039D0001F4B90F83A109C7841446429A8BF642199
:1039E00021EAE17180F83A10002C40F0DD830BF001
:1039F000B1FD1CE4D5F8E400154B90F83B109C7821
:103A00004144FE29A8BFFE2121EAE17180F83B1064
:103A1000002CECD0162012F097FED5F8E400E6E773
:103A2000089A0B4B51784144B1F5967FA8BF4FF4EB
:103A3000967121EAE17151709B78002B40F0CB83A5
:103A4000D5F8E400D3E700BFBC81002004220020A9
:103A50007E840020E0750020287E0020DB0FC9BF97
:103A6000DB0F49C0047E00207A8300205A840020A6
:103A7000482000207D840020D5F8E4008178B54BF3
:103A80004144C829A8BFC82121EAE17181709B780F
:103A9000002BACD0142012F057FED5F8E400A6E7B6
:103AA000D5F8E4004178AB4B4144C829A8BFC821F0
:103AB00021EAE17141709B78002B98D0132012F01D
:103AC00043FED5F8E40092E7D5F8E4000178A14B75
:103AD0004144C829A8BFC82121EAE17101709B783F
:103AE000002B84D0122012F02FFED5F8E4007EE7E0
:103AF000089A984B9179987841446429A8BF642129
:103B000021EAE1719171002840F077830D2C97D064
:103B1000089A904B5179987841446429A8BF642150
:103B200021EAE171517100288AD00E2012F00CFEBA
:103B3000D5F8E4005BE7D5F8E400864B017A9C7881
:103B40004144C829A8BFC82121EAE1710172002CB3
:103B50003FF44DAF0B2012F0F7FDD5F8E40046E737
:103B6000D5F8E4007B4BC1799C784144C829A8BFB3
:103B7000C82121EAE171C171002C3FF438AF0A205D
:103B800012F0E2FDD5F8E40031E7D5F8E400714B1E
:103B900081799C784144C829A8BFC82121EAE171F4
:103BA0008171002C3FF423AF092012F0CDFDD5F830
:103BB000E4001CE7D5F8E400664B41799B7841446A
:103BC000C829A8BFC82121EAE1714171002B40F04A
:103BD0000E83112C7FF452AF09E7D5F8E4005D4B5A
:103BE00001799B784144C829A8BFC82121EAE17125
:103BF0000171002B40F0F582102C7FF453AFF6E6F4
:103C0000089A14794444642CA8BF642424EAE47418
:103C1000147112F0B3FD4F4B9B78002B3FF410AFA3
:103C20000320214612F090FDD5F8E400DFE6089A63
:103C3000484B11784144FA29A8BFFA2121EAE171E1
:103C400011709B78002B3FF4FBAE012012F07CFD3D
:103C5000D5F8E400CBE6089A3E4B917841446429BC
:103C6000A8BF642121EAE17191709B78002B3FF499
:103C7000E7AE022012F068FDD5F8E400B7E6089A36
:103C8000344BD1799878414481F30801D1710028EF
:103C90003FF4D6AE052012F057FDD5F8E400A6E6B5
:103CA000D5F8E4002B4BC1789B784144C829A8BFC4
:103CB000C82121EAE171C170002B40F043820F2C32
:103CC0007FF404AF93E6119AFFF701BB224B1B78F8
:103CD000002B3EF489AA214BDB78002B7EF484AACA
:103CE00095F8A8300133DBB2032B85F8A8307EF6B7
:103CF0007BAA1B4B5B781BB9BAF1000F7EF474AA48
:103D000006F0E8FDFFF71FBA164B17491A684FF483
:103D10007A73B3FBF2F3C3EB431203EB8203049A0F
:103D20001268DB001606A1F8A8307EF55FAA0F4BDB
:103D30001B7898077EF55AAA0D4B1B78042B7EF64C
:103D400055AA1CF0FBF9049B1A6802F00402FEF766
:103D50004FBA00BF7E840020D84400205C200020A1
:103D6000647E002020510020FC480020721E0020AC
:103D7000741E00203AF91110987840F633039942E6
:103D8000A8BF1946B1F5617FB8BF4FF461710C2C23
:103D9000A1F561714FF4966393FBF0F391FBF3F19E
:103DA00073D0182C7FF443AAD5F8E430C9B2C829DF
:103DB00093F817E00846A8BFC82086453FF437AA05
:103DC000D04AD8759278002A3FF431AA204612F0E2
:103DD000BBFCFFF72CBACC4ACC491368CA688B608D
:103DE0009B1AC82B7FF623AB012381F82130FFF704
:103DF0001EBBD9F80010DBF81C30059A0B4416786E
:103E0000CBF81830049B06F00106D3F80090B4F903
:103E10000630FEF764B9BE4B0021BDE5FA0600F19D
:103E2000D9800B2012F032FC002840F0A480BB06A1
:103E300000F1DD8095F8F030002B3FF485ADB9F14D
:103E4000000F7EF443ADFEF751BAB0EE677AFEF78D
:103E50009EBCF0EE477AFEF7B0BC85F8A710FFF7DE
:103E6000C4B9AC4B022197E5B0EE667A31E4F0EECE
:103E7000476A44E4A84BD9F80020DB88642101FBA1
:103E80000323CBF81030FFF700BBA44B5B78C9B21B
:103E90008B423FF4CCA90846099104F003FF994BEB
:103EA00009999B78002B3FF4C2A98FE701231A469A
:103EB0007AE502231A4677E503231A4674E50423BC
:103EC0001A4671E505231A466EE506231A466BE588
:103ED00006F084F8049B1A6802F00402FEF788B921
:103EE000049A8F4B12684FF4C871198002F00402D3
:103EF000FEF77EB91AF0BAF901F0FFFE1AF09EF94A
:103F000003F022FD95F8A630FFF7ABB90B464FF64C
:103F1000FE71844A568990893344014453819181CA
:103F20001AF0A4F901F0E9FE1AF088F903F00CFD8B
:103F3000049B1A68002302F0040285F8A730FEF7FC
:103F400057B90B460221E4E7102008F0FDF82020C5
:103F500008F0F2F87449081F1CF066F9734B02224E
:103F60001A7095F8F030B8F80070002B7EF4AEAC03
:103F70004FF00109E8E46E4B03995B8991ED007AFB
:103F800007EE903AF8EEE77AB0EEC77AB4EEE77A49
:103F9000F1EE10FA7FF54BAF91ED017AB0EEC77AF2
:103FA000F4EEC77AF1EE10FA7FF741AFB9063FF5AC
:103FB00041AF202008F0C8F85E497268B368C5F8C0
:103FC000E820081FC5F8EC301CF02EF9574B0122F1
:103FD0001A70C6E7102008F0AFF8544BB8F800701C
:103FE00083F800904FF001091BE7022391E720209E
:103FF00008F0A2F84D4B00221A70B2E7DFF84081BA
:1040000098F800100B291AD80120884040F60306C2
:1040100006407EF467AF10F4C06F10D00939012953
:104020000DD8452017F03AFBFF2017F037FB424828
:1040300017F020FB304617F031FB059B1A78324908
:104040003E4B096859600B2102F0010388F800100B
:10405000002B7EF4C9A8FFF7C3B80646FEF724B8C4
:10406000029A115D9847032C1BDC40F2EE2240F6C9
:10407000CA0C00283EF486AE39F824E0BAF80210E3
:104080004FF47A73A0EB0E0003FB00F0A1EB0E01DE
:1040900090FBF1F018449042B8BF10466045A8BFAD
:1040A000604600B2FEF76EBEBAF1000F3EF4E5AA1C
:1040B00095F8A520002A4BD11846FEF751B84FF6C7
:1040C000FE7326E70021012385F8A91085F8AA30A0
:1040D000FEF78EB80021FF2011F054FB95F8A630B2
:1040E000FEF71DBF012011F04DFB95F8A630FEF73D
:1040F00013BF0121002011F045FB95F8A630FEF713
:1041000011BF00BF7E840020E07500205C200020ED
:1041100030830020C4830020943800205A8400207B
:1041200068860020407E002088200020DA4500209C
:10413000684600208C250020D8700308287E0020C7
:104140007D8400200F2012F0FFFAD5F8E400B6E5D8
:1041500085F8A580FEF704B895F8A630FEF7B1BE45
:1041600006F0B8FB002385F8A530FDF7F8BF059AE7
:104170001678049A06F00106D2F80090FDF7AFBF5A
:104180003BB12049204A09684FF47A7606FB0313B5
:10419000136095F8A530002B3DF4E2AF00221846DD
:1041A00085F8A520FDF7DCBF172012F0CDFA47E413
:1041B000452017F073FAFF2017F070FA134817F034
:1041C00059FA304617F06AFA049BD3F80090059B21
:1041D0001B78FFF71ABB152012F0B6FAD5F8E400E9
:1041E00005E4102012F0B0FAD5F8E40004E511203F
:1041F00012F0AAFAD5F8E400EBE40D2012F0A4FACC
:1042000084E400BFE0750020C0300020D8700308AF
:10421000002870B51EDB0928044620DD012303EBCE
:1042200083035B00B0FBF3F2092AF8D87BB10E4E92
:10423000B4FBF3F00928CCBF57223022A6FB03E5DC
:10424000024403FB1044EB0801F8012BF0D10023DA
:104250000B7070BD2D230B7040420131DBE7303015
:1042600001F8010BF3E700BFCDCCCCCC884230B4D1
:104270004FF001042ED301FB04F4B0FBF4F58D42A2
:10428000F9D284B1AAB901E0B0FBF4F5092DCCBF95
:10429000572230222A4404FB150003F8012BB4FBFB
:1042A000F1F4002CF0D100221A7030BC7047B0FB42
:1042B000F4F5092DCCBF372230222A4404FB150027
:1042C00003F8012BB4FBF1F4002CF0D100221A709A
:1042D00030BC70470546002AEBD1D7E703685A1C6B
:1042E00002601970704700BF2DE9F047089C2578DF
:1042F000002B804689460CBF4FF0200A4FF0300A51
:10430000661C35B3002A29DD334601E0024698B128
:1043100013F8011B501E0029F8D1971E60B13D46CD
:10432000013D51464046C8476B1C002BF8DC257800
:1043300027EAE770013055B1041B29464046C847BB
:10434000301916F8015B002DF7D1BDE8F087BDE804
:10435000F087002A04DC2846BDE8F0870020EBE760
:10436000571EDCE70A44914251D030B441F2210497
:1043700011F8013B80EA0320430010F4004F84EA67
:1043800003059BB2ADB208BF1D466B0015F4004F8C
:1043900084EA03009BB280B208BF1846430010F4C1
:1043A000004F84EA03059BB2ADB208BF1D466B0007
:1043B00015F4004F84EA03009BB280B208BF184690
:1043C000430010F4004F84EA03059BB2ADB208BF6E
:1043D0001D466B0015F4004F84EA03009BB280B2C7
:1043E00008BF1846430010F4004F84EA03059BB24F
:1043F000ADB208BF1D466B0084EA030015F4004F00
:1044000085B298B218BF28468A42B1D130BC7047F5
:1044100083684268D0ED037A00EB83010133934255
:1044200081ED040A836004BF0023836000EB8303F3
:1044300093ED047A036870EE277A9A42C0ED037A0E
:1044400077EEC77AC0ED037A0CDA013307EE103A43
:10445000F8EEC76AB7EE007A87EEA60A036030EE80
:10446000070A704707EE102AB8EEC77A87EE870A68
:10447000704700BF90ED097A90ED004AD0ED0A6ACE
:10448000D0ED014AD0ED047A90ED035AD0ED025AF6
:10449000A4EE007AB0EE406AB0EE470AB0EE667A5B
:1044A000A6EE247A67EEC07AA0EE457AE6EE257A8B
:1044B00080ED097AC0ED0A7A704700BFD0ED057A29
:1044C00090ED013AD0ED003AD0ED064A90ED024A67
:1044D00090ED077A90ED035A90ED086AD0ED045AFA
:1044E000C0ED067AF0EE406A27EE830AC0ED056A59
:1044F000A3EEA60A80ED087AA4EE240AA5EE470AE8
:10450000A5EEC60A80ED070A704700BFD0ED007A1D
:1045100090ED017A30EE670AE7EE007AB0EE670AB6
:10452000C0ED007A704700BF704700BF4FF40063D2
:10453000038270474FF400630382704750F8043CD5
:10454000012280F83520143803B11847704700BFA6
:10455000BFF34F8F0549064BCA6802F4E06213436C
:10456000CB60BFF34F8F00BFFDE700BF00ED00E061
:104570000400FA0570B4037B04681F2B08D9203BA4
:104580002021626801FA03F31A421CD170BC704703
:104590002021226801FA03F31A42F7D04269144934
:1045A000582000FB021251685689CD6808682968B6
:1045B00021F001012960828992B222EA06028281F9
:1045C000A36070BC704742690949582000FB021281
:1045D00051685689CD680868296821F00101296071
:1045E000828992B222EA06028281E36070BC70473F
:1045F0004458002030B4094B1C786CB1084A00259F
:1046000002EBC404116893884D6288890832034321
:104610009BB2A2428B81F5D130BC7047645C002014
:10462000685C002090F8493013B1002280F84920DE
:104630001846704770B5044682B01830256D94F85E
:104640005C106B460622A847A8B19DF804009DF8AF
:1046500000609DF801109DF802509DF803209DF820
:10466000053041EA062143EA002342EA0522A184FB
:10467000E2842385012002B070BD00BF70B50446FE
:1046800082B00830256A6B4606223B21A847A8B1B4
:104690009DF804009DF800609DF801109DF80250FF
:1046A0009DF803209DF8053041EA062143EA0023E6
:1046B00042EA05226182A282E382012002B070BD3B
:1046C000014B186802F042BBE085002008B502F0FB
:1046D000EFF8044B5B68C01AC0F5FA5020EAE070AE
:1046E00008BD00BF1076002000B5002183B00A206D
:1046F00017F05AFB0F210A2017F056FB01AA0321DD
:10470000102017F079FB9DF90430DFED277ADFEDFB
:10471000275A06EE103A9DF9053006EE903A9DF9BB
:10472000063007EE103AB8EEC66AF8EEE66AB8EE62
:10473000C77A76EEE76A36EE676A37EE677AF7EEA3
:10474000007AB0EE675AA6EE255A194B0021B0EE5A
:10475000456AB0EE675AA6EEA55A0A20E7EE257A1A
:10476000F3EE0E5A26EE256A25EE257A67EEA57A37
:1047700083ED006A83ED017AC3ED027A17F014FB32
:104780000DF103020121022017F036FB0DF10302A7
:104790000121092017F030FB01210A2017F004FB4A
:1047A000012003B05DF804FB000000430000803BE3
:1047B0008400002038B50B4C2378054653B90A4BCA
:1047C0006278186849212B460025257001F00AFF00
:1047D000012038BDFFF77AFF0028F0D002F0B4F8CE
:1047E000EDE700BF107600200C760020F0B54A4CB3
:1047F0002578012D83B013D028D3022D0DD1474B3E
:104800001B780646002B77D16846FFF7D3FF20B10F
:104810009DF8063013F0030022D0002003B0F0BD55
:104820003E4E3378002B62D16846FFF7C3FF9DF8F8
:10483000003008B1DB0764D40023237033784BB118
:10484000002301330020237003B0F0BD334E3378D2
:10485000002BF5D10121022017F0FCFA2378F0E7B4
:104860009DF801E09DF800109DF803709DF802206E
:104870009DF805509DF80430207041EA0E2142EA6F
:10488000072243EA052309B212B21BB2494252423F
:104890005B42234806EE901A07EE102A07EE903A84
:1048A00090ED005AD0ED015A90ED026AF8EEE66AFA
:1048B000B8EEC77AF8EEE77A66EE856A27EE257AD3
:1048C00067EE867AFDEEE66ABDEEC77AFDEEE77A20
:1048D00016EE901A17EE102A17EE903A3180728079
:1048E000B38001210A2017F05FFA03B0F0BDFFF793
:1048F000EDFE002898D090E7FFF7E8FE00288CD165
:1049000082E7337823B90721032017F0A3FA25782B
:104910000135257081E700BF942500201076002026
:104920008400002038B5044690F84D0000285AD184
:1049300004F11805636D80226B2128469847642096
:1049400002F05CF8636D07226821284698476420CE
:1049500002F054F8636D00226B21284698476420CA
:1049600002F04CF8636D01226B21284698470F2016
:1049700002F044F894F84720636D022A8CBF1A2293
:1049800018221B21284698470F2002F037F8636D44
:1049900018221C21284698470F2002F02FF8636D3B
:1049A00094F846201A21284698470F2002F026F84E
:1049B000636D94F84820192128469847642002F036
:1049C0001DF8636D10223721284698470F2002F00A
:1049D00015F82846636D0122382198470F20BDE85D
:1049E000384002F00BB802F0D5F90546F0B1036883
:1049F00081881B6919409BD12023C171837102F00A
:104A00005BFB21460F4B41F8143F284616F082FF0E
:104A1000AB88B3FA83F3C3F11F03012212FA03F345
:104A200086D009490A6813430B6081E7014602F00A
:104A300043FB2146034B41F8143F284616F06AFF1A
:104A400076E700BF3D450108003C014010B5044633
:104A50000120A269138823F040031B041B0C138060
:104A600013889BB223F0380343F03003138013887C
:104A70009BB243F04003138001F066FF2046FFF72E
:104A800051FF102204F118006A2101F09FFC6420FC
:104A900001F0B4FFA269138823F040031B041B0C30
:104AA000138013889BB223F0380343F0080313806C
:104AB00013889BB243F0400313800120BDE81040EF
:104AC00001F042BFF8B5027B466903681F2A2DD961
:104AD000A2F120055F682024AC402742114617D080
:104AE0001022AA40DC60DA605A68EA40D40749D450
:104AF000716B756A0A68B46A22F00102A5420A6005
:104B000037D1012286F84C20027B11461F2A20D97A
:104B10002039082258688A40024200D0DA60042214
:104B2000586802FA01F1014221D1F8BD20241D6824
:104B30009440254211460CD0102191409C60996010
:104B40001968D140C907D3D5012101FA02F29A6050
:104B5000CEE7082218688A40024200D09A600422F8
:104B6000186802FA01F101420BD09960F8BDD960D2
:104B7000F8BD0446304602F095F8227B23681146C2
:104B8000C4E7F8BD012202FA05F5DD60B0E700BF19
:104B900070B582B004466946183016F027FFA8B1F8
:104BA0009DF805009DF801609DF802109DF80350E6
:104BB0009DF804209DF8063041EA062143EA0023CF
:104BC00042EA0522A184E2842385012002B070BD5F
:104BD000F0B484894FF6FF764FF47A7413B3002A49
:104BE0002FD01778013201E0B44218D00589013C7A
:104BF000AD07A4B2F8D5BCB284814FF47A7402E058
:104C0000BCB2B4420BD00589ED0704F1FF37F7D5EC
:104C10008589ADB209B10D700131013BDEE70A4B68
:104C2000984202D00120F0BC7047084A538B0133F0
:104C30009BB25383508B80B2003018BF0120F0BC70
:104C40007047FF27D2E700BF00380040DC73002028
:104C5000427A02B9704710B504460368406804F10F
:104C60000A0198470023637210BD00BF437A5A1CA3
:104C70000344D2B242729972037A934200D802B9C5
:104C8000704710B504460368406804F10A0198476C
:104C90000023637210BD00BF302827D0312827D0F1
:104CA000322827D0332827D0342827D0352827D0BA
:104CB000202827D0212827D0102827D0112827D016
:104CC000122827D0132827D0142827D0152827D01A
:104CD000162805D0172808BF0F2202D000207047E1
:104CE0000E22104B03EB4203587870470022F8E77E
:104CF0000122F6E70222F4E70322F2E70422F0E7BA
:104D00000522EEE70622ECE70722EAE70822E8E7B9
:104D10000922E6E70A22E4E70B22E2E70C22E0E7B9
:104D20000D22DEE7144D030870B5448806460D4693
:104D3000C4F30B042246002128461FF07DFC336992
:104D4000094A934209D3094A934206D22246284689
:104D50001946BDE870401FF04ABC23B121462846E1
:104D6000BDE87040184770BD5C0500080C060008DF
:104D7000064B07498B4202D30023184670471A8816
:104D8000C2F30B029042F8D01433F3E78801000815
:104D90005C050008024A136823EA000010607047AF
:104DA000687E0020F8B51A4D2B789F2B2ED16B789A
:104DB000BE2B2BD105221749A81C1FF088FC28BB4D
:104DC000072229464FF6FF70FFF7CCFA124FEC1D71
:104DD00022884AB1A618BE4218D2052A16D9214601
:104DE000FFF7C0FA3446F3E721460222FFF7BAFA8A
:104DF0000222A118FFF7B6FA0634084B641B1C8088
:104E000041F60F53C31A58425841F8BD0020F8BD6F
:104E1000004000080A72030800800008F8350020EE
:104E20000378202B024600F10100F9D0092BF7D0BE
:104E30002D2B2CD02B2B03BF5378B7EE000A024644
:104E4000B7EE000AA3F13001C8B209289FED467AF7
:104E500010D8F2EE046A07EE901AF8EEE77A12F82C
:104E6000013FE7EE267AA3F13001C8B20928B0EE7F
:104E7000677AF0D92E2B4CD003F0DF03452B0BD0F3
:104E8000F7EE007A67EE276A20EE260A704753781D
:104E9000BFEE000A0246D5E710B451782D2959D04B
:104EA0002B290ABF9178501C901C0024A1F13003DB
:104EB000092B53D8002303EB830301EB430310F8C2
:104EC000011FA1F13002092AA3F13003F3D9B3F590
:104ED0009A7F28BF4FF49A73072B42D9DFED236ADC
:104EE0001A46F7EE007A083A072A67EEA67AFAD849
:104EF00003F007032BB1F2EE046A013B67EEA67ADA
:104F0000FBD124B3C7EE276A5DF8044B20EE260AD6
:104F100070475378A3F13001C8B2092802F10102A9
:104F2000AAD8F2EE046AF0EE665A07EE901AF8EE8E
:104F3000E77A12F8013F87EEA66AA3F13001C8B202
:104F4000092866EEA56A37EE067AEED994E767EE91
:104F5000276AD9E7901C91780124A7E7F7EE007A39
:104F6000CFE7F7EE007AC5E70000000020BCBE4C9A
:104F7000B5EEC00ADFED317AF1EE10FACCBF30EEBB
:104F8000270A30EE670ADFED2E7A20EE270A30B5C9
:104F9000FDEEC07A87B017EE904A054684EAE470C9
:104FA000002303A9A0EBE47001930093029314F093
:104FB00095F9002CACBF20232D2303A88DF80030D9
:104FC0001CF038FB012803A924D002282DD0032887
:104FD00005BF3023684668468DF801301FF052FB4C
:104FE00068461CF027FB0338C4B2224669462846AF
:104FF0001FF0A6FB00232B5528461CF01BFB2E227E
:10500000431C2A540DEB0401E8181FF058FB2846F6
:1050100007B030BD302368468DF801308DF802307E
:105020008DF803301FF02EFBDAE7302368468DF849
:1050300001308DF802301FF025FBD1E76F12033AE3
:1050400000007A442DE9F041064615460846B6FBB5
:10505000F2F43CB905FB1464124B1B5D00F8013BF4
:10506000BDE8F081B4FBF2F767B90E4B05FB1747BB
:1050700005FB1464DA5D00F8012B1B5D00F8013BB1
:10508000BDE8F081B7FBF2F8B8F1000F02D040465E
:10509000FFF7D8FF05FB1878024B13F8082000F83B
:1050A000012BE3E71072030830B402681146531C69
:1050B000036011F8024B0160D31C517803609378B0
:1050C000151D05601B0443EA0123D078234343EAFE
:1050D000006030BC704700BF0368591C1A4601606D
:1050E00012F8021B0260587841EA0020704700BFA6
:1050F00038B50446006815461FF079FA22682A443C
:10510000226038BD036810B40A0E5C1C04601A707B
:1051100003680A0C5C1C04601A7003680A0A5C1CB1
:1051200004601A7003685A1C026019705DF8044B21
:10513000704700BF036810B40A0A5C1C04601A7050
:1051400003685A1C026019705DF8044B704700BF79
:1051500003685A1C026010B4197003680A0A5C1CC8
:1051600004601A7003680A0C5C1C04601A700368FF
:10517000090E5A1C026019705DF8044B704700BF9D
:1051800003685A1C026019700368090A5A1C0260FD
:10519000197070472DE9F047002488B080460F460B
:1051A0001E46A14605AD531C0393117839B325293A
:1051B00033D1931CCDF810900393507830284ED003
:1051C0004FF0000AA0F13003DBB2092B42D96C2862
:1051D00019D0642800F0938024D825281CD063D9E6
:1051E000582876D063281BD131784046B847039AB7
:1051F000531C03931178043601340029D7D120467B
:1052000008B0BDE8F087039B5A1C03921B78642BFF
:105210007CD02AD8252B54D1252140460134B847CB
:10522000039AC0E7732833D044D975284FD106F1CB
:10523000040E30682B4600220A217646FFF716F846
:10524000049A0095534639464046FFF74DF8039AB5
:105250000444A8E704AA03A914F01CF8B7E7D31C78
:10526000039390784FF0010AACE7732B10D05BD911
:10527000752B3AD0782B96D1A3F15802B2FA82F26C
:10528000306852092B4610210436FEF7EFFFD7E7AE
:105290003368049A0093394600234046FFF724F808
:1052A00004360444039A7EE70028B9D1204608B0AA
:1052B000BDE8F0876E28B3D1039A336804361C60CA
:1052C00071E72AD9582BD7D0632B8DD06BE778287C
:1052D000A6D1A0F15802B2FA82F2306852092B46E8
:1052E0001021FEF7C3FF0436AAE706F1040E30686A
:1052F0002B4600220A217646FEF7B8FFA0E7331DB1
:10530000306829461E46FEF783FF99E7331D306853
:1053100029461E46FEF77CFF92E7002B7FF443AF41
:10532000204608B0BDE8F0876E2BC6D03BE700BF33
:105330000EB400B584B005AB019053F8042B0649B8
:10534000039301A8FFF726FF019B00221A7004B007
:105350005DF804EB03B07047DD4201080FB430B5CF
:1053600083B006AB0A490B4853F8042B0968006860
:105370000193FFF70FFF084C0546206801F0D6FCAB
:105380000028FAD0284603B0BDE8304004B070478A
:10539000B02F0020B42F0020E0850020DFED2B7A15
:1053A000B4EEE70AF1EE10FA4ADDDFED296A9FED6F
:1053B000297A01E0B0EE670AB4EEC70AF1EE10FAFE
:1053C00070EE667AF6DC9FED247AF4EEC77AF1EEA1
:1053D00010FA38D5DFED1E6A9FED207A01E0F0EE7D
:1053E000407AF4EEC77AF1EE10FA37EEA60AF6D458
:1053F000DFED1B7AB4EEE70AF1EE10FA14DDDFED13
:10540000137A37EEC00A60EE006A9FED166A9FEDD0
:10541000167ADFED167AA6EE867A20EE266AE6EE9A
:10542000877AA6EE270A7047DFED117AB4EEE70A15
:10543000F1EE10FA44BFDFED087A37EEC00AE2E77A
:10544000F0EE407ABFE7B0EE670AD1E7DB0F4940E4
:10545000DB0FC940E4CB1641DB0F49C0E4CB16C1DA
:10546000DB0FC93F92E741B99730083C15A82ABE27
:10547000DB0FC9BF41404A0011F0800F82F0D50315
:10548000D2B2DBB208BF1346590013F0800F81F08F
:10549000D502C9B2D2B208BF0A46510012F0800F3D
:1054A00081F0D503C9B2DBB208BF0B46590013F037
:1054B000800F81F0D502C9B2D2B208BF0A465100AE
:1054C00012F0800F81F0D503C9B2DBB208BF0B46E2
:1054D000590013F0800F81F0D502C9B2D2B208BFD3
:1054E0000A46510012F0800F81F0D503C9B2DBB239
:1054F00008BF0B465A0082F0D50013F0800FD2B2DD
:10550000C0B208BF1046704709B909E0194690FBC0
:10551000F1F301FB13030846002BF7D1084670474F
:105520000146FBE7F0EEC07AB0EEE07AB4EEE77A3F
:10553000F1EE10FAB4BFB0EE676AB0EE476AB5EEAE
:10554000406AF1EE10FA46D0B4EEE77AF1EE10FAC6
:105550008CBFF0EE675AF0EE475AC5EE866A9FEDB3
:105560001F3A9FED1F6A9FED1F4A9FED1F5ADFED07
:105570001F3ADFED1F4ADFED1F5AA6EEC36AE6EEC3
:10558000A34AA6EE864AB7EE006AA6EE845AA6EEB5
:10559000A46AE6EE855AC5EE866AB4EEE77AF1EEC5
:1055A00010FA48BFDFED147AF5EEC00A48BF77EE77
:1055B000E66AF1EE10FA48BFDFED107AB5EEC00AE8
:1055C00048BF77EEE66AF1EE10FA48BFF1EE666A80
:1055D000B0EE660A7047DFED076ADEE739094E3D37
:1055E000E3B59E3E88FA163E45FE7F3F99FB243F79
:1055F00069A2163EA7DFA834DB0FC93FDB0F494085
:10560000DFED317A30EE277AFDEEC76A16EE903A7A
:105610002033402B02D99FED2D0A7047B4EEE70AE4
:10562000F1EE10FA4DDD9FED2A6ADFED2A6A01E006
:10563000B0EE677AB4EEE67AF1EE10FA77EE467ADB
:10564000F6DC9FED257AF4EEC77AF1EE10FA35D547
:10565000DFED1F6A9FED217A01E0F0EE407AF4EE73
:10566000C77AF1EE10FA37EEA60AF6D4DFED167A15
:10567000B4EEE70AF1EE10FA1BDCDFED197AB4EEB6
:10568000E70AF1EE10FA44BFDFED137A37EEC00AF5
:1056900060EE006A9FED136A9FED137ADFED137AD7
:1056A000A6EE867A20EE266AE6EE877AA6EE270A2E
:1056B0007047DFED0F7A37EEC00AE9E7B0EE670A10
:1056C000D4E7F0EE477ABCE7DB0FC93F00000000EB
:1056D000DB0FC940E4CB1641DB0F49C0E4CB16C158
:1056E000DB0FC9BF92E741B99730083C15A82ABE25
:1056F000DB0F4940FDEEC07A17EE903A2033402B85
:1057000051D8DFED2D7AB4EEE70AF1EE10FA50DD54
:10571000DFED2A6A9FED2A7A01E0B0EE670AB4EE67
:10572000C70AF1EE10FA70EE667AF6DC9FED257A84
:10573000F4EEC77AF1EE10FA38D5DFED206A9FED6E
:10574000227A01E0F0EE407AF4EEC77AF1EE10FA38
:1057500037EEA60AF6D4DFED1D7AB4EEE70AF1EED5
:1057600010FA1BDCDFED1A7AB4EEE70AF1EE10FA5C
:1057700044BFDFED147A37EEC00A60EE006A9FED99
:10578000156A9FED157ADFED157AA6EE867A20EE82
:10579000266AE6EE877AA6EE270A7047DFED067ADC
:1057A00037EEC00AE9E79FED0E0A7047B0EE670AD0
:1057B000D1E7F0EE407AB9E7DB0F4940DB0FC94093
:1057C000E4CB1641DB0F49C0E4CB16C1DB0FC93F68
:1057D000DB0FC9BF92E741B99730083C15A82ABE34
:1057E0000000000010B507EE901A2DED028BB8EE08
:1057F000678ADFED227A28EE008A044628EE278A9F
:10580000B0EE480A1CF04CFEF0EE408AB0EE480ABA
:105810001CF0A8FDF7EE007A9FED197AF0EE675ABA
:10582000E8EE875A0023A361B0EE676AC7EEA56A67
:1058300063612362E361A3626362A8EEC76ABDECA1
:10584000028B77EEC07AB6EE007AF8EE005A27EEB9
:10585000877A20EE250A27EE267A26EE266A67EE5C
:10586000A67A20EE260A84ED046AC4ED017A84ED5E
:10587000007A84ED027A84ED030A10BD27D4D23673
:10588000F304353F10B44C09012250F8243001F0E4
:105890001F0102FA01F10B4340F824305DF8044B7C
:1058A000704700BF4B0901F01F0150F8232001236E
:1058B00003FA01F1114214BF18460020704700BFDF
:1058C0000C4B984213D0A3F5806398420FD003F598
:1058D000804398420BD003F58063984207D003F5CC
:1058E0008063984203D0044B186840087047024B0D
:1058F000186870470004014014580020F0B5774B39
:10590000774A87B01968914200AF00F0DB8000232E
:10591000744A3B607B60136843F48033136003E098
:105920003B68B3F5A04F09D0136803F400337B60E4
:105930003B6801333B607B68002BF1D0694B1B68EF
:1059400013F4003318BF01237B607B68012B7BD0ED
:10595000654D644B654AEA606549586F654A086061
:10596000AA605E6B644C654A654826F080065E63FB
:105970005E6F46F080765E67196B0C431C63596B53
:105980005963996B9963196C41F05B5141F47B1138
:1059900041F41F6141F00F011964596C07F11804BB
:1059A0000A4348F2FF715A6444F8101D002621464C
:1059B0000123FB733E737E73BE730FF0EBFD214634
:1059C0004FF6FF734F48BB600FF0E4FD4FF6FF73D7
:1059D00021464D48BB600FF0DDFD21464B480FF0DE
:1059E000D9FD21464A480FF0D5FD214649480FF020
:1059F000D1FD214648480FF0CDFD214647480FF024
:105A0000C9FD214646480FF0C5FD20460FF00EFEA9
:105A1000444B454C1B68BA6844484549A4FB0343C2
:105A20009B09A0FB0202013B920CB3F1807F0A604C
:105A300007D2404AF0200721536085F82300966082
:105A400011601C37BD46F0BD264B3B4C1A6C3B49E0
:105A500042F080521A6420680A69CD68496940F4AE
:105A600040402060986898609868120640F40040B2
:105A7000986042EA8512986842F48002490842F030
:105A80001902013942EA014240F4A05098605A607C
:105A90001A6842F080721A601A689201FCD528498F
:105AA000104A40F205700860996821F0030199607E
:105AB000996841F002019960936803F00C03082B88
:105AC000FAD145E700221A6062B61E4B1B6883F3C9
:105AD00008881D4B1B689847FEE700BFFCFF0120AC
:105AE000EFBEADDE0038024000ED00E00005FA0533
:105AF000346E002000000008FF916700335F07004C
:105B0000000002400004024000080240000C024075
:105B1000001002400014024000180240001C024025
:105B20000020024014580020D34D621083DE1B4336
:105B3000E475002010E000E00070004084000020C8
:105B4000003C02400000FF1F0400FF1F08B5054B8A
:105B50001B6803B19847044B044A1A6072B6FEF7FB
:105B6000F7FC00BF34510020FCFF0120EFBEADDE8A
:105B700008B5034B1B6803B1984772B6FEF7E8FC03
:105B800034510020F8B50468C4F30D0405460E46F0
:105B900004B32F680FF0EAFC092840F08980464CD6
:105BA000236923F440732361236943F40073236161
:105BB000236943F0010323613E600FF0D7FC2369A2
:105BC000092823F00103236172D12B6804332B6071
:105BD0000020F8BD394B3A4A93422CD902F5804255
:105BE000934227D902F5804293422BD902F5804295
:105BF000934229D902F58032934227D902F5003227
:105C0000934225D902F50032934223D902F500329E
:105C1000934221D902F5003293421FD902F5802226
:105C200093421DD9B3F1016F1CD305200DF002FF83
:105C3000FFF79EFF08240FF099FC092814D04FF0BD
:105C4000FF30F8BD1024F6E71824F4E72024F2E72B
:105C50002824F0E73024EEE73824ECE74024EAE794
:105C60004824E8E75824E6E7134F3B6923F44073E0
:105C70003B613B6943F400733B613B6923F0F803EC
:105C80003B613B6943F002031C433C613B6943F4C5
:105C900080333B610FF06AFC3B6923F002033B61F8
:105CA0003B69092823F0F8033B613FF472AFC6E774
:105CB0006FF00100F8BD00BF003C0240004000084A
:105CC000FF3F0008F8B504460D468E180027B54280
:105CD00001D12069F8BDE368591CE160234415F83F
:105CE000012B1A720429F2D1206918B9A168204643
:105CF000FFF748FF2061E760E9E72DE9F04FDFF8A3
:105D00005C91514F8DB00326A7EB090718220DEBCC
:105D1000020000211EF090FC4C4BCDF81890079724
:105D20001A69002A04DA4A4A5A6002F188325A6033
:105D300001228DF82C20F322DA60464B464C18687D
:105D40009A8804909B79ADF8142004A9072206A82C
:105D50008DF81630FFF7B6FF072204A94FF6FF7043
:105D6000FEF700FBDFF8F8B080464FF0000A5C4514
:105D70003BD30CAC002524F82C5D0222214606A85A
:105D8000FFF7A0FF022221464046FEF7EBFA40BA99
:105D9000C043ADF80800022202A906A8FFF792FF4F
:105DA000099878B108ABC0F10402294618441EF0E6
:105DB00043FC0A9818B9089906A8FFF7E3FE0023E8
:105DC0000A9009939DF82C300A9A23B11F490B6958
:105DD00043F000430B61013E2FD0002A96D1FEF71D
:105DE000E1FF60B30DB0BDE8F08F65888DF80DA0C0
:105DF000C5F30B05AA1DADF808202288C2F30B01DC
:105E0000120BADF80A108DF80C2002A9062206A884
:105E1000FFF758FF062202A94046FEF7A3FA616881
:105E200080462A4606A8FFF74DFF616840462A468D
:105E3000FEF798FA1434804699E7002ACFD005205F
:105E40000DF0F8FDFFF794FE00800008003C0240D2
:105E500023016745344D030888010008004000080D
:105E60005C0500082DE9F04F7A4C54F8204083B0CF
:105E7000002C00F0EA80D4F85C90B9F1000F00F03B
:105E8000E680D9F81050D9F80470734EA16004F17F
:105E900062012660616104F262264FF40071A6611E
:105EA000E1602161A765A0464DB3DFF8B4C14FF0B2
:105EB000000E61464E68B54201F11C0106D00EF19C
:105EC000010EBEF1100FF5D14FF0000ECEEBCE0E4D
:105ED0000CEB8E01DFF884C10E69DCF830E04FF086
:105EE0000C0A4EEA060E461CCCF830E081F818A0E9
:105EF0004E76D9F80810A163043767652563054617
:105F0000D9F80C001F46164600283CD0DFF850C1D7
:105F1000002163465A68904203F11C0303D001310B
:105F20001029F7D10021C1EBC1010CEB81014B4BD2
:105F30000A69186BDFF82CE1104318630B20087610
:105F4000681C4876186B024399F81F001A6383098E
:105F500091F80DC08DF80530002201234C61C1F885
:105F600008E001A88DF806208DF807308DF804C0F0
:105F700015F0AEFCA36DD9F80810D9F80C206263B7
:105F80000433E163236594F8610000F003FF824667
:105F900094F8600000F0FEFE834699F81C0000288B
:105FA00050D1380739D4B2070ED5BAF1000F0BD053
:105FB0000B226B1C8AF806208AF80730504699F8A5
:105FC0001D20222100F0ACFFF30716D4A36B83B988
:105FD00099F81E208DF8042099F820208DF80630BD
:105FE00001A8930901228DF805308DF8072015F0DE
:105FF0006FFC404603B0BDE8F08FBBF1000FE5D069
:1060000001350C238BF807508BF80630584699F869
:106010001D20222100F084FFD8E70135EDB2BAF14E
:10602000000F04D00B238AF807508AF8063017F0C7
:10603000100F50460CBF1221022199F81D2000F0CC
:106040006FFFC3E715F022FCABE7A046D1E7C846D7
:10605000CFE700BFBC2F00203C4D030800380240B2
:1060600004190020C54A01080348D0F8AC3113B127
:1060700000F5D27018477047041900200348D0F883
:10608000903113B100F5C47018477047041900200F
:106090000348D0F8743113B100F5B6701847704753
:1060A000041900200348D0F8583113B100F5A87046
:1060B00018477047041900200348D0F83C3113B149
:1060C00000F59A7018477047041900200348D0F86B
:1060D000203113B100F58C70184770470419002067
:1060E0000348D0F804310BB1FC301847704700BFAB
:1060F000041900200348D0F8E8300BB1E03018470D
:10610000704700BF041900200348D0F8CC300BB111
:10611000C4301847704700BF041900200348D0F866
:10612000B0300BB1A8301847704700BF04190020E9
:106130000348D0F894300BB18C301847704700BF3B
:10614000041900200248836F0BB170301847704764
:10615000041900200248C36D0BB154301847704732
:10616000041900200248036C0BB1383018477047FF
:10617000041900200248436A0BB11C3018477047CD
:10618000041900200248836803B11847704700BF14
:10619000041900201549164B1648CA6810B44C69FA
:1061A0001549B2FBF4F203FB02F30360D1F8882037
:1061B000124B134C42F47002C1F888201A68002078
:1061C00042F001021A6098601A6822F0847222F488
:1061D00080321A605C601A684FF0006422F48022FA
:1061E0001A60D8608C605DF8044B70478400002012
:1061F00040420F001458002000ED00E0003802403B
:1062000010300024044B4FF4F07002210A22D860B1
:1062100059611A61FFF7BEBF84000020436A82699A
:10622000F0B4D154436A0469426B0133A34228BFDE
:1062300000234362FAB1116811F0010101D0F0BCF2
:106240007047856A1768866927F001072E449D42CA
:106250001760D6600BD3641B546081621368002101
:1062600043F0010380F84C10F0BC136070475D1BD5
:1062700055608362F2E7826DD36843F08003D36098
:10628000DDE700BF026B10B462B1836CC268446981
:10629000D11A013B615C5DF8044B08BF134683646F
:1062A000C8B27047016A4369C4685B5C0131A142AE
:1062B00028BF114601625DF8044BD8B2704700BF99
:1062C000436B13B190F84C007047836A406A181A08
:1062D000B0FA80F040097047416A836A99420AD354
:1062E000CB1A416B026961B14968501E0B4483426D
:1062F0000AD2C01A704702691144CB1A416B0029B7
:10630000F2D1501EC01A704700207047036B43B192
:10631000826C5B6893422FBF981AC0689B1AC018A2
:106320007047C269036A9A422FBFD01AC0688018AA
:10633000C01A70470A4B30B503F1100493F90020DE
:106340005D78072AC8BF143A811804330D7313F817
:10635000025C855413F8012C0A76A342EED130BDBD
:10636000644D030803682DE9F041DF691FB13B4626
:10637000BDE8F0411847002A164611DD04460D46D7
:106380000E4400E023689B68204698470028F9D017
:10639000236815F8011B1B6820469847AE42F1D1CF
:1063A000BDE8F08110B424211824322200230470A7
:1063B00041708270C3705DF8044B70472D234370A9
:1063C0002E2303712F23C371704700BF30B445687B
:1063D00015B12B68AC885C83036840F2E93001E0BA
:1063E000002830D01C89013814F0020F80B2F7D099
:1063F00089B2998140F2E93100E021B3188901396D
:1064000010F0010F89B2F8D0998940F2E93100E02B
:1064100019B31889013910F0020F89B2F8D092B27D
:106420009A8140F2E93200E0BAB11989013A11F0DB
:10643000010F92B2F8D09B8915B12B68AA881A83F4
:10644000012030BC70470A498B42DED10948418B9C
:10645000013189B24183418BD7E7054A9342EBD1A1
:10646000044A538B01339BB25383538BE4E700BF41
:1064700000380040DC73002030B50446806D617147
:106480008389A26823F400531B041B0C838185B00D
:10649000A379009213F004022ED04FF4805213F02F
:1064A0000203ADF804203CD1ADF806304FF4806310
:1064B0000022ADF8083011F00103ADF80C2026D110
:1064C000ADF80A3008238A07694648BFADF80A309C
:1064D0000FF0F6F8A379A26D13F0080F938A1BD181
:1064E00023F008031B041B0C938293899BB243F493
:1064F0000053938105B030BD13F00203ADF80420C2
:1065000012D04FF400551346ADF80650D0E70423DF
:10651000ADF80A300C23D6E79BB243F00803938210
:10652000E3E74FF40053BFE7ADF80630C0E700BF24
:1065300010B50446806DA160838923F400531B04C9
:106540001B0C8381A37984B013F00402009133D033
:106550004FF4805213F00203ADF804203CD1ADF8A3
:1065600006304FF480636279ADF80830D1074FF000
:106570000003ADF80A30ADF80C3045BF0423ADF888
:106580000A3008230C236946920748BFADF80A3049
:106590000FF096F8A379A26D13F0080F938A16D125
:1065A00023F008031B041B0C938293899BB243F4D2
:1065B0000053938104B010BD13F00203ADF8042022
:1065C0000DD04FF400511346ADF80610CBE79BB247
:1065D00043F008039382E8E74FF40053BFE7ADF8B8
:1065E0000630C0E770B5054640680E46194610B142
:1065F00003688088588346F08006286840F2E933B3
:1066000000E0EBB10489013B14F0020F9BB2F8D01B
:10661000B3B2838140F2E93300E08BB10489013BDE
:1066200014F0010F9BB2F8D0838913460022FEF7C5
:10663000CFFA6B6813B11A689B881383012070BD71
:10664000044B9842F1D1044C638B01339BB26383BA
:10665000638BEAE700380040DC7300202DE9F04F3F
:10666000013085B0C3B203930B4602918B4C8C4E24
:10667000002B00F099808B4D8B4FDFF830921AF091
:1066800051FD4FF4FA7A4FF0100C4FF47A70D9F8AC
:106690000430C3F30803002B40F0DE80EFF31183D6
:1066A000002B40F0D9802968A26800BF2B6899426E
:1066B000F9D1D7F800E000FB0EF39B1AB3FBFEF311
:1066C00000FB01314FF0010E0191D9F80430C3F302
:1066D0000803002B40F08780EFF31183002B40F07C
:1066E00082802B68A16800BF2A689342F9D1D7F84D
:1066F00000B000FB0BF2521AB2FBFBF200FB0323CB
:10670000019A9B1AB3F57A7FDFD3BAF1010ABED1A1
:10671000039B002B40F0BD804FF47A7ADFF88C9118
:1067200050464FF0100CD9F80430C3F30803002B87
:1067300075D1EFF31183002B71D12968A26800BFD6
:106740002B689942F9D1D7F800E000FB0EF39B1AB1
:10675000B3FBFEF300FB01314FF0010E0191D9F8BC
:106760000430C3F3080313BBEFF31183FBB92B68A9
:10677000A16800BF2A689342F9D1D7F800B000FBA6
:106780000BF2521AB2FBFBF200FB0323019A9B1A95
:10679000B3F57A7FE3D3BAF1010AC4D1029B013B7E
:1067A0000293002B7FF467AF05B0BDE8F08FEFF3E5
:1067B00011888CF31288A1682368DB0344BFC6F8F4
:1067C00000E0A1682B6832685FFA88F888F31188C6
:1067D000D7F800801A4400FB08F35B1AB3FBF8F308
:1067E00000FB0233D2E7EFF311888CF31288A16823
:1067F0002368DB0344BFC6F800E0A1682B68326859
:106800005FFA88F888F31188D7F800801A4400FBF3
:1068100008F35B1AB3FBF8F300FB023370E7EFF306
:1068200011828CF31288D4F808E02368D90303D5C9
:1068300001233360D4F808E02B683168D2B282F3C8
:1068400011883A68194400FB02F3A3EB0E03B3FB73
:10685000F2F300FB01317FE7EFF311828CF3128832
:10686000D4F808E02368D90303D501233360D4F8B2
:1068700008E02B683168D2B282F311883A68194473
:1068800000FB02F3A3EB0E03B3FBF2F300FB0131B9
:1068900018E718461AF0ECFA3EE700BF10E000E0F7
:1068A000DC750020E0750020E475002000ED00E0BC
:1068B000204B5B68C3F3080330B4BBB9EFF311831B
:1068C000A3B91D4B1D4C1868A16800BF1A689042FF
:1068D000F9D11B4B1C684FF47A7202FB04F3591A6E
:1068E000B1FBF4F130BC02FB00107047EFF31182F2
:1068F000102383F3128811498C680B6813F4803FCE
:10690000104B02D0012018608C680B49D2B20D6880
:10691000186882F311880A4B19684FF47A72284478
:1069200002FB01F31B1B30BCB3FBF1F302FB003095
:10693000704700BF00ED00E0E075002010E000E0CF
:10694000E4750020DC7500202DE9F84F8046FFF744
:10695000AFFF254E2549DFF8A0E0254A254D8446A6
:1069600010274FF47A740120DEF80430C3F30803D3
:10697000D3B9EFF31183BBB90B68D2F808A000BFFD
:10698000D1F800904B45F7D1D6F800B004FB0BF9D5
:10699000A9EB0A09B9FBFBF904FB0393A3EB0C0376
:1069A0004345E1D3BDE8F88FEFF3118A87F31288EE
:1069B000D2F808B01368DB0344BF2860D2F808B0EF
:1069C0000B68D5F800905FFA8AFA8AF31188D6F836
:1069D00000A0994404FB0AF3A3EB0B03B3FBFAF307
:1069E00004FB0933DAE700BFE4750020E0750020FE
:1069F00010E000E0DC75002000ED00E02DE9F04F34
:106A0000DFF830C1474A4849484E494D8046102773
:106A100018F1FF38C0F08480DCF80430C3F30803B9
:106A2000002B5CD1EFF31183002B58D10B689468D5
:106A300000BF08688342F9D1D6F800904FF47A700D
:106A400000FB09FEAEEB040EBEFBF9FE00FB03EEFD
:106A5000DCF80430C3F308034FF47A740120FBB967
:106A6000EFF31183E3B90B68D2F808A000BFD1F8A7
:106A700000904B45F7D1D6F800B004FB0BF9A9EB19
:106A80000A09B9FBFBF904FB0393A3EB0E03B3F56F
:106A90007A7FBDD2DCF80430C3F30803002BDFD0CB
:106AA000EFF3118A87F31288D2F808B01368DB037A
:106AB00044BF2860D2F808B00B68D5F800905FFAA0
:106AC0008AFA8AF31188D6F800A0994404FB0AF3E5
:106AD000A3EB0B03B3FBFAF304FB0933D5E7EFF3A6
:106AE000118487F31288D2F808901368D80303D56D
:106AF00001232B60D2F808900B682868E4B284F375
:106B00001188D6F800A04FF47A7400EB030E04FB52
:106B10000AF3A3EB0903B3FBFAF304FB0E3E97E77A
:106B2000BDE8F08F10E000E0E0750020E475002083
:106B3000DC75002000ED00E030B4EFF3118310228B
:106B400082F312880649074C0A680748013200257B
:106B50000A602560DBB2026883F3118830BC70479D
:106B6000E0750020DC75002010E000E038B5254B12
:106B70009C68236B73B1A36D626BCAB1998A1A8842
:106B8000C90592B201D5D20700D438BD4FF6F772CD
:106B90001A8038BDA36D99891A88890692B2EBD5FF
:106BA0009206E9D5E26ACAB1988880B29047E2E7D6
:106BB00099891A880D0692B2E0D51006DED5A26A30
:106BC000616A8A4219D0A1692569885C988001327E
:106BD000B2FBF5F105FB1122A262CFE79B88E269C7
:106BE0006169DBB28B54E269E068A36D0132B2FBEC
:106BF000F0F100FB1122E261BEE7DA6822F08002C8
:106C0000DA60BBE7BC2F002038B5254B5C68236BEE
:106C100073B1A36D626BCAB1998A1A88C90592B221
:106C200001D5D20700D438BD4FF6F7721A8038BDAF
:106C3000A36D99891A88890692B2EBD59206E9D597
:106C4000E26ACAB1988880B29047E2E799891A88C7
:106C50000D0692B2E0D51006DED5A26A616A8A42BC
:106C600019D0A1692569885C98800132B2FBF5F1E1
:106C700005FB1122A262CFE79B88E2696169DBB262
:106C80008B54E269E068A36D0132B2FBF0F100FBC6
:106C90001122E261BEE7DA6822F08002DA60BBE727
:106CA000BC2F0020436B826A816930B41C68456A3E
:106CB00024F001041144AA421C60D9600DD301697B
:106CC00000248A1A5A6084621A68002142F0010284
:106CD00080F84C1030BC1A607047AA1A5A6085625E
:106CE000F2E700BF03682DE9F041DF691FB13B46C1
:106CF000BDE8F0411847002A164611DD04460D464E
:106D00000E4400E023689B68204698470028F9D08D
:106D1000236815F8011B1B6820469847AE42F1D145
:106D2000BDE8F08103689B69184700BF03685B6991
:106D3000184700BF03681B69184700BF0368DB687A
:106D4000184700BF03685B68184700BF03681B68EB
:106D5000184700BF38B50C46097849B105460134DB
:106D60002B6828461B68984714F8011B0029F7D1A7
:106D700038BD00BF064B53F820302BB11A689B88F2
:106D800051690B4201D1138370475383704700BF91
:106D90005C86002010B50409013C032C17D80D4B6C
:106DA00033F8142000F00F0042FA00F313F001034F
:106DB0000DD0012303FA00F0013810401BF0E4F875
:106DC000054A064B125D104403EBC00010BD0020C5
:106DD00010BD00BF206D03081C6D03080C7400205B
:106DE0002DE9F04F4A484B494B4B4C4C4FF0010AB0
:106DF0004FF002094FF004084FF0080C4FF0100E4E
:106E000020274026802530F8022B12F0010F03D0F6
:106E10001960A3F804A0083312F0020F03D0196020
:106E2000A3F80490083312F0040F03D01960A3F8FC
:106E30000480083312F0080F03D01960A3F804C0CF
:106E4000083312F0100F03D01960A3F804E00833E0
:106E500012F0200F02D019609F80083312F0400F0B
:106E600002D019609E80083312F0800F02D01960A2
:106E70009D80083312F4807F05D04FF4807B196029
:106E8000A3F804B0083312F4007F05D04FF4007B60
:106E90001960A3F804B0083312F4806F05D04FF4E2
:106EA000806B1960A3F804B0083312F4006F05D0AA
:106EB0004FF4006B1960A3F804B0083312F4805F3C
:106EC00005D04FF4805B1960A3F804B0083312F4C6
:106ED000005F05D04FF4005B1960A3F804B00833DD
:106EE00012F4804F05D04FF4804B1960A3F804B022
:106EF0000833D20B04D04FF4004219609A80083353
:106F000001F58061A1427FF47EAFBDE8F08F00BF44
:106F1000206D0308000002400C74002000100240A5
:106F200000286AD003682DE9F04F03F13F4404F5CF
:106F30007E045F4EA40A0125345D04F01F06640937
:106F4000032C05FA06F559D0042C00F0AC80022C75
:106F500059D08588B5FA85F0C0F11F0080B2C40809
:106F600003EB840400F00700266A80000F278740A7
:106F700026EA07062662276A01F003068240701E91
:106F80003A430128C1F3810CC1F300182262C1F316
:106F900041113DD90024224601274FF0030E03E0A2
:106FA000102A04F1020426D007FA02F0A84302F1E5
:106FB0000102F5D1D3F800C00EFA04F0C04300EA94
:106FC0000C0CC3F800C0D3F8008006FA04FC4CEAAD
:106FD000080CC3F800C0D3F80CC000EA0C00D8605D
:106FE000D3F80CC001FA04F040EA0C00102AD86073
:106FF00004F10204D8D1BDE8F08F70472D4C266C07
:1070000035432564A5E72B4C666C35436564A0E7E2
:10701000002002464FF0010E4FF0030904E0013258
:10702000102A00F102003CD00EFA02F737EA0504FC
:10703000F5D1D3F800A009FA00F4E4430AEA040AFF
:10704000C3F800A0D3F800B006FA00FA4AEA0B0A27
:10705000C3F800A0D3F808A004EA0A0AC3F808A0FD
:10706000D3F808B00CFA00FA4AEA0B0AC3F808A0F1
:10707000D3F804A02AEA07075F60D3F804A008FA4F
:1070800002F747EA0A075F60DF683C40DC60DF68C0
:1070900001FA00F401323C43102ADC6000F10200E6
:1070A000C2D1BDE8F08F034C266B3543256350E712
:1070B000E464030800380240002855D0026802F159
:1070C0003F4303F57E032DE9F04F9B0A544DEB5CE3
:1070D00003F01F055B090124032B04FA05F444D0D7
:1070E000042B00F09780022B44D001F00306731E9E
:1070F000012BC1F3810CC1F300188588C1F3411144
:107100003DD90024234601274FF0030E03E0102B46
:1071100004F1020426D007FA03F0A84303F10103A7
:10712000F5D1D2F800C00EFA04F0C04300EA0C0C0E
:10713000C2F800C0D2F8008006FA04FC4CEA080C41
:10714000C2F800C0D2F80CC000EA0C00D060D2F83F
:107150000CC001FA04F040EA0C00102BD06004F1DE
:107160000204D8D1BDE8F08F70472E4B1D6C2C4324
:107170001C64BAE72B4B5D6C2C435C64B5E70020C4
:1071800003464FF0010E4FF0030904E00133102BCA
:1071900000F102003CD00EFA03F737EA0504F5D1FE
:1071A000D2F800A009FA00F4E4430AEA040AC2F89B
:1071B00000A0D2F800B006FA00FA4AEA0B0AC2F8B8
:1071C00000A0D2F808A004EA0A0AC2F808A0D2F87F
:1071D00008B00CFA00FA4AEA0B0AC2F808A0D2F882
:1071E00004A02AEA07075760D2F804A008FA03F7B8
:1071F00047EA0A075760D7683C40D460D76801FA6D
:1072000000F401333C43102BD46000F10200C2D1E2
:10721000BDE8F08F034B1D6B2C431C6365E700BF7B
:10722000E46403080038024018B10368828809B991
:107230005A8370471A83704710B40A4B0A4A1C7865
:1072400001238340234052F8200029B9B3FA83F187
:1072500049095DF8044BE7E7191C18BF01215DF8E7
:10726000044BE1E7588600205C8600202DE9F041C0
:107270000B4E346873691C400FD0DFF8288001275B
:10728000B4FA84F3C3F11F0307FA03F558F8230097
:1072900003689847AC437561F2D1BDE8F08100BF47
:1072A000003C0140947500202DE9F0410B4E3468FC
:1072B00073691C400FD0DFF828800127B4FA84F3EB
:1072C000C3F11F0307FA03F558F823000368984732
:1072D000AC437561F2D1BDE8F08100BF003C0140D4
:1072E000947500202DE9F0410B4E346873691C4001
:1072F0000FD0DFF828800127B4FA84F3C3F11F030D
:1073000007FA03F558F8230003689847AC43756102
:10731000F2D1BDE8F08100BF003C0140947500202F
:107320002DE9F0410B4E346873691C400FD0DFF833
:1073300028800127B4FA84F3C3F11F0307FA03F589
:1073400058F8230003689847AC437561F2D1BDE853
:10735000F08100BF003C0140947500202DE9F04110
:107360000B4E346873691C400FD0DFF8288001276A
:10737000B4FA84F3C3F11F0307FA03F558F82300A6
:1073800003689847AC437561F2D1BDE8F08100BF56
:10739000003C0140947500202DE9F0410B4E34680B
:1073A00073691C400FD0DFF828800127B4FA84F3FA
:1073B000C3F11F0307FA03F558F823000368984741
:1073C000AC437561F2D1BDE8F08100BF003C0140E3
:1073D00094750020084A094808B5536C43F480436B
:1073E0005364002140221DF027F9054B4FF0FF3276
:1073F0001A60C3F8032008BD0038024094750020CD
:10740000D47500202DE9F041044618460D46164675
:1074100098461AF00FF92768E6722844A0722946A8
:107420007D69434632462046AC46BDE8F0416047A0
:10743000036810B504461B689847236820469B687C
:107440009847A37B0133A37310BD00BF03680A7A7A
:10745000591C01601A70704738B50B4C23688BB10A
:107460005A68821A002A054604DA0CE05A68AA1AF9
:10747000002A07DB9A68226018461A68904723683A
:10748000002BF3D138BD38BDC04300200B4B002288
:1074900010B4027203F1C004032102E0072A09DCE0
:1074A0009979890702D51979815401329C4203F1F7
:1074B0001803F3D15DF8044B704700BF446C030818
:1074C00012230370704700BF01233421352241701D
:1074D000427103700371704770B54E6805463046BF
:1074E0001AF0A8F831460446024628681DF07FF8D5
:1074F0002A68131901333B212B60115570BD00BF61
:1075000008B508F081FCFEF733FB00BF038A2DE9C4
:10751000F0478589ADB21D4029D00F4606464FF091
:1075200000484FF00009B5FA85F328FA03F2D24378
:1075300091B21B3B15403182042B16D8DFE803F0D3
:107540003129211903007B6A002B32D003F1FF3A65
:107550001FFA8AFAC7F824903C6A34B1236820469F
:10756000514698476468002CF8D1002DDBD1BDE866
:10757000F0873868716B036889B29847002DD2D1C3
:10758000F5E77868B16B036889B29847002DCAD1D6
:10759000EDE7B868F16B036889B29847002DC2D156
:1075A000E5E7F868316C036889B29847002DBAD1D5
:1075B000DDE7F36A1FFA83FACEE700BFF0B5464B6A
:1075C0001A6883B0012351024449009358BF03F164
:1075D0008053096858BF0093D7005CBF43F0100385
:1075E00000938E0744BF43F0C60300930C0744BFCB
:1075F00043F020030093100644BF43F4406300931C
:10760000D1053749097848BF43F0006301F0EF0026
:1076100048BF009308286D4651D00E294FD03148FD
:10762000009B0078D70454BF43F0884343F0C8431D
:10763000002843F400530CBF07200F20960648BFD4
:1076400043F48073540748BF43F4003343F40024E9
:107650005205009402D5244A1279A2BB182936D0CB
:1076600001900027012639462846FCB2FEF71AF998
:1076700060B11E4B002203F5D87103E08B420FD09E
:1076800013F80C2C944203F10C03F7D10137242F8B
:10769000E9D195E80300164B83E8030003B0F0BD81
:1076A0007A0904F01F0455F8223006FA04F4013771
:1076B00023EA0404242F45F82240D4D1E9E743F417
:1076C00080530093ABE743F4C0130093C6E7009BDD
:1076D00043F060730093C3E7386E002038510020F8
:1076E00028220020405800208882002008480308F3
:1076F000A41C00202DE9F84F4E014FF0000B174D50
:107700008146904606F120075C46594628465FFAB6
:107710008BFAFEF7C7F8C0B1A64215D8A74213D915
:1077200000200F4A014604E00131242914D012F848
:107730000C0C504502F10C02F6D10A4B01EB410151
:1077400003EB81014846C04701340BF1010BBBF14B
:10775000240FDAD1BDE8F88F0021F3E7A41C002044
:1077600008480308FC47030800210A4A0B4604E0C6
:107770000133242B0BD012F80C1C884202F10C02AE
:10778000F6D1054803EB430300EB8300704700206C
:10779000704700BF10480308FC47030800210A4A4D
:1077A0000B4604E00133242B0BD012F80C1C88424A
:1077B00002F10C02F6D1054803EB430300EB830012
:1077C00070470020704700BF08480308FC470308C3
:1077D00008B501210220FFF72FFD094B1B7803F0AC
:1077E0000503052B08D000210120FFF725FD00210E
:1077F0000846FFF721FDFEE708F0B6FBF3E700BF00
:10780000B82F0020022810B428BF0220064C074BD6
:10781000207000EBC001064A5DF8044B00EB8100CC
:1078200003EB4000106070475A8400203083002032
:107830004820002008B516F019FDFEF75EFABDE8F5
:10784000084016F0FBBC00BF38B5384B5A899989FF
:10785000914224BF00225A81198ADA89914224BFB9
:107860000022DA81DA788AB1072A0FD0304C314809
:10787000A27801210025062A01709970DD714CD98A
:107880002379DFED2D6A002B36D138BDDA799B786C
:10789000284807EE103A002A44D0DFED276A017825
:1078A000234CB8EEC77A07EE901AA278F8EEE77A82
:1078B00027EE267A062A67EE877A2BD81F4B03EB32
:1078C0008203D3ED006AF4EEE76AF1EE10FA10DD00
:1078D000C6EE877AFDEEE77A17EE903A102BA8BF36
:1078E0001023012BB8BF0123DBB28B4228BF0B460C
:1078F00003702379002BC8D0013A032AC5D8B7EE0C
:10790000000A80EE260A1AF07FFD2388984238BFCD
:10791000208038BDDFED086AD5E7DFED097AB0EEEB
:10792000677ACBE7DFED076AB9E700BFE8480020D8
:1079300018580020347E00206F120338744D03085D
:107940006F12833A6F1203392DE9F047AD4FAE4EF7
